:040000050000FDC139
:020000040000FA
:1000000028430020B96F000001CA011001CA011085
:1000100001CA011001CA011001CA011001CA011070
:1000200001CA011001CA011001CA011001CA011060
:1000300001CA011001CA01103FCA011000280000C6
:100040000328000001290000022900002000000010
:0C0050000A000000A80800206D1C000041
:100100003C0000000000000000000000340100007E
:1001100000000000000000000100000000000000DE
:1001200000000000000000000000000001000000CE
:100130000000000008000000000000003400000083
:100140000000000000000000680100000000000046
:10015000000000000100000000000000010000009D
:100160000000000000000000080000000000000087
:1001700030000000000000000000000098010000B6
:10018000040000000000000001000000FFFFFFFF6E
:10019000FF00000001000000080000000000000057
:1001A0002C0000000000000000000000C40100005E
:1001B000040000000000000001000000FFFFFFFF3E
:1001C000FFFFFFFF080000000000000034050000F2
:1001D000E401000099A1011095A70110A5C201102A
:1001E00009B2011045B80110000000000000000035
:1001F0002F000000280000000000000000000000A8
:10020000140200000000000000000000FFFFFFFFDC
:1002100000000000080000000000000030050000A1
:100220003002000069C201106DC101101FC201102F
:1002300095BA011000000000000000002D00000031
:10024000300500005402000075C20110A9B601106B
:100250009DBF011049B60110000000000000000021
:100260002E0000002400000000000000000000003C
:1002700080020000000000000000000000000000FC
:100280000800000000000000240000000000000042
:1002900000000000A40200000000000000000000B8
:1002A0000000000008000000000000002400000022
:1002B0000000000000000000C80200000000000074
:1002C0000100000000000000080000000000000025
:1002D00000000000100800200400000000000000E2
:1002E000000000002000000070010000300000004D
:1002F0001C02000030080020040000000000000084
:10030000000000000C000000300400001800000095
:100310004002000038080020040000000000000037
:100320000000000024000000480400001800000045
:100330000000000078080020040000000000000019
:100340000000000010000000A00100002C000000D0
:10035000CC01000080080020040000000000000024
:1003600000000000200000006402000024000000E3
:10037000FFFFFFFFA00800200400000000000000B5
:100380000000000028000000880200002400000097
:10039000FFFFFFFFC808002004000000000000006D
:1003A00000000000580000003C0100003400000084
:1003B000FFFFFFFFD0080020040000000000000045
:1003C00000000000100000006004000018000000A1
:1003D000FFFFFFFFD808002004000000000000001D
:1003E000000000001C000000AC020000240000001F
:1003F000FFFFFFFFE00800200400000000000000F5
:100400000000000038000000F40100002800000097
:10041000FFFFFFFF4809002004000000000000006B
:100420000000000054000000000100003C0000003B
:100430001800000000000000000000004004000060
:10044000080000000000000018000000000000008C
:100450000000000058040000080000000000000038
:100460001800000000000000000000007004000000
:10047000080000000000000001000000580000001B
:100484000100000000000E0000000F003200000018
:100494000100000018080020000200000000000015
:1004A40001CA011000000000000000000800000064
:1004B40000002300400800200100000088080020FC
:1004C4000800000000000000000000000000000020
:1004D400000000000000000001000000E808002007
:1004E4000600000001000000500900200000000088
:0C04F400000000000002000000000000FA
:0F0502002900010025002D002E002F000100010F
:1005140004000000F86F000000000000000000006C
:10052400000001000000030087C40110380500002A
:10053400380500000000000090000000900000005A
:100544000000000088080020496900002000000025
:10055400D06F0000D86D00000DC30110951A000083
:10056400971A000099C801109BC8011000000000F0
:100574003E1B0000406D0000586D0000286D000017
:090584000800090001000000015B
:10059000000000000000000000000000000000005B
:1005A000E1190000011A0000051900002B1A0000D3
:1005B0004D190000231900007F190000571A000090
:1005C000C16800000D6A0000116A00000800000008
:1005D0002400000018000000280000002000000097
:1005E0003C0000000C00000034000000DFF800F0C8
:1005F00049C10110DFF800F019C20110DFF800F066
:1006000041AC0110DFF800F0CDA00110DFF800F0E0
:1006100085C10110DFF800F0C1C20110DFF800F061
:10062000E3BF0110DFF800F0CDC10110DFF800F0EA
:100630003DC10110DFF800F0DDB20110DFF800F07D
:1006400085B00110DFF800F029AF0110DFF800F0ED
:1006500079B50110DFF800F0C1C10110DFF800F03A
:1006600009B70110DFF800F0D5C00110DFF800F085
:10067000E1B5011020B1082328220021FFF7D2BFE5
:10068000704720B1082330220021FFF7CFBF704709
:1006900038B500F091FF25680DB129682160FFF79A
:1006A000A9FF284632BD70B504460D4626680020D5
:1006B00028601EB9FFF79AFF25600DE0FFF796FF4F
:1006C00000E0366831680029FBD1AE4203D1FFF764
:1006D00091FF002070BD3560FFF78CFF012070BDD9
:1006E0000022DFF8541C01EB4211CB7F1B0605D51D
:1006F000B1F91C30834201D108467047521C082AC8
:10070000EFDB0020704770B50646FFF76FFFDFF89C
:10071000545C0446A87E01001AD0401EA876C0B2E0
:10072000B0B9082100F026FC96B1A86B703001F03A
:100730007CF800F010FE301AB0FBF1F1022938BF4E
:100740000121EC352846FFF765FF2846FFF766FFD5
:10075000204600F065BE10B50446207B00F00F0077
:1007600002280FD100F012FDA168081ADFF8F41B6F
:10077000896BC968800801F57A71814238BFB0F190
:10078000405F00D3002010BD38B5DFF84C0ADFF819
:100790004C2A0168DFF87C4C02EA0105E94301605C
:1007A000A90608D54068800605D54FF4005104F12C
:1007B0004C0001F064F815F4602F08D0206905F4AE
:1007C000602108432061002104F19C00D0E131BD8B
:1007D00070B5FFF70BFFDFF83C4C0646206910F4BC
:1007E000602F27D02069C5012D0EE80748BF0025DE
:1007F00006D4A80748BF012502D4680748BF0225D0
:10080000681D40B200F040FF2069012105F111028E
:100810009140884320613046FFF7ECFE04EB8500F1
:100820004668300009D0206800224FF00063691D3F
:10083000B04702E03046FFF7DDFE206930B104F139
:100840009C00BDE87040002101F019B870BD70B582
:1008500001F024F9DFF80C5BDFF8BC4BAB6A024611
:1008600090071DD4D3E90401104007D0EB629969C9
:10087000084398614FF4804100F07CFBA86A00288F
:1008800047D16E6A002E44D0F068A96B884224D00C
:1008900005F14C00BDE870404FF4805100F0EFBF0F
:1008A0000BB9A86AEAE70020A862D3E904019E69AF
:1008B000024042F0020232439A61626982436261FD
:1008C000E26822EA0100E060194605F13000FFF716
:1008D000EAFE022100F04EFBE3E7B068FFF73BFFC2
:1008E000A86408B1A86CD8E0D6E9040162690243A3
:1008F0006261E26841EA0200E0600020E061B06805
:100900002060E0690028FCD005F12400FFF7C0FE5C
:10091000AE6270BD0020F6E6F8B506461446376EA6
:100920001D4607B1B847A00708D4D6E916012040F4
:1009300029400022914208BF904207D0C6E91A45DB
:1009400006F13800BDE8F240FFF758BEF1BDFEE702
:1009500080B500F084FFDFF8BC2A0146906BD26BB3
:10096000BDE80840104710B5DFF8A84A0FF2311172
:10097000E06B884202D101F0EDF8206404F14C00F4
:10098000BDE81040042100F07ABF80B501F086F880
:10099000DFF8881A084207D0BDE804404FF0005144
:1009A000DFF8100C00F06BBF01BD70B5040073D010
:1009B000A168202001E04968401E79B1C2B26AB145
:1009C0000A8840F603039A421CBF40F604039A4289
:1009D000F1D1E0681822203001F0D8F8A069002198
:1009E000A1616168D9B140F00202E07F002300F00C
:1009F0000700012807D0022809D0042804BF0022DC
:100A00004FF0805306E000224FF0005302E0002236
:100A10004FF08043B4F91C10E0686568A847FFF701
:100A2000E5FDDFF840590646E88E401CC0F30B0098
:100A3000E8860020296BC87705F13000FFF728FE13
:100A40003046FFF7D7FDB5F93610E06800F1B8027F
:100A5000B2F90030994204BF297E00291CD1917857
:100A600009B9016811B90020907016E0AA6B1268EC
:100A700012F1010F10D0DFF8F42B1268B1FBF2F184
:100A8000022938BF01217030FFF7C4FDE068BDE8DE
:100A900070407030FFF7C2BD70BDBDE8704032E6F7
:100AA00038B50D46A807DFF8BC4816D5206BFFF710
:100AB0007CFF206B25F0020510B145F0020109E032
:100AC000680702D4606A002851D004F1EC0000F0FD
:100AD000ACFE042104F14C004AE0680747D5606A87
:100AE00008B1C068A063A06BDFF8E42A41680B7806
:100AF0001360126809788A421CBF8569002D05D0F1
:100B000000224FF000736FF0FF01A847022001F0B0
:100B1000A1F9112001F0B3F901206077A06BE17E0B
:100B2000007C084204BF0E2001F0A9F9A06BDFF899
:100B3000E81840688268002A04BFC068002804D012
:100B40000020C861DFF8D80A086040F2FF70DFF8C3
:100B5000D42A106000208861DFF8C00848610FF2D5
:100B60001900E0631920BDE83240FFF763BD31BDD5
:100B7000BDE8344000F083BE2DE9FF478046880081
:100B800040F1B580DFF8DC57A86B40684068010091
:100B900018BF8047A86BDFF88098406881680029FB
:100BA00004BFC168002914D0D9F81C100029FBD05B
:100BB0000021C9F81C108068010018BF8047A86B8D
:100BC0004068C068010018BF8047DFF8B40A00F031
:100BD0006DFF0020C9F81C0040F60A0ADFF8A40ADD
:100BE000DFF8E07AC9F8000008F10804012000F0FD
:100BF000A5FF0FF25110E863A7F800A0002078804D
:100C0000002100F0B0F900F0A7F9206806467180D5
:100C1000E97E09B1617A99B1018840F602029142F8
:100C200005D1318A4FF60F421140318204E0318BF9
:100C30004FF60F42114031830021617200F06CFFCA
:100C40002068694600F05AFF684600F066FF00E041
:100C50000646706800281CBF01885145F8D17760AE
:100C600040F60301707B00F0F0007073686A8068E2
:100C7000008888421CBF40F60401884202D100204F
:100C8000286417E0208BA8B100206083E06108F1A0
:100C90002C00017801F0F0010170417801F0F001C1
:100CA00041F00101417008F120007860787B00F08C
:100CB000F0007873D9F81C000028FBD00020C9F898
:100CC0001C00012001F08EFB012808D0707B00F091
:100CD000F00040F0010070730FF21900E8634FF666
:100CE000FF322068018A11400182C9F80000BDE886
:100CF000FF870000DFF8D009014200D170470120D2
:100D000010B501F06FFB0128DFF8584608D10FF24B
:100D10003500DFF80417E063DFF8A809086010BDAC
:100D2000DFF8481909683220B0FBF1F1022938BF19
:100D30000121EC342046FFF76DFC2046BDE8104051
:100D4000FFF76CBC2DE9FE4306460C466004DFF855
:100D5000145619D5FFF74AFCEE6AB769B9070ED4E5
:100D60006EB10021B161FFF745FC706848B1B6F97A
:100D70001C10F06876683A460023B04701E0FFF7A0
:100D800039FC24F48044E1E0A0070AD5286BFFF782
:100D90000CFE286B002824F0020401D044F0020469
:100DA000D4E0A00005F1800840F60909DFF81479C5
:100DB00071D5B068018840F60202914205D1028ADD
:100DC0002D2161F30912028204E0028B2D2161F3CF
:100DD00009120283286CB8B1042001F003FB98B11A
:100DE00000F0B8FE296C814228BF401E401A718A6B
:100DF00011EB1030F06040F2D761A0F2EE20884293
:100E000024BF40F6C410F060D6F818C0BCF1000F43
:100E10001CBFDFF8BC188C450DD0787B0F21084231
:100E200004BF708C484506D100224FF000736FF468
:100E300080713046E0470022DFF89818404600F005
:100E400031FD287F50B10220ADF80000684600F067
:100E50002DFEBDF80800A8820020287701206876C2
:100E6000A87E401CA87600206877686A18B119200F
:100E700000F01BFD01E044F00204D6F81480B8F144
:100E8000000F05D000224FF0806300213046C0479C
:100E900024F000545AE095F8200024F0080628B108
:100EA000200703D5002085F820003CE020073CD532
:100EB000002068760120A877002000F03FFE0FF2A6
:100EC000BD00DFF81418DFF86047E86300224046F1
:100ED00000F0E8FC297FE87E81F00101084202D1A0
:100EE0000120E8760FE0A86CB8B100F033FE296C61
:100EF0006A6C401A02EB10306864A96CB0EBC11F39
:100F00000BD300206864A7F8009000F025F80020BB
:100F1000788000F028F8276003E04FF0005100F0DF
:100F200029F800202864344610E0A0040ED5AE6AEB
:100F3000002E1CBF7068002806D0B6F91C10F0689F
:100F4000766800222023B04724F4005414B12146CF
:100F500000F010F8BDE8F783787B00F0F00040F077
:100F6000010078737047387B00F0F0003873002080
:100F70007860704705F14C0000F081BC70B5054603
:100F80000E46B007DFF8DC430BD5206BFFF70DFDF5
:100F9000206B08B1022129E0B0002DD54FF000519F
:100FA00024E0B00028D500F08EFDDFF83007DFF830
:100FB0003067E063307818B905F13800FFF71EFBA1
:100FC000DFF8601600200860022000F0D9FE112032
:100FD00000F0EAFE287C10B90E2000F0E5FE0020AB
:100FE000E083B07840B10020B070042104F14C00DF
:100FF000BDE8704000F043BC70BD30B58DB000F06E
:1010000040FEDFF8E006DFF8E0460168DFF8545301
:1010100041F00201016001A8FFF72CFBA078DFF886
:10102000CC160790002301AA05F14C00FFF706FB40
:1010300001A8FFF726FB0020ADF81C0001AB2078CB
:10104000DFF89426099019210020009005F1800016
:10105000FFF7F8FA01A8FFF70DFBE078DFF890162C
:101060000790002301AA05F19C00FFF7E7FA01A809
:10107000FFF707FB0120ADF81C0001AB6078DFF83B
:10108000742609901A210020009005F1D000FFF786
:10109000D9FA00230022DFF8601605F1EC00FFF713
:1010A000D5FADFF83806E8630DB04FF6FF70A88276
:1010B000012028770020E875E8766877E88385F8CE
:1010C0002000286430BD2DE9F041DFF814660446A5
:1010D00030788EB00F4690461D4618B9FFF78DFF49
:1010E00001203070002F1CBF6760B8F1000F4BD09B
:1010F000C4F80880FFF77AFA7178002942D10121FB
:101100007170FFF777FA35B909A80FF2246114223C
:1011100000F03CFD09AD286820606868E060287C2C
:101120002074A868606101206074688A6082E86841
:10113000010018BFA061A02104F1200001F008FA0D
:101140000823242200216846FFF784FA01208DF845
:1011500018006A46002104F13800FFF77FFA0823DF
:10116000242200216846FFF751FA06946B460022BC
:10117000DFF8881504F17000FFF768FA20460EB01A
:10118000BDE8F081FFF736FA0020F8E738B5FFF741
:101190002DFA7449497E31B1DFF868150C68FFF704
:1011A00029FA204632BDFFF725FA00F0D3FC10F5EE
:1011B0000030DFF8542541F10001A2FB0045DFF8C3
:1011C0000C0502FB015501690020221845EB0103C3
:1011D000184632BD000000000810044020000E0038
:1011E0002DE9F84F04460E4692469B46FFF7FEF95E
:1011F0005C4D8046B5F93400B5F93610401AC0F39D
:101200000B0008286FF0010944DAA88E401CC0F3D7
:101210000B00A886B5F93400ADF80000002046495F
:1012200001EB4017F97F090604D5401CC0B208281D
:10123000F5DB002704F1700000F0F7FABE6087F8D4
:101240001EA0C7F804B02021BDF80000B883FC60E0
:10125000DDE90A23DFF8B40410401940C7E90401AE
:10126000B8340020F87740F6FF76686A00283946DF
:1012700005F1240006D0FFF716FA30B100F05EF851
:1012800040464BE0FFF70FFA40B9A88E3018C0F384
:101290000B00A88600F070F948464AE000F04EF8CE
:1012A000E87F697E084208D0012085F820000020F0
:1012B000E8772877A87E401CA87600F05DF9A86A38
:1012C000002834D1687E18B1192000F0EEFA2EE023
:1012D000687F60BBFFF78AF90446A87F20B1DFF87A
:1012E00000140120887018E0B868FFF734FAA86489
:1012F000B8B100F030F8AA6C121AB2FBF1F2022A6F
:1013000023BFAA6C101AB0FBF1F10121EC3528467D
:10131000FFF780F92846FFF781F92046FFF76AF9C1
:1013200005E02046FFF766F90421FFF723FEBDF92B
:101330000000BDE8F28F0000F00A0020BDF80000B8
:101340002080F87F40F08000F877A07810B100206E
:10135000A07028777047A86BDFF81013C068096881
:1013600070470000001700202DE9F04106460F46A7
:1013700014461D46FFF776F980463846FFF7B0F968
:10138000070003D14046FFF771F90AE0F87F072113
:10139000084209D04046FFF769F90721F87F084263
:1013A000FCD10220002116E07968DFF86403814255
:1013B00002D0796831667860C6E916454046FFF785
:1013C00055F94FF0FF3106F13800FFF71BF9002007
:1013D0003066D6E91A01BDE8F081DCB5DDE90667C3
:1013E0000446CDE90067180008BFDFF82433204623
:1013F000FFF7F6FE002803D500204FF00041DCBDCA
:101400000146204602B0BDE8D04002224FF0E04342
:10141000AAE700000017002000100440020000406E
:10142000BDE87040FFF7E6B801E042F002022DE9A6
:10143000F843DFF8CC42606A0090894603271546DE
:10144000FFF7D4F819F1010F05F0010680460AD123
:10145000A06A002819BFA06AB0F91C90E08E00F1C4
:1014600001090020E0750FFA89F0FFF739F9010052
:1014700070D0A06A814205F0020525D1280003D072
:10148000606A0090002060620122C87FB240104371
:10149000C877FFF7E7F80746002E14BFDFF874029D
:1014A000DFF8740200F002FB00F066F825B906E0F0
:1014B00000F055F800F05BF800980028F8D13846A5
:1014C000FFF7D4F8832747E0009A8A4204F1EC0042
:1014D00016D100F0AAF9280012BF0020606A006847
:1014E000606200F049F8009800F039F800F03FF829
:1014F000009818B32800F6D120E0009A12680092F4
:10150000009AEAB112688A42F7D100F08EF9009889
:1015100000681DB1009A0021116004E00168009A82
:10152000116000210160009003E000F018F800F065
:101530001EF800980028F8D100F01EF8832701E07B
:1015400000F01AF8607F38B9022104F14C0000F075
:1015500096F901E000F010F83846BDE8F283C07F4C
:10156000009940F00400C8776846FFF791B801463B
:1015700004F13000FFF797B84046FFF73BB838B5A5
:1015800000F01AF805465E48407E68B1204600F03B
:101590008DFA044600F04AF804F0FF00012801D15A
:1015A000812032BD022032BD00F040F8012032BD62
:1015B000000000004C1700200446FFF717B80A4649
:1015C0004F49896B884201D00320704709E0000031
:1015D000D02108400A464A49896B884201D003203D
:1015E000704700211046CAE770B545498A6B9042A2
:1015F0006FF07F0411D1487E78B1FEF7F7FF054602
:10160000464800F053FA064600F010F806F0FF00D6
:10161000012802D13002001670BD204670BD0000C6
:101620005100070600000460001004402846FEF741
:10163000E1BF70B50E461546FEF7D8FF832430494A
:101640001EB1022E0DD005D30EE08A6A3AB1896A26
:10165000898B02E00A7F12B9898A298005E08024FB
:1016600003E0497E297000E003245BE050000000A5
:1016700080B50846FFF734F800B1806802BD00006D
:101680000100070601010E0438B5FFF795FF1C495C
:10169000CA7D520702D58B7D9C420FD001228B8AD6
:1016A00002FA04F52B438B820C341D4B1D68A240BB
:1016B00025EA02021A601A6802B90A76BDE83240C9
:1016C000FEF798BF1018002004000020101800201A
:1016D0004F0900004F0800008B090000A10A00001C
:1016E000F71C002000200940106D00005109000087
:1016F000D1070000890700006709000015090000F4
:10170000001700200430044000093D00F1EFFF9F66
:101710001909000001000204010001040100030492
:101720000C100440FEF766FF204670BD000000006C
:10173000FFFFFFFFC4090000000000004F09000088
:1017400001001A01DFF800F021B30110DFF800F00A
:1017500095C00110DFF800F00DA80110DFF800F0CF
:10176000BDBE0110FEE7DFF80001007D70476DE0AF
:1017700038B5FFF7FCFFDFF8F8500446A8680021F1
:10178000FFF7E4FF6969081AA969814238BF0020A0
:1017900084F3118832BD2DE9F041FFF7E8FFDFF84F
:1017A000D0500446A8680121FFF7D0FF0121A9838A
:1017B0000021E9836E6929682A68871B801A711ADB
:1017C000884204D20020A88384F311882BE084F39C
:1017D0001188002406E0A61931460120FFF7BAFF60
:1017E0003F1B0446A742F6D2FFF7C1FF8046E88BB5
:1017F000012804D131460020FFF7ACFF0446A96957
:1018000014F1010F08BF084603D0E01B814238BF26
:1018100008468119FFF7A2FF012028840020A88331
:101820002E6088F31188BDE8F08100218182DFF805
:101830003C10C0684969884204D1DFF85C00006848
:10184000FEF7ECBE7047808A70477047DFF84C1097
:101850000968EFF3118081F311887047F6E7DFF82C
:101860004000806870470000A4010020780100203B
:1018700078010020616280F311882046704738B5F6
:1018800004460D46FFF7EAFF616A2943FFF7F2FFBE
:10189000BDE83240FFF756BF540000004C00000086
:1018A000C8010020816042607047102804D3DFF82F
:1018B0000C101038C1F8000F7047000000E000E085
:1018C00000F04ABEFFF7C2BFDFF89811C20744BF5D
:1018D00001220A60820744BF4FF480720A60400709
:1018E00044BF4FF4803008607047DFF87C21C307A5
:1018F00048BF1160830748BF5160400748BF9160EF
:101900007047000010B504460020D4E90A2347F6CA
:10191000906100F0CDFE0123994228BF4FF0FF30C7
:1019200010BD10B50C4600F00BF9011D201AB0F1E6
:10193000004F05D8081BB0F1004F38BF8C4200D2D1
:101940000C462146BDE810400120CEE72DE9F041CC
:1019500080460A46D8E90A01D8E90C45A0FB02678F
:1019600001FB0277A6196F41340C002244EA0741BB
:101970004046FFF7D6FFC8E90E67BDE8F081F8B52D
:101980000646FFF79FFF0446DFF8E050DFF8E070FF
:101990000120E861FFF798FFF96A096A1420884777
:1019A0003069B0F5802F34BF0421010C0120FFF70E
:1019B0009CFF3A681268232100209047DFF8B4109A
:1019C00001200860DFF8B400016821F4E02141F44F
:1019D000803101600120286084F31188F1BD00008E
:1019E00000F0B8B810B5DFF89000446800F006F8D1
:1019F0006069A169BDE8104008470000012063E765
:101A0000F8B504460D4600F0A5F8D4E90A67324659
:101A10003B4600F04DFE3DB1A6FB002306FB013323
:101A200007FB0033C4E90C23F2BD10B5DFF83C001E
:101A3000DFF84C40002101600121C1612160206874
:101A4000FFF7DCFFDFF848100968096A14208847AF
:101A5000206810BD000080B500F07CF8000C40EA62
:101A6000014002BD04200940182009400000244321
:101A70008401001080022443E4010020002009407A
:101A80002C200940DFF81000C088704700000000DB
:101A9000B0010010FEE77047F001002021490868FE
:101AA000C2430A600A680242FAD170471E490A68B6
:101AB000002AFCD1CA610860C8690028FCD0002057
:101AC000C86148687047194801686FF00202114008
:101AD00041F40071016003211548816041F2300139
:101AE00041610121C160502141610121C1604FF478
:101AF000CA6141610121C160016070470D480268FF
:101B00000A6082684A60C2688A60406B20F0784050
:101B100040F08050C8607047704701461022064868
:101B200000F024B8101004400010044000000460CD
:101B3000004104404C130050180000217047000081
:101B400009480168426803689942FAD1100C40EADA
:101B50000140704710B5044A136850681468A342E6
:101B60001946F9D110BD00000820094062B38B0767
:101B700008D0521E11F8013B00F8013B00F0248010
:101B80008B07F6D1830740F0208000BF103A07D3BF
:101B900030B4B1E83810103AA0E83810F9D230BCAF
:101BA000530724BFB1E80810A0E8081044BF51F85B
:101BB000043B40F8043BD20724BF31F8022B20F845
:101BC000022B44BF0B7803707047083A07D3B1E883
:101BD0000810083A40F8043B40F804CBF7D253070A
:101BE000E4E70000DFF800F0F5C00110DFF800F0D6
:101BF00049BA011020B1082324220021FEF706BDB6
:101C0000704780B50120009009234FF40072002135
:101C1000DFF8F00600F009FE01BD80B500230122C7
:101C20003421DFF8E00600F013FE00B10120C0B25D
:101C300002BDDFF8D40680687047DFF8CC16401884
:101C400090F8ED0070470022022904D1012806D146
:101C500040F2EE2203E0012808BF4FF47A721046EA
:101C60007047DFF8A406D0F8DC007047DFF898066C
:101C700090F8E61021B1D0F80C01010018BF004720
:101C800070472DE9F041DFF8808608F1E1058AB060
:101C9000A879002861D10120A871DFF87066DFF80B
:101CA0007076307B68717068C8F80C0101A8FFF786
:101CB000A1FF00200690ADF81400079001AB0022B0
:101CC0000FF2DD4108F10C00FEF7C0FC01AB002271
:101CD0000FF2895108F13000FEF7B8FC01AB002289
:101CE0000FF2C14108F15400FEF7B0FCB1680120C9
:101CF0008847DFF8200600787868C0F38154707B4D
:101D000020B1032C02D10120287003E0032C18BF5E
:101D1000022C16D1022000F09DF8032CDFF8F815F4
:101D20000CBF4FF47A7042F210700968B0FBF1F109
:101D300008F15400FEF76EFC08F15400FEF76EFC4B
:101D400005E0012C03D100F057FAFFF75AFF38687D
:101D500040075CBF002000F07DF80AB0BDE8F081CC
:101D600010B508B1140001D1022010BD8160C2601D
:101D700003610146DFF8900500F084FD002010BDEE
:101D800010B50446FEF732FCDFF87C15621892F8B5
:101D9000E8305B1E82F8E830DBB223B98A680123A1
:101DA000A3409A438A6066E02DE9F0410546FEF7BC
:101DB0001DFC8046DFF85015681890F8ED20521E83
:101DC00080F8ED20D2B2002A3FD10FF28850DFF820
:101DD0004C4500EB85052E786F88300615D52168B7
:101DE000096A384688472168896A384688472168E1
:101DF000096B38468847DFF8281501200860DFF8AE
:101E0000240500688007FAD512E0700606D501EBBC
:101E100087010020D1F80011884709E0216889690D
:101E2000384688472168496B384688470228F9D1E7
:101E300006F03F003F2818BFFFF7B6FF687800F0B4
:101E40003F003F2818BFFFF7AFFF4046BDE8F04115
:101E5000FEF7D0BB10B50446FEF7C8FBDFF8A814A8
:101E60008A680123A3401A438A60611891F8E82028
:101E7000521C81F8E820BDE81040FEF7BBBBF8B566
:101E80000646FEF7B3FB0446DFF87C54701990F861
:101E9000ED104A1C002980F8ED2039D10FF2B44032
:101EA00000EB8607387800F03F003F2818BFFFF7A7
:101EB000E6FF787800F03F003F2818BFFFF7DFFF0C
:101EC0007E883878DFF8547401060ED53968C96900
:101ED000304688473968496A304688473968C96A50
:101EE0003046884700F019F812E0400606D505EBA9
:101EF00086010120D1F80011884709E03968496955
:101F0000304688473968496B304688470128F9D1FF
:101F10002046BDE8F240FEF76DBBDFF80414012057
:101F20000860DFF8000400688007FAD570472DE9E3
:101F3000F04F002483B04FF0000A0128D04618BFAC
:101F4000012664D1DFF8C093D9F8DC0001285DD107
:101F50000220C9F8DC00FFF745FE0090012000F0E8
:101F600056F9060054D1FEF77DFBDFF8C01301904F
:101F70000C60012000F036FA012804D1002000F0A6
:101F80009BF94FF0010ADFF8A813DFF89C030C60FF
:101F900000681120FFF751FE08B14FF00108102032
:101FA000FFF74BFE08B148F002080F20FFF745FE8F
:101FB00008B148F004080B20FFF73FFEDFF85C6330
:101FC00020B13168096B4FF4806088470A20FFF721
:101FD00034FE20B13168096B4FF481608847DFF827
:101FE0004013DFF85073DFF850B30120086048F069
:101FF0002000316889698847DFF8401301200860B4
:1020000099F80800C00707D5012416E0042673E0FC
:102010000120C9F8DC006CE0584600F047FC05469A
:10202000042DF9D0012D04D1326A5268032158469B
:1020300090473868800880003860002000F042FC3B
:10204000B94800683068806B804754B9012D04D1CD
:10205000326A5268012158469047386840F00300C0
:1020600038600120B24908604046316849698847B4
:102070000B20FFF7E2FD20B13168C96A4FF48060A0
:1020800088470A20FFF7D9FD20B13168C96A4FF4AB
:1020900081608847A249012008600020A7490860A4
:1020A0000320C9F8DC003168496B404688470128A5
:1020B000F9D1042000F0ABF89C49012008609A484F
:1020C00000689F4800688006FBD5BAF1000F1CBF6E
:1020D000012000F0F1F800F041FD082000F097F831
:1020E00006460120C9F8DC000198FEF7BFFA00F0AF
:1020F000B9FC0098FFF77AFD3046BDE8FE8F30B599
:10210000002401288BB004D021D303281DD018D37C
:102110001DE001A8FFF76EFD7B4D8A490694ADF8DE
:102120001440079401AB012205F17800FEF78EFA06
:1021300000940023844A2C2105F19C00FEF782FACA
:1021400005E000F027FD044601E000F0C9FD20464F
:102150000BB030BD00F053B938B5FEF747FA05466D
:10216000694890F8E000012410B1FFF756FD0446DD
:102170002846FEF73FFA204632BD38B5FEF736FA5C
:10218000614D044695F8E00020B100F07FF9002091
:1021900085F8E0002046BDE83240FEF72BBA00008B
:1021A0007047000010B582B0042000F01BF902282F
:1021B00018BF032807D100F01FF8FFF722FDBDE884
:1021C00016400220DCE56148534900684E4CC0F3DC
:1021D000815003280CBF4FF47A7041F288300968AF
:1021E000B0FBF1F104F15400FEF714FA04F15400CD
:1021F000BDE81640FEF712BA032000901C234FF0F2
:10220000405200213F4800F010BB0020704770B5DD
:1022100004463D4E304600F02BFB002598B9304671
:1022200000F02CFB0646B068204207D03269F36804
:102230000021204698470546012D05D0304600F084
:102240001FFB0600EFD1284670BD414901280CBF95
:1022500040F2FF70002008600020704770B5FEF764
:10226000C5F9294E294D044696F8E00028B100F042
:102270000DF968B1002086F8E0000220AD68A8479B
:1022800006461020FFF7C3FF8EB10320A8470EE0DB
:10229000214909683220B0FBF1F101B9012106F1B1
:1022A0003000FEF7B7F906F13000FEF7B7F9204627
:1022B000BDE87040FEF79EB938B501281ED100F088
:1022C00091F801281CD000F0D7F80F4C12490120DA
:1022D00084F8E00032200968B0FBF1F505B901256A
:1022E00004F13000FFF7A1FA294604F13000FEF7AF
:1022F00091F904F13000FEF791F901E000F0E8F8FF
:10230000002032BD00A00C40D0090020006D00006C
:10231000B03F0050FB1C002050000000B80100102E
:1023200028200860282008402C2009400C40094043
:10233000000222432422084000400340800104435D
:10234000141009401D2E0000ED2B0000B43F00507A
:10235000000004608F3F00008F3F01008F3F0200AC
:102360008F3F0300903F00018F3F0101903F00022B
:10237000903F00038F3F01048F3F00058F12080438
:102380008F3F00048F3F0006513F00007F3F010058
:102390003F3F04003F3F02003F3F01007F3F0200FC
:1023A00070B50446E00782B00D46624E05D5A8B26E
:1023B00000900023012200F011F8A00705D5A8B273
:1023C00000900123022200F009F8600705D5ADB2A4
:1023D000009502230C2200F001F873BD0021304665
:1023E00000F023BA0146042907BF1D234FF0C04265
:1023F0001C234FF080524F48342100F029BA38B5E1
:102400000546FFF79DFB4C4CA168401A4FF47A71CA
:10241000484305EB104500F0D7FD2169401A48BF3D
:10242000404240F6B9318D4207D2062805DAA0684D
:10243000E168814201D322685AB940494A68D2070B
:102440004FF4FA6017D4086800F0FF007D2148437C
:1024500008E0081A3A494843000C00EB900090420B
:1024600038BF1046C82801D2C82032BDB0F57A6FF7
:1024700088BF4FF47A6032BD80B501210320FFF799
:102480008FFFFFF75DFB2C49886001BD80B50120FF
:10249000FFF7A8FF012819D0002301223421254885
:1024A00000F0D6F998B100F026F8FFF749FB224971
:1024B0008B680A68C860A2EB9202C01A204B58438E
:1024C000000C0860904238BF10460860012002BD31
:1024D00010B500210320FFF763FF0120FFF782FF03
:1024E00008B100F008F8144CFFF72AFB606000F018
:1024F0006BFD206110BD1348006800F079BD10B578
:1025000011490A6811490968140424161B38444308
:10251000E41004EB2244120600FB00F31216090635
:102520005A435843091604EBA222484302EBA04049
:1025300010BD000000A00C40D81C0020AC3F005093
:1025400040420F008000001090130050A410005073
:10255000002200F069BD000010B54048046814F185
:10256000010F08BF002400F0E1FD3D490020086094
:1025700001203C4908603C49086000F0A7FF3B4847
:10258000006820B13A480068204600F01CF839493C
:10259000394A00200860394801686FF31B41114334
:1025A000016037480168C1F30131012906D1016892
:1025B000344A114041F40032026001603248006840
:1025C0000028FBD110BD70B50546304801210160DF
:1025D0002F4909680029FBD02E4C2F4AC0212160C9
:1025E00053682E499B075DBF13681B0C43F0F00333
:1025F00072230B70002101639668304600F0A0FD45
:102600003146284600F0CFFD2548816D89B240F261
:102610000F22914213D201680068C1F30361C0F335
:10262000034001B1491E072805D006280EBF072028
:10263000801C00F00F0041EA00101A490870304673
:1026400000F020FE18490968C96802208847402028
:10265000206001201549086070BD00001C13005067
:10266000840460425C600C400822044380012843DB
:10267000000120438C21084000003901482003401C
:1026800004000940FFFFFCFC0C00684210100940E8
:102690009402224300600C40AC3F00505662084058
:1026A000BC12005002600840A00100109404604277
:1026B0001B4213D1094236D12AB18446B0FBF2F055
:1026C00002FB10C2704700F071BFFCD30022002350
:1026D00070470B000200002100207047904271EB10
:1026E000030CF6D370B5B1FA81F4B3FA83F52C1B61
:1026F000A340C4F1200532FA05F63343A2405FF04F
:102700000046E64002E05B085FEA3202841A71EBA1
:10271000030524BF204629467641F4D302000B006E
:102720003000002170BD012ACFD970B5140C20D023
:10273000B1FA81F4B2FA82F5C4F120046419B4F15B
:102740002006D6D3B2405FF00044F440002502E0FA
:1027500052085FEA3303C61A71EB020E24BF3046FB
:10276000714664416D41F3D302000B002000290043
:1027700070BD0C46B1FBF2F102FB11452D0445EA98
:102780001045B5FBF2F402FB145580B240EA054552
:10279000B5FBF2F002FB105240EA044070BD0000AD
:1027A00070B504460D46164600F0D4F9401E80412F
:1027B000C00F1A490A68002AFCD0012E02D0022E4E
:1027C00002D003E0257002E0258000E025600122B0
:1027D0000A6000281CBFBDE8704000F0BFB970BDA2
:1027E00038B504460D4600F0B5F9401E8041C00FD3
:1027F0000A490A68002AFCD0012D02D0022D02D01D
:1028000003E0247802E0248800E0246801220A60C2
:1028100008B100F0A3F9204632BD000000800C4052
:102820000B46114604221818BAE710B500EB410018
:10283000102B144600F5007002D3103B001D240C31
:102840000299994041EA0441BDE810400422A7E7FB
:1028500038B51D460818102D144602D3103D801CB3
:10286000240C0221FFF7BCFF204080B2E84032BDBB
:10287000006800280CBF01200020704700687047E6
:102880000068704738B504460D4600F090FE002100
:102890002960616869606168002914BF0D60256066
:1028A0006560FFE7BDE8324000F083BE00680107C5
:1028B0004CBF042000F00300704700001628A8BF9A
:1028C000203870472DE9F84F06469348934C00682E
:1028D000934D800704D50820A87192482060BFE07E
:1028E00000F072FB804690480068009000270017B7
:1028F00000F101090098800208D4C8F13E00C01020
:102900000928A8BF08208145B8BF814687480068CC
:10291000C0F30460FFF7D2FF824685480068C0F329
:102920000440FFF7CBFF09EB0A011629A8BF1521C8
:1029300004DA6FF009029142B8BF114601F01F029C
:102940007C4B42F4F8521A807B4A126812F0030F53
:1029500018BF0127520748BF47F002070EB147F0E2
:10296000040795F90720A8EB0202052A02DAAA79E2
:1029700097425DD0A8F10F0C0026BCF1000FB646BF
:1029800007F0010207F00403DFF8B09123D40CEB49
:102990000C1C4FEA2C2EBEF1080F28BF4FF0070E7B
:1029A0007646072E28BF062609EB860A59F82660C8
:1029B000DAF804A0AAEB060A0AF0FF0613B1CAF37C
:1029C000072B5E445FEA877B44BFCAF3074B5E4434
:1029D0000AB106EB1A6659F82E9009F0FF0A13B1F6
:1029E000C9F307239A44BB0744BFC9F307439A447A
:1029F0000AB10AEB196A401AACEB0E220099AF71CA
:102A0000724380320128B8BF0120342301F0FF0156
:102A100058430AEB12224843B0FBF2F0B0F5803F76
:102A200028BF4FF6FF7008F30708A88085F80780D5
:102A300043480068A988286000201F2904D21F216C
:102A4000A98004E04908401CB1F5007FFAD20F3993
:102A5000090940EAC1003B4908432060002060604A
:102A6000BDE8F18F10B53848006884B21CB300F09F
:102A7000ABFA2B4991F90720904205DA6FF07F02FB
:102A80009042B8BF1046C8718888844201D28C80B9
:102A900010BD2B4A12680B68D21A921C202A28BF3C
:102AA0001F22231A5208D3401818B0F5803F28BFC0
:102AB0004FF6FF70888010BD2448026802B9704745
:102AC00010B5234B996801F04060B0F1406F21D000
:102AD00011480468A4071DD45C68A4071AD40468CC
:102AE0001B68C3F303531C331B0114F0050F06D0FE
:102AF0009A420FD26FF005012140016010BD934250
:102B000008D20A0158BF44F00104490158BF44F0FB
:102B10000404046010BD00000000094030100940AA
:102B2000EC1C0020FDFDA400B43F0050B812005082
:102B30003C1100506E620840242208409C13005053
:102B40000820094000E7A4803410094028500940BB
:102B5000AC3F0050EFF3108072B67047EFF3108077
:102B600062B67047DFF800F099C8011010B50C1874
:102B7000FFF7F0FF401E8041C00FDFF8F0130A6836
:102B8000002AFCD0246801220A6008B1FFF7E6FFA2
:102B9000204610BD38B5DFF8D843DFF8D8132078C9
:102BA000897B002508430AD0FDF720FDA178002984
:102BB00006BF0121A1700125FDF71CFD0DB100200C
:102BC00032BD0220FFF746F90E20FFF758F9DFF873
:102BD000A803016809B1012032BDDFF8A02340211C
:102BE00011600121C1610020607032BD70B5DFF855
:102BF0008C0382B0002101604821C160DFF88003AE
:102C000000F1D804A17A002968D00129DFF87423E3
:102C100029D110684BF2F5214843050ADFF8680313
:102C20000068C0F38140012806D100F0CDF9FFF71C
:102C300066FC684305EB9055607B10B10020607323
:102C400005E0D2480068000215EB10204508D04886
:102C50000560290C416001218160C648807B002805
:102C60003AD0052039E0022909D11568284600F03C
:102C7000FDF8A5F2FF5003282ED308202DE00329EC
:102C80002CD1116800F1B805A1F5C0612868E9618F
:102C9000002848BF4042002948BF49428842A8BF97
:102CA000002018DA6868BB4E80B2009008234FF409
:102CB0007F4230213046FFF7B8FDA86800F072F976
:102CC00004213046FFF7B1FDA86900F071F93046E4
:102CD000FFF7ABFD012020700B202073BDE873408F
:102CE0002DE9F041A64CDFF8AC82AB4FAB4EA348C8
:102CF00004F1E10582B0E9784A1E0B2A00F28080D7
:102D0000DFE802F0062233465B33465B3346636EF0
:102D1000A34909680968202088470F20F860072325
:102D200041F61D5038614FF4C0720220009000F04F
:102D300070F807234FF4C07200214046FFF788FD6A
:102D400001203060022044E00120F861287800284A
:102D50001DBF0020306103200620E870032038608A
:102D6000002070607068800734D4E878032804D1AC
:102D7000022000F04BF8042007E0002000F046F8A5
:102D8000E87806280CBF07200A20E87001201AE026
:102D9000042903D12021B961012105E00122BA6192
:102DA0000A290CBF03210221697000213960082122
:102DB000C16001600120386026E005290CBF0620B3
:102DC0000920E8700020706004E00020306070602E
:102DD0000C20E87004F17800BDE8F641FDF71EBC58
:102DE000002101600120644908600E20FEF7DCFF2D
:102DF0000220FEF7C5FF0120E8700020A87003E064
:102E0000BDE8F341FFF7AEBEBDE8F38100900523B6
:102E1000602200214046FFF708BD000080B55849F8
:102E20005E4891F8E410891E0A291AD8DFE801F0FB
:102E3000060A0E190A0E190A0E19120001688907EE
:102E4000FCD510E041688907FCD40CE04168890793
:102E5000FCD508E001688907FCD441688907FCD4E7
:102E600001E0FFF77FFEBDE8014039E7F8B507460E
:102E7000484C30212046FFF779FE414E06F1B80557
:102E8000C0F30720686004212046FFF76FFEC0F3FF
:102E90008440A86020212046FFF768FEC0F381200F
:102EA000A861B7F5C060286002D186F8D800F1BDEE
:102EB000296996F8D8202AB96A68A968EA60E861A1
:102EC000AA696A61E86900284CBF6FF0010202221A
:102ED00000EB40001018421000EB927001EBA000D4
:102EE0006968E960012810DA6A69032A04D115309B
:102EF00001281DDA01201BE00B300128B8BF01209A
:102F0000491E48BF0021E96007E01F2812DB6A69FB
:102F10002AB915381F28A8BF1E20032109E00B3845
:102F20001F28A8BF1E20491C4029A8BF3F21E960D7
:102F30000021696128610823E86880B200904FF49D
:102F40007F42302100F03CF80120009011234FF423
:102F5000003200F034F8286900F024F800F02FF86F
:102F6000686900F025F800F02BF8F1BD00800C40F6
:102F7000B10A0020006D000004800C402C500C4071
:102F8000D009002008400C40B43F005010200940F8
:102F90003C600C4000A00C4000400C4034600C40F1
:102FA000A001001080B2009012234FF4F802704785
:102FB00080B200900A234FF4406220217047042120
:102FC0002046FFF732BC00000748084A81681278A3
:102FD000006852B2A0F54070C9035043C913A1EB79
:102FE0002010803000127047285009400C13005008
:102FF00070B50446FFF7AEFD451EAD41ED0F074E1F
:1030000030680028FCD0A04701203060002D1CBF94
:10301000BDE87040FFF7A2BD70BD000000800C400D
:1030200062F30F2262F31F4200B500BF1300964601
:103030009446103928BFA0E80C50FAD85FEA417CCA
:1030400028BF0CC048BF40F8042BC90728BF20F890
:10305000022B48BF00F8012B00BD0000304800687B
:10306000000C00F00700052828BF4FF0FF30704724
:103070002C490A68C2F30F324BF69A139A424FF06A
:10308000FF3006D10868000F0B280CBF0420002079
:1030900070474BF6BE118A4201D1012070474BF6B2
:1030A00041318A4201D1032070474BF620318A42D8
:1030B00008BF0220704700001A48F8B50068050FE5
:1030C0001948006800F0FF06802E28BF0026FFF791
:1030D000CFFF04284FF0FF3406F10A071DD8DFE8C0
:1030E00000F003121A1A1B00012D12D0032D06D076
:1030F000072D06D0082D08BF06F116040DE0142494
:103100000BE0152409E025B1022D08BF06F11404D7
:1031100003E00A2401E005B93C4660B2F2BD0000BC
:103120009412005018130050A010005080B5FFF703
:103130009FFF20B9FFF7C0FF162800DB01BDFEE7A7
:10314000DFF8E8130968C1F304611629A8BF203924
:1031500001EB2071491C1629A8BF152104DA6FF074
:1031600009029142B8BF114601F01F01DFF8C023E8
:1031700041F4F8511180DFF8BC13096889074FBF8B
:1031800040F040600021DFF8B0231160DFF8AC139D
:10319000C0F3C06282F00102C0F380600A6080F078
:1031A00001008860704770B5054682B0084600F09F
:1031B000EEF80246DFF88843182100F060F800F0CE
:1031C00012F980B20090002340F2FF322C212046F9
:1031D000FFF72BFBDFF86C63F068C0F30D021C21D6
:1031E00000F04DF8706800F0FC32142100F047F850
:1031F0003068DFF85413DFF8546301EA000210214D
:1032000000F03DF8284600F0F8F802460C2100F0E6
:1032100036F8284600F01CF9400040F020003072DB
:10322000284600F01EF940F010003072284600F0E9
:1032300021F90246282100F022F8284600F0FFF884
:10324000400040F06000F072284600F02DF9C00008
:1032500040F080003070284600F02FF98000BC4913
:1032600040F47C400880284600F011F9024608210D
:1032700000F005F8B7494FF48000086073BD2046A0
:10328000FFF7CEBAF8B5810C01F003010129B24C69
:10329000B04D02D002292AD026E0216A8A0323D425
:1032A0004FF480422A606FF08F06AC4AD2F80230A9
:1032B00033404E0A06F080063343C1F303363343EE
:1032C000C2F80230C1F30326D2F801301B0946EAE6
:1032D0000313C2F801306FF0E7061368334001F0C2
:1032E000E7011943116002E04FF0004129609C4E54
:1032F0009C4AB16809075CBF4021A9624FF4007184
:103300002964800D216AC90C01F0030141F03001EC
:1033100010F00300117003D0022826D008D326E055
:1033200001210420FFF73CF88F4800F0F0F822E07C
:103330000120FFF757F8074639460420FFF730F819
:103340000420FFF74FF8B842FAD1366826F07F40E4
:1033500000F0DDF8854B1B681B684FF060220721E9
:10336000300E98474FF480602860032100E002216E
:103370000420FFF715F820687D4900F03F00087031
:1033800047F618007B4908807B480068F1BD7B49FF
:103390000968C1F383628303C1F38F2120D4000441
:1033A00000164FF6FF7307E0490804D1194652088A
:1033B00004BF01220121401C0028F5D401280FDBA5
:1033C000490041F00101B1F5803F21BF01215200C8
:1033D00042F00102102A24BF0F221946401EEDE7D9
:1033E00041EA024070476548016800680002C1F385
:1033F000870100F440700843704730B5604C614964
:103400000A686568ED07C2F30351C2F303430AD4A7
:103410002468250501EB2571240481F3040103EBE5
:10342000247383F304031B0443EA015193B2194349
:10343000222824BF02F080400143084630BD00210D
:10344000202803D350480068C0F301510846704754
:103450000121222803D34D480068C0F300710846BB
:1034600070470121222803D348480068C0F3407107
:10347000084670470021202807D343480068C10C44
:1034800001F44071C0F3845001430846704720287E
:103490003F4907D33C483F4A0068810A02EA0030AE
:1034A00040EA8151084670470021222803D337485B
:1034B0000068C0F3C061084670470021222803D38A
:1034C00032480068C0F345510846704732480068EA
:1034D0000028FBD13148324A4168126889088900C6
:1034E00041F0005141F00401520748BF41F0010191
:1034F0000BD4026812F0030F07D041F003024260C0
:10350000026802F00302032AFAD14160704725499C
:1035100082B20A60C0F307404860012088602248F8
:1035200000680028FBD0002088607047B812005067
:103530006E6208400000094094042A4300002043C2
:1035400000A00C4070130050FFFFFC0041A10C4094
:10355000DCA10C4040A00C406C1300500A600840F5
:10356000A83F005008A10C40BD378600B4010010F0
:103570000BB00C4070B00C402C2009405013005090
:10358000AC3F005078130050981300508C1300503B
:1035900000803F4000F03F000C00684200400340C4
:1035A000B03F00503C600C4084088C437047FDF7EE
:1035B0001DB8FDF71FB80000DFF800F0D9C10110F9
:1035C000DFF800F0ADB50110DFF800F019AE011022
:1035D000DFF800F0E5C10110DFF800F085C201104E
:1035E000DFF800F081C20110DFF800F055C10110D2
:1035F000DFF800F043C20110DFF800F079AB0110F2
:10360000DFF800F0D9B60110DFF800F0EDB30110DB
:1036100020B108232C22002100F012BD704720B1F8
:1036200008233C220021FFF7C7BF704780B5FEF793
:10363000D9FAADF80000FCF7D9FFADF80200009808
:1036400002BD01B5BDF80200FCF7D4FFBDF80000D3
:10365000BDE80240FEF7CABA38B5DFF8A008DFF8C7
:10366000A018DFF8A04880088000091A2161E060F6
:10367000034602E0002523F8025B0D18AB42F9D3A4
:103680008B0800EB8303002223F8042CE82202803D
:103690004FF6FC721140EC39A0F8E810E830606099
:1036A000002000F004F8A060E068606031BDF8B56B
:1036B00000240025061D16F003001CBF311D0E1A44
:1036C000FFF7B4FFDFF83C28B6B21060112EB4BF8C
:1036D000576897683A88130403D582F4004200259E
:1036E0001AE02B0014D0238839880B4423809BB226
:1036F000B34211D327461A46B7B1921B92B2042A9D
:10370000A7BFBA5346F40041398841F4004109E0AB
:10371000B242F1DA01253C4617443A88002ADAD150
:10372000002701E027F8041BFFF78BFF3846F2BDA6
:1037300010B50446FFF77AFFDFF8C817086034F8C1
:10374000042CC2F30E0224F8042C221F4B689A4268
:1037500038BF4A60BDE8104073E738B50446FFF74C
:1037600065FF00210C23DFF8A0274B43D518AA6C76
:103770004AB1944204D1FFF764FF05F1480032BD1D
:10378000491C0329EED3FFF75CFF002032BD70B562
:103790000546FFF74BFF044600200C22DFF86817B0
:1037A00042438E18B16C49B900203065B5640022DF
:1037B000FFF706FFF06418B900F04CFC8D4205D10C
:1037C0002046FFF73EFF06F1480070BD401C03286D
:1037D000E3D32046FFF735FF002070BD38B504461F
:1037E000FFF724FF0025DFF820170C226A438A5ACE
:1037F000130008D0944203D1FFF723FFE8B232BD93
:103800006D1C062DF1D3FFF71CFFFF2032BD10B554
:1038100004462088FFF7E2FFFF2800D16BE10C226D
:10382000DFF8E416504308448168080002D16FF0C5
:10383000010010BD2046BDE81040084702460FF2C7
:103840003870104710B500200C21DFF8BC2600248A
:1038500001FB00F31344401C03289C641C65F7D350
:103860000020002301FB00F4401C13530628F9D369
:10387000082010800FF2E9609060BDE81040EBE690
:1038800070B590B0FEF7AEF904466846FFF7C7FE84
:1038900005200690002240F2B630089069464FF6A7
:1038A000C1500490DFF864060590DFF86406FFF766
:1038B0008BFE050006D0FFF7B9FE06462846FFF747
:1038C00066FF08B900F0C6FB3046FFF7BAFE204697
:1038D000FEF78CF910B070BDF8B500F0E6F8FFF710
:1038E00056FF05006FF0020616D0FFF79FFEA28874
:1038F00000210C27DFF810364F433B441F883FB9A7
:103900001A805D60A2689A60217369682161C4E2CF
:10391000BA4203D1FFF795FE3046F2BD491C062995
:10392000E7D300F097FB00BF38B500F0BEF8FFF713
:103930002EFF050016D0FFF779FE00210C23DFF8DB
:10394000C8254B431A4413884BB94FF6F8731380BC
:1039500055600023936021716968A16013E7491CD9
:103960000629EBD300F076FB00BF10B50446606873
:103970000C3080B2FFF79BFE00B91AE0616801814C
:1039800000210160FF2181720C30A060002010BD79
:1039900080B540680C3811E080B288E610B5044666
:1039A000606880B2FFF783FEA06000B901E00020EC
:1039B00010BD6FF0030010BD80B54068FFF7B8FE82
:1039C000002002BD38B504460D46FFF72FFE00214A
:1039D00045F80C1C216811B9256006E0114651F824
:1039E0000C2C002AFAD141F80C5CBDE8324028E6E4
:1039F0002DE9F04104466FF00206E068A0F10C05E5
:103A0000A0790628BCBF207906280BDAFFF70EFE46
:103A1000A179DFF8F4840C2779434144496819B946
:103A2000FFF70FFE304617E0FFF70BFE20792871F5
:103A3000A0796871207AA871A079E1687843404440
:103A400040680830FFF7BEFFA079784340444068E3
:103A50004068FCF7D3FD0020BDE8F08170B500F0B0
:103A600024F8FFF77AFE060002D16FF0040070BD63
:103A7000FFF7DCFDB168002541B10D46A5F10C0151
:103A80000A68B26000220A60FF228A72FFF7D9FD3D
:103A90002800A56001D1022070BDA5F10C000179BC
:103AA00021714079A071002070BD0446FFF790BDE0
:103AB00006280ADA0C23DFF850245843105A020073
:103AC0001CBF4FF6F872904202D14FF0FF307047A2
:103AD000088000207047811D0079E9E710B5044691
:103AE000E088FFF77BFEFF2800D104E0A0712046AC
:103AF000BDE810407CE74FF0FF3010BD3EB50446F6
:103B0000FFF7ACFF050017D120796946FFF7D0FF1A
:103B100078B10820ADF804000320ADF80600DFF806
:103B2000F413A0688968029001A888476FF0050027
:103B30003EBDBDF80000A08028463EBD10B5DFF8B0
:103B4000D82312680C464FF47A71A1FB00010023C0
:103B5000FEF7AEFD002399424FF0004201D890429B
:103B600002D36FF0020010BD2060002010BD38B5F8
:103B7000FFF79BFFFFF7F1FD0546FDF7F4FD002879
:103B800018BF012800D015B96FF0040032BD60687D
:103B900040B9009000996868FCF734FD401E8041F0
:103BA000C00F32BD10F1010F08BF4FF0FF30F0D051
:103BB0006946FFF7C3FF0028ECD032BD80B54068EE
:103BC000FCF71CFD002002BD00F044FA00BF80B5E8
:103BD0004068FFF701FD002002BD80B54068FFF797
:103BE000FFFC002002BD80B5FFF7FEFCFFF700FDE3
:103BF000002002BD80B5FDF7F5FFFCF7F7FC0020C3
:103C000002BD10B58CB004466846FFF701FDE02008
:103C100000F013F808B900F01DFA0BE010B58CB0F5
:103C200004466846FFF7F4FCE06800F006F808B9BF
:103C300000F010FA00200CB010BD08900023A1681D
:103C400060686A46FFF7D8BC10B50446FFF7D8FC99
:103C50006060002010BD0146886849680847F0B5DB
:103C600007468BB0BC68AB4D6CBB0C20FFF71FFD4B
:103C700004006FF003061ED008232422002101A8AF
:103C8000FCF7C4FC0020ADF8140006900794002354
:103C90007968A24801AAFFF7B7FC206068B908203C
:103CA000ADF800000C20ADF802006846A96888470E
:103CB0002046FFF73DFD304618E0F868606038693F
:103CC000A060BC600AE02868804706462068FDF7CF
:103CD000ACFD3869A060304669688847796820681B
:103CE000FCF798FC2068FCF799FC00200BB0F0BDB5
:103CF00010B5044682B060686946FFF71FFF20B91F
:103D0000009860602046FFF7AAFF16BD80B54068A6
:103D100010B96FF0020002BD0068FDF786FD0020BB
:103D200002BD7D49096841600020704750B50446D6
:103D3000794802686FF00046A6FB020100234FF4A9
:103D40007A72FEF7B5FC002399424FF0004201D889
:103D5000904200D330466060002050BD2DE9F04114
:103D600086B00646FFF734FCFFF7F7FC0446002058
:103D700002900025FDF7F7FC002818BF012800D0AD
:103D800014B96FF0040063E0706820B110F1010F06
:103D900003D14FF0FF30009004E06946FFF7CEFEFC
:103DA000070054D1FFF72CFC0099012701EB000814
:103DB00000E0009000996068FCF724FC78B303A849
:103DC000FFF74CFE07001AD19DF8100001A9FFF77C
:103DD0006FFE80B9059A9DF81210BDF80400B36813
:103DE000984740B1BDF80400B0819DF81200B0734F
:103DF0000598306113E0059902A8FFF7E3FD0098EC
:103E000001276D1C10F1010F18BF0028D2D0FFF759
:103E1000F7FBB8EB000002D000998142C9D2029EA4
:103E2000FFF704FC56B1314600E0114651F80C2C66
:103E3000002AFAD1A26841F80C2CA660FFF701FC19
:103E4000002D03E06068FCF7D9FB6D1EFAD13846FF
:103E500006B0BDE8F081F8B5FFF727FE0546FDF78F
:103E600082FC002818BF01286FF0040613D0FFF76A
:103E7000DDFB0021244A0C234B43D75A4FB1134496
:103E80005B681B68AB4201D1217106E0491C062921
:103E9000F1D3FFF7D6FB3046F2BDFFF7D2FB00208F
:103EA000F2BDF8B50446FDF75EFC002818BF0128F6
:103EB00002D16FF00400F2BDFFF78AFB0546FFF761
:103EC000B5FB0021104A0C234B43D65A37000ED0C5
:103ED000A788BE4208D1D11849680968A9420CBF19
:103EE00001210021A160D8E7491C0629EBD3FFF787
:103EF000A8FB4FF0FF30F2BD00000000001D0020C5
:103F0000283F0020DC14002070140020A8040020AA
:103F10003D3800009404002050000000573C000091
:103F200070B504463C20FFF7C2FB05006FF00306A6
:103F300011D0FFF774FB207AA86100226089286203
:103F40002946E06828616068FFF73EFB0446284682
:103F5000FFF7EEFB0CB9304670BD002070BD0000CD
:103F600041882D2902D36FF0010070470FF214022F
:103F700052F82110084700000F3800002D360000CD
:103F800043360000D9380000293900006B390000A1
:103F9000913900009D390000B9390000F139000065
:103FA0005D3A0000DD3A0000FD3A00006F3B000082
:103FB000BD3B0000C93B0000CF3B0000DB3B0000E5
:103FC000E73B0000F53B0000033C0000493C0000DB
:103FD000F13C0000233D00002D3D0000D73A0000D9
:103FE0002B670000FF6700005D3D0000573E0000AA
:103FF0005F3C00000D3D000099670000D1670000A4
:10400000E5670000A33E0000316800004968000039
:10401000213F000000000000000000003F68000099
:10402000576800001D3C0000000000000000000078
:104030000000000000000000DFF800F0F1C50110F2
:1040400001B90149FFF7F8BFA0010000DFF800F057
:10405000ED8C01100120FFF7F9BF0000DFF800F040
:1040600025B101102DE9F04EDFF8BC79924600260B
:1040700040F2013B0C46BA787B7997F804C097F878
:104080000190B0EB0B0540F67B4132D06D1E38D06D
:104090006D1E3DD0AD1E41D06D1E00F07A806D1EAC
:1040A00000F07D806D1E00F087806D1E00F0948012
:1040B0006D1E00F099806D1E00F09E806D1E00F058
:1040C000A5806D1E00F0AA80ED1E00F0AF806D1E71
:1040D00000F0B4806D1E00F0B9806D1E00F0BE804F
:1040E0006D1E00F0C3806D1F00F0CB80AD1E2DD083
:1040F000E1E0102C40F0DD801022514607F1A400D1
:1041000081E0102C69D11022514607F1B4007AE009
:10411000042C62D1DAF80000F862D7E0012C5CD1FF
:10412000012B34D09AF800003871BCF1000F06D092
:104130000028F2D1022A19D0052AEED116E0002873
:10414000EBD0012A1FD0042A1BD11CE0012C44D142
:10415000BCF1010F1BD09AF80000787153B1002810
:1041600007D1032A1CBF072A052A02D1484600F0BE
:10417000D8FEABE00028FCD0012A1CBF042A062A86
:1041800001D0052A02D1012000F047FC9EE0122652
:104190009CE0022C21D1BAF80000F88396E0202C94
:1041A0000BDA07F1CC0600F094F800F09AF8BC7135
:1041B0003346224601210BE0202C7ADA07F1EC0687
:1041C00000F087F800F08DF8FC713346224600219C
:1041D000484600F088FE76E0012C6AD19AF800008B
:1041E000052866DA387271E0012C62D19AF8000075
:1041F00004285EDA787269E0062C5AD14FF4867092
:10420000062251463844FDF7B1FC5FE0012C50D145
:104210009AF8000008284CDAB87257E0012C48D10F
:104220009AF80000042844DAF8724FE0012C40D1DB
:104230009AF8000006283CDA387447E000F04DF8A0
:1042400037D1821F8A4234D278823FE000F045F8AD
:104250002FD1821F8A422CD2B88237E000F03DF87D
:1042600027D1B0F5FA7F24DAF8822FE000F035F894
:104270001FD1A0F10A0140F67742914219D238834A
:1042800024E0012C04BF9AF80000012811D107F1A5
:10429000800001F004F950B907F1100100F070FB43
:1042A000060013D107F15C0001F000F90EE01626BC
:1042B0000CE018260AE0282807DA022C05D1BAF803
:1042C000001000F041FE064600E002263046BDE840
:1042D000F08E1F21304601F02FB9BAF80000022CF1
:1042E0007047224651463046FDF740BC38B50024A1
:1042F0004FF440730D46C21ADFF82C1736D0521E09
:1043000036D0521E37D0521E38D0521E39D0521ECF
:104310003AD0521E3CD0521E3CD0521E3DD0521EAE
:104320003ED0521E3ED0521E3ED0521E40D0521E93
:1043300040D0521E40D0921E40D0521E40D0521E3D
:1043400040D0521E40D0521E40D0521E40D0521E6D
:1043500046D0521E46D0521E46D0921E48D0521E03
:1043600014D0521E42D0521E44D046E0C87842E0DB
:104370001022A43130E01022B4312DE0C86A286048
:1043800042E00622C43127E0087934E0487932E07F
:10439000C88B36E08A79CC311EE0CA79EC311BE05B
:1043A000087A28E0487A26E006224FF4867012E068
:1043B000887A20E0C87A1EE0088C22E0087C20E0A1
:1043C000488A1EE0888A1CE0C88A1AE0088B18E038
:1043D00006224FF48A7001442846FDF7C7FB13E01C
:1043E000488C0EE0888C0CE0C88C0AE0087B02E068
:1043F000887800E0487B287006E0282803DA00F07F
:10440000BAFD288000E00224204632BD1CB5DFF84A
:104410001846A17881B900B1206304F12C00019005
:1044200004F1B400009004F1A403E1786078002264
:1044300000F010FD002016BD112016BDDFF8E805C4
:104440008178062918BF072904D1018C40781322EE
:1044500000F02ABD1220704700B58FB008233C221F
:1044600000216846FFF7A8F8DFF8C00500F1500109
:10447000079100234FF4DC7108916A4603210691ED
:104480000FF2D101FFF7EAFD0FB000BD70B584B0A7
:1044900000F019F90120DFF89815DFF88C4509685C
:1044A0000FF29155ADF802000026684688479DF846
:1044B000040060700298A0620020A0704FF6FF70A8
:1044C000208400F076FD207000230120019000225E
:1044D00000200090294604F1380000F0A5FF0220DA
:1044E00000F02FF804F15C0000F09EFF042000F0C3
:1044F00028F804F1800000F097FF0420E07004F138
:10450000A40200200021002300252BC204F1B405E1
:10451000103A4BC5E06220726072E1720720A0720F
:104520001021022000F016FF103D2A461021032022
:1045300000F010FF04F12C020421042000F00AFF17
:104540007FBD019000230020009000222946704783
:1045500000000000FEB5FFF799FFDFF8CC54DFF84C
:10456000D04405F1800700F0AEF80A20ADF8020053
:104570004FF0FF30019068462168884700284BD1F2
:1045800000F0A1F80920ADF80200684621688847CC
:104590009DF80610029E00283ED1BDF804001028A8
:1045A00004BF687881422DD130884FF6FF71884270
:1045B00009D17088400425D505F12C02042104207E
:1045C00000F0DDFE1EE03078A22805D0D02804BF20
:1045D000304600F07CF815E07079132812D130894C
:1045E000012804BFA87B022805D1384600F05EFFF1
:1045F000FFF724FF06E0052000F0BDFC0146384629
:1046000000F038FF46B100F05EF80320ADF802007C
:104610000196684621688847A88BC10730D54FF6B8
:10462000FE710840A88329796879014328D018B120
:1046300003208DF800000DE0287A8DF80000062296
:10464000687A8DF801004FF4867029180DF1020088
:10465000FDF78CFAA87A8DF808006946E87A8DF89B
:104660000900687800F03BFC00281FBF0820A870F4
:10467000286B002804D0016808001CBF0820884768
:10468000A88B810708D54FF6FD710840A88305F176
:104690001001002000F074F9A88B41070AD54FF6ED
:1046A000FB710840A883A87B012804D0022808BF1A
:1046B000FFF7C4FE57E700902B8BEA8AA98A688A25
:1046C00000F093F94FE70820ADF800007047FEB501
:1046D000D54DA9784FF48A730446EE18A27868790C
:1046E000130005F1800715D0022A3CD0032A18BF19
:1046F000042A5CD0052A00F07F80062A00F0AC80F6
:10470000072A00F0CD800F2A00F0E580112A00F082
:10471000E780F7BD607801001AD105F1A4021021ED
:10472000022000F02CFE05F1B4021021032000F05D
:1047300026FE0622E11C05F1C400FDF717FA012050
:10474000A87005F1CC03AA796878012100F0CBFBB1
:1047500008B10820A870286B20B1016808001CBFB0
:10476000A8788847F7BD6278EAB9E27842B1EA7979
:10477000687805F1EC03002100F0B5FB607012E0F1
:10478000022918BF07290ED0062902D101280AD113
:1047900001E0032907D005F1380000F080FE10B9D0
:1047A000012000F03AF960780028DBD0D1E7637887
:1047B0000BBB2B79032A08D1062908BF0720C9D0D3
:1047C000002B0CBF03200220C4E7E98B0A0006D0AF
:1047D00018430AD005F1380000F04CFE05E0012B2B
:1047E00007BF0020287100206871A878072814BF2F
:1047F00004200620AEE7ACE76078010026D106224F
:10480000211D3046FDF7B2F9608928840620A87082
:10481000E0896884208AA884608AE884E078287324
:10482000287C012818BF022809D11F2000F0A3FB13
:104830004FF47A71414305F15C0000F01BFE628980
:10484000E0780423211D00F00DFA84E73128D2D14D
:104850000020287104207DE7A08800F01AFA0621C4
:10486000FFF738FD00206884A884E884A079687385
:1048700005F15C0000F01AFE384600F017FE4FF616
:10488000FF702884687908B1032063E7A0790828BD
:104890000CBF05200420A870012000F0BEF85AE7E4
:1048A000384600F003FE6078002813D1E088688461
:1048B0002089A8846089E88405F15C0000F0EFFDA0
:1048C000002807D16B6B002B04D0EA8CA98C688C74
:1048D0001B689847F7BDA088052100F027FBF7BDAE
:1048E000A088ADF80000287C052803D100208DF8B1
:1048F0000A0041E001208DF80A0005F15C0000F09B
:10490000D5FD287C012818BF04281AD1688AE188BF
:10491000814228BF0846ADF80200A98A2089884252
:1049200038BF0846ADF80400E98A6089884238BF7C
:104930000846ADF80600298BA08988421AD208469D
:1049400018E0032818BF02280AD1688AADF80200CF
:10495000A88AADF80400E88AADF80600288B09E0C3
:10496000E088ADF802002089ADF804006089ADF858
:104970000600A089ADF80800684600F091FAF7BD7E
:10498000FEB50F46284D7A880446688C904224BFB5
:10499000B988814207D3A88CF988884202BFE88C85
:1049A000398988421ED0052000F0E5FA0646288C99
:1049B000ADF800007888ADF80200B888ADF80400C2
:1049C000F888ADF806003889ADF80800684600F0B0
:1049D00062FA070007D1AC73314605F1800000F0A0
:1049E00049FD00E018273846FEBD3EB50E4CA578BF
:1049F000062D01D014203EBDADF80200ADF8041024
:104A0000ADF80620ADF8083004F15C0000F04EFD72
:104A100006986946FFF7B4FF3EBD03498A8B1043F1
:104A20008883886AFBF7EABDD8040020F8140020C8
:104A30009C040020F1E70000E0B50821ADF800106B
:104A40000190022100F00FF808B100200EBD02987D
:104A50000EBD00B583B00821ADF800100190032110
:104A600000F001F807BDADF802106846DFF87413D6
:104A7000096808471FB5ADF806108DF80400082432
:104A8000DFF860138DF808200393ADF80040ADF80F
:104A9000024068460968884704B010BD30B585B04B
:104AA000144608220291ADF800201922DFF83413D1
:104AB00009680190ADF802201D466846884714B188
:104AC000BDF80C10218015B19DF80E102970089AC0
:104AD0000499116005B030BD00B583B00820ADF871
:104AE00000001A2000F015F810B99DF804000EBD62
:104AF000FF200EBD00B583B0ADF800008DF80610A4
:104B0000002000F006F810B99DF807000EBDFF2048
:104B10000EBDDFF8D0120968ADF8020068460847FC
:104B200050B110F1040F01D10420704710F1030FB0
:104B300001D102207047012070478123037042EAAF
:104B4000C111002341F47C41C370818070478223EE
:104B5000037081800023C370827170473EB50446A4
:104B60000820ADF800000D462020ADF8020010200E
:104B7000DFF870120968ADF804006846884720B96C
:104B8000029810B16FF004003EBD00950023002292
:104B900021464FF0FF30FFF781FF3EBD10B582B0D8
:104BA0001446CA78012A03D18A88DFF844351A806E
:104BB00000F010F858B9009069462046FFF7CEFF84
:104BC00028B900984478FFF744FF204616BDFFF748
:104BD000A7FF16BD0B46022210214BE738B51C4635
:104BE0001546FFF7F7FFC0B9009069462846FFF762
:104BF000B5FF90B900984578280002BF0098C079A9
:104C0000A04205D10098816804982246FCF7AEFFC7
:104C10000098FFF71EFF284632BDFFF781FF32BD27
:104C2000F8B500F084FA00F0C1F907000DD0324663
:104C30002946FFF78CFF00F04EF93872FFF74CFF62
:104C40003B4601B0BDE8F0405FE0F1BD102201211C
:104C5000E6E738B500F00FFA050002D00422012182
:104C60004AE031BD2DE9F04100F064F907000FD0B2
:104C7000142200F019F83C72FD603E8287F8128021
:104C8000FFF72AFF3946BDE8F041DFF8682485E7E1
:104C900025E038B500F02BF8050004D0152200F00F
:104CA00003F82C812BE031BD012150E700220421C3
:104CB00083E02DE9F04100F03DF907000FD002221A
:104CC00000F010F8BC60BD81BE73C7F81080FFF71C
:104CD00003FF3946BDE8F041DFF81C245EE70420FD
:104CE000BDE8F081042132E71022022198E7044652
:104CF0000A20A1E602212AE7FFF729FFAC60FFF7AF
:104D0000EBFE2B4601B0BDE8304002221021B1E697
:104D1000F8B500F0AAF907000AD01522FFF7EAFF5C
:104D200000F045FB3946BDE8F840DFF8D02335E711
:104D30000420F2BD002203213FE000B583B00FF252
:104D40004903019306230093032300F04DF80EBDA1
:104D50001078802802BF508840F27F61884208D1D5
:104D60009088984202BF91790098814201D1012038
:104D700070470020704710B582B00624FFE700940A
:104D8000FFF7E6FF16BD00000323F4E71078802844
:104D900002BF508840F27F6188420CD1908803287E
:104DA00018BF042807D1907901001CBF10281128D2
:104DB00001D10120704700207047F8B500F057FA84
:104DC00007000CD032462946FFF7C1FEBC60FFF752
:104DD00083FE3946BDE8F840DFF82423DEE60420F0
:104DE000F2BD00009C0400202DE9F04100F02BF8FA
:104DF00007000AD0069A4146FFF7A9FE3C817D8153
:104E000000F0D7FA079A00F075BA68E704460D4635
:104E10000C2011E6424603218FE670B582B000F007
:104E200086F9FFF759FE1B210091034632462946B9
:104E3000204600F02AF976BD10B582B01D240094FA
:104E400000F023F916BD04460D461646984610207C
:104E5000FFF7F2BD2DE9F04180460D4616461F468C
:104E60001820FFF7E9FD040014D0002200F069F8D3
:104E700000F068FA20726572A672E76006982061F9
:104E800007986061FFF728FE2146BDE8F0410FF268
:104E9000153283E623E70FF21133112200214AE194
:104EA0000FF209331222F9E7F8B500F0E8F807002D
:104EB0000FD00A2200F045F800F00DF838727D811D
:104EC0003E73FFF709FE3946BDE8F8400FF2E122D4
:104ED00064E60420F2BD21465020FFF70BBE0FF21E
:104EE000D523062238E12DE9F04180460D461646CD
:104EF0001F461020FFF7A0FD040011D0072200F08C
:104F000020F800F01FFA20726572A672E760FFF7C2
:104F1000E3FD2146BDE8F0410FF29D22FFF73EBEC2
:104F2000DDE60FF299230822002115E10FF291230B
:104F30001022EBE004460D46164698461420FFF773
:104F40007BBD0421FFF7F9BD70B5FFF75FFF0600D9
:104F50000BD03022FFF7F5FF00F009F83146BDE82D
:104F600070400FF26122FFF719BE042070BD34813A
:104F70007581FFF7B1BD30B583B004460020ADF8B0
:104F8000040000F013F805000DD03122FFF7D9FF1F
:104F90002C81FFF7A1FD01A9009102230FF2292224
:104FA0002946FFF71BFEBDF804003EBD0A20FFF7AF
:104FB00043BD1CB500F077F904000AD01222FFF7B8
:104FC00073FEFFF789FD00F005F80FF2012200F0F3
:104FD00018F813E001A90091012370471CB500F0F7
:104FE00062F904000AD01822FFF75EFEFFF774FD95
:104FF000FFF7F0FF0FF2E51200F003F89DF8040050
:1050000016BD2146FFF7EABD70B500F014F80600A2
:105010000BD01922FFF748FE00F009F83146BDE831
:1050200070400FF2C112FFF7B9BD042070BD34818A
:10503000F560FFF751BD04460D461020FFF7FCBC9C
:10504000F8B500F012F807000DD03622FFF779FF0F
:105050003C817D8100F0ADF93946BDE8F8400FF2A2
:105060008D12FFF79BBD0420F2BD04460D46164687
:105070001020FFF7E1BC04460C20FFF7DDBC04461E
:105080000D4616460E20FFF7D7BC2DE9F041FFF77D
:1050900051FF070011D0069AFFF7BDFE3C813E7418
:1050A000FD6000F04FF97874FFF716FD3946BDE852
:1050B000F0410FF26D12FFF771BDFFF710BE38B56A
:1050C0001446104A15682A0006D0009302460B4683
:1050D00021460120A84732BD002032BD0A4A13688C
:1050E0001A0003D00A460146012018477047000005
:1050F000E00A0020415200005152000047520000D7
:105100008D4D0000F0140020F41400202DE9F04132
:1051100000F00DF898460C20FFF78EFC070004D035
:1051200000F016F83C81BD72E1E0FFF7D8BD0446FF
:105130000D46164670472DE9F041FFF784FE070043
:1051400004D000F005F8BC60FD60D0E0FFF7C7BDFB
:1051500032460421FFF7F1BC2DE9F041FFF773FE61
:10516000070006D0FFF7F4FFFFF7B5FE3872FD60C9
:10517000BDE0FFF7B4BD1078802802BF508840F230
:105180007F6188420CD190884FF680710140B1F563
:105190007E4F04BF00F07F00984201D1012070478C
:1051A000002070470023E6E71123E4E71223E2E73B
:1051B0000A23E0E70623DEE70723DCE70823DAE734
:1051C0001023D8E73023D6E73123D4E780B5122364
:1051D00000930123FFF7BCFD02BD000080B518233A
:1051E000F6E7000080B51923F2E700003623C2E796
:1051F0001078802802BF508840F27F6188420DD12C
:1052000090884FF6807101404FF68052914204BF62
:1052100000F07F00984201D10120704700207047C4
:1052200070B5FFF784FF1D23FFF7E2FF30B9324668
:1052300029462046BDE870401B23D9E7012070BDF8
:1052400080B51423C4E780B5152300930223C1E77A
:1052500080B5022300930423BCE70FF20D0142F254
:105260002F000AE00000000042F22F0347E004464E
:105270000D4616460C20FFF7DFBB70B504460D4601
:1052800000F014F806000CD081203070B4800120AA
:10529000F070FFF721FC2A463146BDE87040FFF769
:1052A0007DBC042070BD00208DF804000820FFF7AD
:1052B000C3BB2DE9F041FFF73AFF98460E20FFF7F8
:1052C000BBFB070009D000F00AF83D817E81A7F8FA
:1052D0000C80FFF701FC069A0CE0FFF700BD81206F
:1052E00038700120F870BC8070473D81FE60FFF788
:1052F000F3FB42463946BDE8F041FFF74FBC10785A
:10530000802802BF508840F27F61884204BF9088A5
:10531000984201D10120704700207047000038B545
:105320000446154600F00FF80FF221010091C2B2B9
:105330002B4621464FF61840FFF7BBFF32BD3C819C
:105340007D81BE8141465020FFF7D4BB4FF6184304
:10535000D5E70000F8B5FFF788FE07000DD0012261
:1053600000F022F83C727D7200F023F83946BDE867
:10537000F8400FF27902FFF711BC0420F2BDF8B536
:10538000FFF773FE07000DD0022200F00DF83C720B
:105390007D7200F00EF83946BDE8F8400FF2510278
:1053A000FFF7FCBB0420F2BD0521FFF7C6BB3C8123
:1053B000BD72FE60FFF790BB1078802802BF508856
:1053C00040F27F6188420DD190884FF68071014094
:1053D0004FF68062914204BF00F07F00984201D1F5
:1053E0000120704700207047000000000123E3E720
:1053F0000223E1E7DFF800F0F5B80110DFF800F074
:105400002DBF0110DFF800F011BF011000B583B00F
:105410000821ADF8001001900521ADF80210684692
:1054200043490968884707BDF0B589B004460D4671
:1054300016461F460823242200216846FBF7E6F89B
:105440000F983C49096806906B464FF47A70B0FBA0
:10545000F1F101FB07F0059001FB06F20E98ADF8A3
:10546000100029462046FBF7F1F8204609B0F0BDB0
:10547000FBF7D4B838B504460D46FCF7E4F910B193
:105480002046FCF7D2F900F013F800FB05F12046A6
:10549000FBF7C0F82046BDE83240FBF7BFB880B547
:1054A000FCF7D1F900B10120C0B202BDFCF7BDB9D3
:1054B000204909684FF47A70B0FBF1F0704710B5DD
:1054C00004460021FFF796FF204610BD70B584B05A
:1054D00004460820ADF800000D460420ADF8020097
:1054E0000C2013490968019016466846884758B948
:1054F000029949B18E602046FFF780FF15B128461A
:10550000FBF77CF8012003E03046FFF77FFF002027
:1055100004B070BD10B50446FFF774FFA04204D07C
:105520008468FFF773FF204610BD002010BD000007
:105530009C04002050000000002200F001B8000090
:10554000401810F0030308D0C91A1FD3DB0748BF67
:1055500000F8012D28BF20F8022D130030B41446A6
:105560001546103928BF20E93C00FAD8490728BF62
:1055700020E90C0048BF40F8042D890028BF20F81E
:10558000022D48BF00F8012D30BC7047C91818BF64
:1055900000F8012DCB0728BF00F8012D704700004F
:1055A000DFF800F013C1011000B583B00821ADF899
:1055B000001001900321ADF802106846DFF8C8140E
:1055C0000968884707BD00B58FB008233C22002139
:1055D0006846FDF7F1FFDFF8B40400F150010791D0
:1055E00000234FF4217108916A46012106910FF2C0
:1055F0003521FEF733FD0FB000BD10B584B000F0CB
:1056000008FA0120DFF88014DFF884440968ADF857
:105610000200684688479DF8040020700298A06048
:1056200004F13800FFF74BFFE060002304200190F5
:1056300041F288320020009004F114000FF2094179
:10564000FFF7F2FE0020606006211F20FFF77CFCC0
:1056500001208DF801000DF101020020ADF80A00D3
:10566000012101208DF800005020ADF808004FF412
:105670004870ADF806000020ADF804004FF47A70D1
:10568000ADF8020040F20530FEF7ECFC0DF10A0225
:10569000022140F20630FEF7E5FC04F144021E212F
:1056A0004FF44270FEF7DEFC04F16402072140F281
:1056B0000730FEF7D7FC6A4601214FF44470FEF72D
:1056C000D1FC02AA022140F21130FEF7CBFC0DF111
:1056D0000602022140F21230FEF7C4FC01AA0221A8
:1056E00040F21330FEF7BEFC0DF1020202214FF42E
:1056F0004570FEF7B7FC04F16C0215210020FFF79E
:105700001CFBA0210620FFF71FFCA0210720FFF7AC
:105710001BFCA0210820FFF717FCA0210920FFF7A0
:1057200013FC0020019001AA01208DF803008DF8E0
:105730000200042100208DF8010001208DF80000F6
:105740004FF48160FFF77CFC0DF1030201214FF45F
:105750008060FFF775FC0DF10202012140F202406A
:10576000FFF76EFC0DF10102012140F20340FFF74B
:1057700067FC6A46012140F20640FFF761FC4FF0EA
:10578000FF30FFF7D7FA4FF0FF30FFF78FFA00F046
:1057900085F94FF0FF3000F08BFA01208DF80300FF
:1057A00002208DF8020003208DF8010004200FF282
:1057B000E4218DF80000D1E9002301A80121C0E90E
:1057C000002300200DF1030200F0A4FA0DF1020203
:1057D0000121012000F09EFA0DF1010201210220B9
:1057E00000F098FA6A460121032000F093FA01AA1A
:1057F0000521042000F08EFA04F1900000F083FAF5
:1058000004F18400FEF702FE04F18800FFF721FA9C
:105810002078FFF71BFA2078FFF766FAFFF71DFDE7
:105820001FBD00002DE9F04E8EB0FFF7E6FE06AE7C
:105830004FF6FF7A964DDFF8509214E068884107E2
:1058400011D54FF6FB710840688005F11400FFF791
:105850000FFE02A9022000F099FA20B902AA012144
:10586000032000F057FA00F0D4F80A20ADF8020047
:105870004FF0FF30019000F0C8F80028DED108207A
:10588000ADF80C000920ADF80E0003A800F0BEF83A
:105890009DF81220059F002878D1BDF81000012442
:1058A000102804BF29788A4240D1388850451CD13D
:1058B000B87800073AD52869C0B36978491C69707F
:1058C00000F1080201794088FFF722FA162818BF74
:1058D000042883462AD02869297840880022FFF7C7
:1058E0001EFD584600F099F820E03878912802D043
:1058F000B02808D01AE07878102817D100210820A5
:1059000000F002FB12E0787816280AD17888082285
:10591000FFF705FD28B9012000F07FF82F61002472
:1059200004E0397907F10800FFF7D8FB77B36CB3CF
:105930003846FFF739FE29E006A94FF44170FEF71B
:10594000D5FC9DF818008DF800006A4670788DF837
:1059500001000821B0788DF8020000208DF80400C5
:105960008DF8030070798DF8070030798DF8060006
:10597000F0788DF80500002000F098F800F049F864
:105980000520ADF80200019400F03FF8E868FFF749
:1059900007FE00287FF452AFE868FFF7BBFD040064
:1059A000F4D0208801280AD00228E7D1A078002866
:1059B00018BF0228E2D102A900F0E8F9DEE7A078DA
:1059C0000128B9D0042808D0052802D0062809D01B
:1059D000D4E7142000F021F8D0E705F11400FFF718
:1059E00065FDF6E705F11400FFF742FDFFF7F6FA53
:1059F000504408A980B2FFF707FB0028BED06946D3
:105A000040F21530FEF772FCB8E76846D9F800108E
:105A100008470820ADF80000704710B51C4C2269FB
:105A20005AB120B1117902F10800FFF757FB206944
:105A3000FFF7BAFD00202061607010BD0146012013
:105A400009E00146022006E011494A8810434880D7
:105A50008868FAF7D3BD3EB50446FFF7DAFF0D4676
:105A600004200949ADF8020001906846096888479A
:105A700040B9029A32B11480957005488168C068B7
:105A8000FFF724FD37BD00009C04002024180020EF
:105A90007C07002001020304050000000FF204232C
:105AA0007D4810221321FFF704B900002DE9F043CF
:105AB0000024082885B00E469146784F00F28A806F
:105AC000DFE800F0050C1824303C48537D00082E18
:105AD00076D13246494607F1080076E0152E77DA8E
:105AE000152107F11000FCF733FD3246494607F156
:105AF00010006AE0152E6BDA152107F12800FCF77B
:105B000027FD3246494607F128005EE0152E5FDA90
:105B1000152107F14000FCF71BFD3246494607F10D
:105B2000400052E0152E53DA152107F15800FCF71A
:105B30000FFD3246494607F1580046E0152E47DA78
:105B4000152107F17000FCF703FD3246494607F1C5
:105B500070003AE0152E3BDA883715213846FCF7FD
:105B6000F7FC3246494638462FE00820ADF80800D9
:105B70000420ADF80A00039602A8DFF82481D8F8C3
:105B800000108847C8B9049DBDB1786807F1A0012D
:105B900088420AD00821ADF8001001900521ADF827
:105BA00002106846D8F80010884732464946284611
:105BB000FBF7DCFF7D603E700DE013240BE0072E49
:105BC00006D13246494607F1B000FBF7CFFF02E0AD
:105BD000182400E00224204605B0BDE8F083000050
:105BE0002DE9FE4990464A680A9C107852780B9D30
:105BF00000EB02201F46002680B242F62322274BEC
:105C0000801A03EB040C07D0401E052810D9801F12
:105C10001ED0263829D03AE0092C28D2C4F1080039
:105C2000854228BFC4F108053D800CF1080129E038
:105C3000D1F80CB0584600F07FF980B2A04216DBD4
:105C4000011B8D42A8BF051B3D800BEB040119E031
:105C500018780146A1420AD3001B8542A8BF0D1B3C
:105C60003D8058683A8801190DE0082C01D30726B9
:105C70000FE0C4F10700854228BFC4F107053D804D
:105C80000CF1B0013A884046FBF770FF01E03E801E
:105C90000A263046BDE8FE8964030020AC020020DD
:105CA0009C040020E15B00000000000000000000F8
:105CB0003EB504460820ADF800000420ADF802000F
:105CC0007549764800780968754D800001906846EE
:105CD0008847002814BF002002980100A86001D165
:105CE00013203EBD4FF6FF7000F042F9E00708D5E3
:105CF0000FF2B0131022112105F11400FEF7D9FFA5
:105D00003EBD00203EBD18B1654948600020704787
:105D1000112070473EB5002404281346604D31D849
:105D2000DFE800F003080D122500012928D11878BA
:105D3000287028E0012923D11878687023E0012910
:105D40001ED11878A8701EE0012919D11878E870C2
:105D500005F114030FF2710002900022FF20019060
:105D6000E91C11200090A86800F01CF90BE005293F
:105D700006D10522194605F10C00FBF7F7FE02E0FB
:105D8000182400E0022420463EBD000010B5024663
:105D900000240846042A424912D8DFE802F003052D
:105DA00007090C00097804E0497802E0897800E0EE
:105DB000C978017005E005220C31FBF7D7FE00E041
:105DC0000224204610BD000038B51046049A002475
:105DD0000AB10B2032BD0A78022A1ED14A68157812
:105DE000527805EB022292B24FF6F175521B012A4E
:105DF00004D9D21E02D0521E06D00BE001221A8016
:105E0000C968097801700AE005221A80C968FBF7A1
:105E1000ADFE04E01C800A2401E01C800124204621
:105E200032BDF0B583B00C780025022C18BF0125D7
:105E300026D14E6837787678089C07EB0626B6B2EE
:105E400042F60217F61B1DD04DF2EF67F61B01D08C
:105E5000B61E1ED11CB9012B03D00D2510E00B2559
:105E60000EE01078CA681070C8680D4A51689042F8
:105E700014BF0220002019B109680A0018BF884722
:105E80002846FEBD01250195009400F0EEF8054678
:105E9000F6E70A25F4E700009C040020D80400205F
:105EA000F4050020C95D0000235E00000000000032
:105EB000DFF800F055C0011038B50FF24D000F4C5F
:105EC0000F4D00F067F90F4800F021FA23681B68B6
:105ED000012201212846984722685268012128465C
:105EE0009047FDF7AFFCFDF7CBFCFEF7B5FAFFF7E7
:105EF0006AFBFFF7DDFF002032BD0000D801001073
:105F000000400340CC6C0000022818BF042881B078
:105F100010D0052807D101208DF800009DF8000061
:105F20000028FBD106E001208DF800009DF800005C
:105F30000028FBD101B0704700F10103810704D0B4
:105F400010F8011B89B18107FAD10268B2F1013161
:105F5000914311F0803F04BF50F8042FF6E710F88A
:105F6000011B11B110F8011BFBE7C01A70470000BC
:105F700038B54FF6FF74A0420DD10020654A137862
:105F800098420EDA21F8204001EB80050023401CE6
:105F9000AB70C0B2F3E700F0A9F810B104800021A3
:105FA000817031BD2DE9FE4F80460026B8F1000F0B
:105FB00082B006D0080004D0180002D0109F38002C
:105FC00001D1022035E00F9C00252CE0EDB2A9465E
:105FD00038F829004FF6FF7188421EBF08EB890A86
:105FE0009AF8020000281DD0029ABDF838100498D3
:105FF00000F02AF85FEA000B14D09AF80200C007FC
:1060000005D500F019F8012100F086F806439AF84A
:106010000200800706D500F00FF8022100F07CF89E
:106020000643F6B26D1C3B490978E8B28842CDD3ED
:10603000F0B205B0BDE8F08F019700949DF80C20F8
:1060400038F829005B46704730B5002400E0641C36
:10605000A3B28B4207D2A4B200EB0413DD689542D1
:10606000F5D1184630BD002030BDF8B5044606987D
:106070000D460026F0B9022B1AD11078517800EBAA
:1060800001270798C043B9B201420FD1E8680168FF
:10609000204600F012F8B9B288420CD0E8680168D6
:1060A000BAB2204600F00FF8064604E0802602E06F
:1060B0000D2600E00B263046F2BD80B500F016F844
:1060C00000B1807802BD70B504460D46164600F05A
:1060D0000DF840B929464FF6FF7000F007F808B9EF
:1060E000112070BD04808670002070BD10B50022A4
:1060F00000E0521C074C2478D3B2A34207D2D2B29C
:1061000031F822308342F4D101EB820010BD00202F
:1061100010BD0000D80400202DE9F04186B00D46E6
:1061200090461F46044603AB4FF6FF721B21FEF755
:10613000C6FF059040B3FF2102910246BDF80C1046
:10614000DDF834C001910DF11203002100912046C9
:106150003946E047064688B97889ADF81000E80767
:1061600005D5424604A92046FEF757FE05E00C9BE4
:10617000424604A92046FEF75FFE06462EB11B21CB
:1061800004A8FEF7ABFF00E01526304606B0BDE8D8
:10619000F08100000149086070470000A80200205B
:1061A00081B001208DF800009DF800000028FBD18F
:1061B00001B070477047000070B5FBF750FB044614
:1061C0000026DFF8C4520DE024FA06F0C00708D517
:1061D00005EB8600406820B1026811001CBF314603
:1061E0009047761C2868F6B28642EDD370BDDFF882
:1061F0009C020168DFF898020160DFF89802FBF763
:106200003EBB2DE9F0470E00F5B2044644BF86F0D0
:10621000204686F4C046A80000F1804000F5012029
:1062200004EA06030168DFF870723B4086EA010267
:10623000A1431943224004F4E023120EB3F5E02FEA
:1062400002F0010202D1CA0105D411E014F4E02FDA
:1062500008BF002A0CD001F4E022B2F5A02F04D030
:10626000B2F5C02F04D1052200E0062262F31241EC
:10627000DFF8287201603868E84000F0010805F195
:10628000804000F50839B00DB8F1000F00F0010AA8
:1062900003D1600248BF89F800A020020DD5FAF7AB
:1062A000A5F901223968AA4033024CBF13460023E6
:1062B000914319433960FAF79DF9B8F1000F03D003
:1062C000600248BF89F800A0BDE8F087002948BFF8
:1062D0000021800000F1804000F5012001F03F0125
:1062E0000268920941EA82110160704710B5DFF837
:1062F000B001006800F07F04FCF7BAFE012804D169
:10630000FCF7ACFE022808BF641C204610BD2DE936
:10631000F04FA1B00546FBF7B4FCFCF7A9FE002640
:10632000012804D1FCF79AFE022808BF0126DFF8F5
:106330007401C168C1F3815101294FF0010A04D1F0
:106340000068000E0AFA00F00643DFF85C01DFF88F
:1063500038410078DFF85491FFF7C8FF206020B182
:106360000146FF224846FCF75BFE4FF0000800277D
:1063700006E00AFA00F001F8097040EA08087F1CFC
:1063800055F82700C1B2FE290AD0FF29F7D02268AC
:10639000914203D226FA00F2D207EAD502206FE03A
:1063A0000920FBF76CFDC4F880500823242200214B
:1063B00017A8FAF74FF98DF874A017AA012104F174
:1063C000D400FAF74BF90027DFF8E4A00BE05046C1
:1063D000FFF717FF4FF0FF31F8B2FFF777FF00200C
:1063E000CBF804007F1C2068874213D226FA07F0FE
:1063F000C00704EB870B48BF0420F1D428FA07F04C
:10640000C00747BF17F8090055F82010F8B240F44C
:10641000C041DCE70823302200210BA8FAF706F977
:10642000DFF89050DFF89020287813900BAB002015
:106430000090102104F18400FAF704F908232822BF
:10644000002101A8FAF7EEF86868DFF870100790ED
:1064500000230020089001AA04F1A000FAF7EEF84A
:10646000DFF85C00016821F47C5141F400510160C7
:106470000120DFF850100860DFF84C1008600020A1
:1064800021B0BDE8F08F0000C81B0020E0200240D2
:10649000E0200260681C0020007F077FD0200240BF
:1064A00044130050A83F0050FB1C0020B81C0020E3
:1064B000007FC767F86C0000EF610000B961000061
:1064C000003009400C4009400800094001680A6892
:1064D0000A4482604B681A44C26008310160704708
:1064E0008168C268914208D101680A680A448260E2
:1064F0004B681A44C260083101608168491C8160A0
:1065000011F8010D704738B504460D46A068E168E2
:10651000884212D120686168884208BFFDF79AFD61
:106520002068227C016802B14944A16042680A44A3
:10653000E260083091422060ECD0A068401CA0606E
:1065400000F8015D31BD2DE9F0418AB000F108018C
:1065500005910268520801EBC201069100210791E2
:1065600008910168490800EBC101083100910179E7
:1065700001F001018DF8101040680099400801EB0E
:10658000C000019000200290039006E005A8FFF7EC
:106590009DFF07980899884207D105980699884277
:1065A000F4D101980AB0BDE8F08105A8FFF798FF83
:1065B000044614F0030603D105A8FFF791FFC61C9B
:1065C00025090F2D14D105A8FFF78AFF00F10F054B
:1065D0000EE007980899884204BF05A8FFF776FFE8
:1065E0000798401C079010F8011D6846FFF78BFFC5
:1065F000761EEED1002DCCD005A8FFF771FF064620
:10660000A00800F00300032804BF05A8FFF768FFF7
:10661000DDF800800299039F06EB002008E0A8F156
:106620000808A8F10801801A0A684968571839460D
:1066300058F8082C8A1A8242F1D340420C18AE1C3A
:10664000A7D0BC4206D158F8044B58F8040B2718C1
:10665000BC42F8D00298039914F8015B884217D124
:1066600000980199884208BFFDF7F4FC0098006883
:106670009DF81010029009B14844029000990298C8
:106680004968009A01440832884203910092E7D099
:106690000298401C0290761E00F8015D3FF479AF2D
:1066A000CFE7000080B501280CD002280CD00428C8
:1066B00002D008280AD00BE000201146126890474B
:1066C000002002BD0220F8E70420F6E70520F4E7E9
:1066D000FDF7C0FC00BF10B5044601E0FBF7BAFBB4
:1066E000B4FA84F0202800D110BD00F016F8F5DBD4
:1066F000401FFBF7C4FBF3E710B5044601E0FBF7CE
:106700003FFBB4FA84F0202800D110BD00F005F85A
:10671000F5DB401FFBF748FBF3E7C0F11F00C0B2F9
:10672000012181404C400528704738B505460120BD
:1067300068713D4C2879A8B1FCF778FF05462078B0
:10674000FF2805D12846FCF77CFF6FF0060032BD1C
:10675000401C2070C0B2012804BF6068FFF7BBFF77
:10676000284615E0FCF762FF21780A0004D1FCF707
:1067700068FF6FF0070032BD491E2170C9B239B9F8
:10678000FCF75FFF6068FFF7B7FF0020687101E06A
:10679000FCF757FF002032BD70B50446606810F06A
:1067A0007F4F02D06FF0020070BDFCF73FFF1E4E1E
:1067B0000546307828B17068FFF79EFF6068FFF7E4
:1067C0008AFF606870602846FCF73BFF002070BDC0
:1067D00080B5406810F07F4F00D00DE0FFF77BFFE1
:1067E000002002BD80B5406810F07F4F00D003E06C
:1067F000FFF782FF002002BD6FF0020002BD10B55E
:10680000044682B0A168606808601420FDF7C4F8EF
:10681000009010B96FF0030016BDA368034A0F2162
:10682000FBF79EFA002016BDA0040020A56600001C
:1068300010B50446FBF790FC2071002010BD80B518
:10684000FBF79BFC002002BD10B50446FBF709FADC
:106850006060002010BD10B504466068FBF77AFC4C
:10686000A060002010BD0000DFF800F00DC3011093
:10687000DFF800F081C60110DFF800F095B70110D5
:10688000DFF800F08DC20110DFF800F03DC201100A
:10689000DFF800F009C30110DFF800F045C0011077
:1068A000DFF800F0D1C70110DFF800F067BE01107B
:1068B000DFF800F011C80110DFF800F021C8011066
:1068C0000C381F283ED8DFE800F0103D3D3D3D3D2F
:1068D0003D3D3D3D3D3D3D153D3D3D1A3D3D1F246A
:1068E0003D3D3D293D3D3D2E3338DFF82801006810
:1068F00000687047DFF81C01006840687047DFF8E7
:106900001401006880687047DFF808010068C068FB
:106910007047DFF80001006800697047DFF8F40095
:10692000006840697047DFF8EC00006880697047D4
:10693000DFF8E0000068C0697047DFF8D800006841
:10694000006A70470020704700B589B00921684689
:10695000FFF78AFF09B000BD00B581B0FAF7B0FFBC
:10696000DFF8B400DFF8B4100068884218BF00F008
:1069700039F8DFF8AC00B0F5B26F03D001B05DF8C4
:1069800004EB30E001B000BD00B581B0FBF77AF850
:10699000012818BFFAF7E6FE0FF21D00FFF768FFA7
:1069A000FFF76AFFFFF76CFFFFF76EFF01B05DF8BE
:1069B00004EBFFF76DBF000000B581B0F9F752FEA0
:1069C000FBF710F901B05DF804EB0320FFF764BF9B
:1069D00010B504460320FFF75FFF2046BDE81040D6
:1069E000FFF75EBFFEE7FEE700B581B0FFF75CFF93
:1069F000DFF83000C06801B05DF804EBFAF7A2BE22
:106A0000DFF82410DFF8240088617047FFF750BFDB
:106A1000FFF752BFF001002098CA011070472820EC
:106A200090050000780100204401002000040000CF
:106A300080B5F9F7DBFD36490A7822B9354B1B687A
:106A40001A7001220A7080B2BDE80240F9F7D2BD87
:106A500038B5F9F7CBFD04462E4D284600F064F812
:106A6000A0B2F9F7C7FD284632BD70B50E461446F0
:106A7000F9F7BCFD85B227480168097809B900F02B
:106A800053F826B94FF480710122084612E03046CF
:106A900000F027F858B114B14FF0FF3020700820F3
:106AA000FBF782F92846F9F7A5FD002070BDB26812
:106AB0007168306800F042F81749012008601748F3
:106AC0000068C007FBD50220154909684968884756
:106AD00006460CB1002020702846F9F78BFD3046A1
:106AE00070BD4FF0FF3180B102681AB1403AB2F583
:106AF0007F5F0AD2426822B1A2F58072094B9A42A6
:106B000003D28068102838BF002108467047000073
:106B1000FA1C0020186D0000A802504208800240B4
:106B2000CC01001000FFFF0001680A782AB9012299
:106B30000A7040680068FBF7A2B9704710B50A4BAD
:106B40001C6824F480641C6009021202090CA4B2BF
:106B500002F4706244EA014442EA0141C0F3871042
:106B60001C600843586010BD1480024030BF70475D
:106B700038B5FBF7EFFFFBF79FFFFBF75AF804462A
:106B800004F00C000C2849D0600721D4FAF7F0FD7E
:106B9000054601210120FBF756F82349096801FB4E
:106BA00005F2904214D28220B0FBF1F01F4C291A5A
:106BB00004F10C00F9F72EFD04F10C00F9F72EFD9D
:106BC0000120FBF7B4F904F10C00FAF72EFE27E0E0
:106BD000200723D41648FBF769FE0428FAD0E20602
:106BE000144900D418B9086840F0010002E00868B0
:106BF000400840000860104C1048114D016841F0F9
:106C0000030101602020216889698847286820687D
:106C1000806B804701202860286801E0FFF7A6FF0D
:106C2000BDE83140FBF79ABF50000000D0090020BA
:106C3000004003408C210840B80100102422084085
:106C40002C200940EBC70CEEC90CF1CB0CF44B1413
:106C5000F74E19FA521DFD58250061310114420208
:106C6000184E031C5A04249305309300446C000012
:106C70000D070000C7100000A1610000E111000035
:106C8000A1610000DB130000291400002B14000098
:106C9000A1610000A1610000BF150000D515000032
:106CA000A1610000A1610000A1610000A1610000DC
:106CB0008D110000E9150000331600007116000068
:106CC000316A0000516A00006B6A0000060880808B
:106CD000070880800D2007C00E2007C01400C08068
:106CE000024000800300C08009400080084000800E
:106CF0000A400080FE000000FF00000000000000CD
:106D000000000000716B0000FF2000000101010085
:106D1000FFFF050508000000F61C0020146D0000B0
:106D200000000000000000007B756E6B6E6F776ED8
:106D30002D696E7374616E63652D6E616D657D0086
:106D40007B656D7074792D696E7374616E63652DEA
:106D50006E616D657D0000007B7374617469632DE5
:106D6000696E7374616E63652D6E616D657D000083
:106D700019E050F8041BCB0744BFA9F101035918CF
:106D8000121F0023042A41F8043BF9D25FEA827CF7
:106D90000B4604D54FF0000CA1F800C09B1CD10796
:106DA00044BF0021197050F8042B002AE1D170472C
:106DB00010B5074979441831064C7C44163404E078
:106DC0000A68081D114488470146A142F8D110BD48
:106DD0002C0000006C0100007FC80110C9BC01102C
:106DE00051B2011037C20110BDAD0110C1B1011087
:106DF00071BA011069BB011021C0011075FFFFFFBE
:106E00000C120000F00A0020000000003BF7FFFF1A
:106E100002000000020000007405000018000000DD
:106E2000780100202C0000001FF7FFFF0200000087
:106E300002000000A505000003000000EC01002096
:106E40000400000003F7FFFF020000000200000042
:106E50008305000003000000F0010020080000008E
:106E6000E7F6FFFF02000000020000003805000006
:106E70001A000000A401002024000000CBF6FFFF50
:106E80000200000002000000360500000C000000B7
:106E9000C80100201C000000AFF6FFFF0200000048
:106EA00002000000AA0400001B00000000010020F6
:106EB0004400000093F6FFFF020000000200000003
:106EC0001C05000006000000000200200400000075
:106ED00077F6FFFF0200000002000000FA04000045
:106EE00003000000F8010020080000005BF6FFFF2F
:106EF00002000000020000007104000023000000F6
:106F000044010020340000003FF6FFFF02000000B3
:106F100002000000B604000009000000E4010020A7
:106F20000800000023F6FFFF02000000020000003E
:106F3000D80000004603000008020020E808000016
:106F4000DFF800F059C501100548012808BFFFF718
:106F500003BD70470348012808BFFFF7F1BF704722
:106F600001000000010000000A18232A242A252A13
:106F7000262A272A282A292A2A2A502A02000000FB
:106F8000686F000000F00BF8002803D0FFF710FF37
:106F9000FFF7E0FF0020FEF78FFFFFF781FC0120E5
:106FA000704700B581B0FFF7CFFFAFF3008001B0AD
:106FB0005DF804EBFFF7E6BF44F22830C2F20000B0
:106FC000854646F6A370C0F200008047FEE7000049
:106FD00001000000000000000000000000000100AF
:106FE00000000000F0FFF1FFF2FFF3FFF4FFF5FFF8
:106FF00002000000E46F000045B50110016A0000C6
:1070000099A6011019B80110120001830100014373
:10701000C5A70D63E96915B007010018080020C570
:10702000A7000161106108100F07100000384035FB
:10703000002D400140028460005D08101700F80137
:1070400018A384070083057EA40306E0EA23060153
:107050000003040102351C102308047F1763040099
:107060003888604500C3003801AC526003A302AD0C
:107070000163026801438AFF0043022804FF0110F4
:1070800003B56100000E6360024C03002082A00A79
:107090004D6F64656C204E756D62657296F00302EB
:1070A000536572696119500F4669726D7761726537
:1070B000205265766973696F6E1CF0020348617235
:1070C0006418F00203536F667418500F4D616E75AB
:1070D0006661637475726572204E616D6518100388
:1070E000FE006578707C14046D656E74616C3212FC
:1070F0000D1910021001000207473C006030017CAE
:107100006F00105240102002E20A002010436A6F04
:107110001043B40210612052E320526C20D2BC20F4
:1071200052E420526E20D2D42052E520527020D258
:10713000EC2052E620527220C304032052E7205272
:107140007420D21C2052E820527620D2342052E9FA
:1071500020527820D24C2052EA20527A20125C2011
:1071600010032D360000430430010F3800012206C1
:107170002C1002051B0050BC166C587001746C007A
:107180000112C00C12A818100703030000F014002D
:1071900020F404432C01201966820001100206002D
:1071A000800CB03113F003983075FFFF0001F0013F
:1071B00050020106AD8B0200A4DAF0A456EBA41233
:1071C000E618253F43F40510524420C71807D4524F
:1071D000EC3056E8D4D2F530D22C3052ED3052EAB1
:1071E00078D2F630D2403052EE303001EC6F0001F0
:1071F00052F730434800A0D2FC40D2544052EF40F6
:1072000012EE40220443C206301268301C0243686A
:107210006172E3031DCE0320047374696320312778
:10722000D114F2023214F2023314F2023414F3369F
:10723000350001100A140953696D706C65424C45A4
:10724000505D1C0770686572616C05125012031363
:10725000020A65193C40030302F0FF0026122027B2
:107260008220281120833D5A8A12430C1E10E40507
:107270002104611647E519543001FF001413123040
:107280001C2104523804834002404D770310010151
:10729000005418F206541C1270182104527804523B
:1072A000800412CC2112082443F00B7C438006108A
:1072B00012A01C2104439C01046301004C410143C2
:1072C0004B180D12C824210452D00452D80452E0A5
:1072D0000452E8048397173D12050BC320000143B5
:1072E0004009131218082104522004522804523075
:1072F000045238045240045248045250048300009F
:10730000A862046415104370121CD0030BC2011054
:107310000001D20111129C48210452A40452AC0471
:1073200052B40452BC0452C4046178F1C701652010
:10733000F3090101E610034B220000B904430B22BC
:10734000246001FFFF020100030A0208100283010A
:107350000001A10CD0039C090020000152CC142094
:10736000023401002004523C041200011007F41CF6
:107370000020C01B0020C404211043283F08110135
:1073800070052001010000F81A10310152000110AF
:107390000708020020E80800200111C301000112C3
:1073A000A818210422000150026CDC0200015003E5
:1073B0005C080020030D100389690000D104F3016B
:1073C0000100012002180900201712000100020824
:1073D00002002052000152000112000100020800C8
:0273E0000000AB
:10FDC00038B504460D460DF08BFF084821680160E8
:10FDD00061684160A16881600CF0C5FB0CF0B5FB67
:10FDE0002846BDE8324007F0A4B800BFD84700203D
:10FDF0004F7D0100AFAA0100D7910100CBAC0100FB
:10FE0000B564010031AF01004743010063130100F5
:10FE1000813B0100A9FF00000A006E1902000000EA
:10FE200094CC01000200000090CC01000061310080
:10FE30002CFE0000010000000000D0020A050000B6
:10FE4000000000000201000000000000100000009F
:10FE500000000000EC000021000000000000000095
:10FE600054FE000038FE0000000000003CFE0000D0
:10FE700040FE000044FE000048FE00004CFE000072
:10FE800050FE0000B4460020DFF800F0419500105D
:10FE9000DFF800F071950010DFF800F0D195001048
:10FEA000DFF800F03D970010DFF800F065970010D4
:10FEB000DFF800F029980010DFF800F0F598001046
:10FEC000DFF800F0C9990010DFF800F0F999001090
:10FED000DFF800F0159A0010DFF800F0319A0010FA
:10FEE000DFF800F0A19A0010DFF800F0F59A00109A
:10FEF000DFF800F0159C0010DFF800F08D9C00107A
:10FF0000DFF800F0099D0010DFF800F0459D0010BB
:10FF1000DFF800F0D19D0010DFF800F02D9E0010FA
:10FF2000DFF800F04D9E0010DFF800F06D9E00102D
:10FF3000DFF800F08D9E0010DFF800F0AD9E00109D
:10FF4000DFF800F0CD9E0010DFF800F0ED9E00100D
:10FF5000DFF800F00D9F0010DFF800F0499F00105F
:10FF6000DFF800F0699F0010DFF800F0D19F00106B
:10FF7000DFF800F011A00010DFF800F031A0001051
:10FF8000DFF800F075A00010DFF800F0F1A000101D
:10FF9000DFF800F009A10010DFF800F0B5A10010B3
:10FFA000DFF84019087070472DE9FE430C46200425
:10FFB00054D5DFF83009007800F0A9FD05004AD0DB
:10FFC000DFF8247939680126002918BF11F1010FE3
:10FFD00007D0DFF81809007800F03BFD4FF0FF3044
:10FFE00038602878812802D082282CD02FE0002089
:10FFF0008DF808608DF80900AE88AF7995F8028019
:020000040001F9
:10000000B00A3F2807D1C6F3C21020B100F029F88A
:1000100000F02EF803E000F024F800F088F88146A4
:10002000284600F007FD9DF80800A0B1DFF8C008E1
:1000300001904B469DF8090000903A4631464046F3
:1000400000F0BAF907E0284600F064FB064616B156
:10005000284600F0EFFC84F4004000E00020BDE8FA
:10006000FE8302AB0DF109022946304670470000BD
:1000700038B500F07F04C00900F00700401E0428D6
:100080000D4652D8DFE800F0030C2C474C00122C30
:100090004BD12A7CE9682889BDE8384000F0E3BFED
:1000A0002889E968012C17D00B2C11D00D2C0BD00E
:1000B000132C05D0192C38D1BDE8324001F0D5B849
:1000C000BDE8324001F0BEB8BDE8344001F08CB864
:1000D000BDE8344001F07AB8BDE8344001F023B8FF
:1000E00028891B2C11D01D2C07D0432C1DD1AA8987
:1000F000698902F0C2F8002032BD6B7C2A7CE96875
:1001000001B0BDE8304002F0C5BA2A7CE968BDE81C
:10011000384002F0F5BA204601B0BDE8304013E2A5
:10012000204601B0BDE830408AE1012032BD0B46D7
:1001300040F21D41401A00F0978040F2E471401AED
:1001400000F09580801E00F098802A3800F097809B
:10015000363800F08F8040F29E31401A00F09480D3
:10016000401E00F09380401E00F09280801F00F03F
:1001700091804FF47F71401A00F08E8040F6FC3180
:10018000401A00F08C80801E00F08C80001F00F070
:100190008B80083800F08A80401E00F08980401E65
:1001A00000F08880401E00F08A80C01E00F08C8025
:1001B000401E00F08C80401E00F08C80401F00F03C
:1001C0008D80401E00F09180401E00F08980401E0E
:1001D00000F08F804DF6E231401A00F08C80401E16
:1001E00000F08D80C01E00F08E80401E00F08F80D9
:1001F000401E00F08F80401E00F09480401E00F0F2
:100200009780401E00F09680401E00F09780401EB0
:1002100000F09680401E00F09680401E00F0968010
:10022000C01E00F09580801E00F09680401E00F0F9
:100230009680401E00F09880801E00F09980401E3D
:1002400000F09B80801E69D0401E00F09C80401E04
:1002500000F09E80401E00F09E80801E00F09F8077
:10026000401E00F0A280A5E01889FFF70DBE986837
:10027000FFF70EBE986802F045BE02F09FBD598997
:100280001889C9B2FFF708BE02F09ABE02F0A7BDF6
:10029000FFF706BEFFF708BE188902F0BDBE9868DA
:1002A00002F073BEFFF704BEFFF706BEFFF708BEFD
:1002B000FFF70ABE1889D968C0B2FFF709BE1889CE
:1002C000D968C0B2FFF708BE1889FFF709BE1889C0
:1002D00002F0F1BDD9689868FFF706BEFFF708BEC7
:1002E0009A7A597A187A02F0FBBD1889C0B202F0E6
:1002F00000BEFFF701BE1889C0B2FFF701BE188922
:10030000C0B2FFF701BED9689868FFF701BE9868D0
:10031000FFF702BE1889C0B2FFF702BE1889C0B24B
:10032000FFF702BE59891889C9B2C0B2FFF700BEF3
:10033000FFF702BE1889C0B2FFF702BEFFF704BE86
:100340009868FFF705BE1889FFF706BEFFF708BEDD
:100350001889C0B2FFF708BE1889FFF709BE59898E
:100360001889C9B2FFF708BED9681889FFF708BE17
:1003700018895989C0B2FFF707BE59899A89188927
:10038000C9B202F000BE18895989C0B2FFF700BE99
:10039000188902F0E6BD1889C0B202F0CFBD5989B4
:1003A0001889C9B2C0B2FFF7F7BD1A69D968986851
:1003B00002F01FBD012070472DE9F843089C8046DC
:1003C00004F10C000F461546994680B200F020FB60
:1003D000060016D08020307086F8019040F27F60D1
:1003E0007080B780B57106F10C00F471B0602246E0
:1003F000099900F0BEFA31464046BDE8F44300F0EA
:1004000028BBBDE8F18310B502460020941E012CE4
:1004100002D9A41E02D004E0102900E004290ED065
:100420000CE0A2F12004402C04D2BDE8104010469C
:1004300003F03CBCA2F18001102900D3022010BDC2
:1004400070B5401E052882B00C461546DFF8A4643E
:100450004FD8DFE800F0030C15182A3D00F04BF8E8
:1004600008BBE2683146284603F006FF76BD00F07F
:1004700042F8C0B9E2683146284603F00DFF76BD68
:1004800003F031FF0FE0A06868B1DFF86C14016081
:10049000DFF868140988818091218171032101812D
:1004A0001421418123E0022076BDDFF854341B681B
:1004B000083300221B68002100209847B071010A10
:1004C000F171010C000E70723172042028700EE080
:1004D0004FF6FF70ADF8000002F00CFCADF8000024
:1004E0000222022028706946B01D00F042FA002066
:1004F00076BD012076BD257A667A3146284682E7A8
:1005000038B5012815461C4602D0022809D00DE056
:10051000049B0A462146284601B0BDE8304004F05D
:1005200017B80846BDE8324004F036BB0846BDE8BF
:10053000324004F03FBB0B4601281146184608BF65
:1005400004F042B804F04DBB2DE9FC410F461546BE
:100550000024DFF8A06380B3032849D0062837D0F1
:1005600007283AD008283FD00A2846D00B2852D076
:100570000C2869D00D2800F08D800E285ED00F2841
:1005800053D010284CD011283DD012283FD030280D
:1005900064D031286BD032285BD0332800F07F80C4
:1005A000342800F08080352800F08C80362800F058
:1005B0008C80372800F09180A7E078690190386935
:1005C0000090FB68BA7A797A387A04F059FB82E0B5
:1005D000F968387A04F07EFB7DE0FB68BA7A797AB4
:1005E000387A04F0C0FB76E0387A04F0F0FB72E071
:1005F000F968387A04F0C9FE6DE03A7B7989387A77
:1006000005F020F867E0B86805F059F863E0B868CD
:1006100005F089F85FE0F968B86805F0F1F85AE08C
:10062000B97A388905F03AF955E0387C0090FB68D2
:10063000FA7AB97A388905F080F94CE0FA68B97A23
:10064000388905F0B9F846E03989F86805F035F9D8
:1006500041E0F968B86805F0B5FC3CE03889798973
:1006600026282DD028282BDA04F044FE33E04FF65C
:10067000FF78ADF800803889FF2821DA26281FD0BE
:1006800028281DDA04F043FE4045ADF8000017D0DD
:1006900002200EE0B97A388905F0ECFC1BE0B8685E
:1006A00004F0BBFB17E0387A04F00CFC009038B182
:1006B0000420287002466946B01D00F05AF925E072
:1006C000022423E004F023FC05E07989FA683889E4
:1006D000C9B202F0D9FC044618E03F89B11D384682
:1006E00002F09AFD044640F201403F1A04D03F1F39
:1006F00004D0FF1E04D005E0022004E0102002E038
:10070000042000E00120287000E001242046BDE81C
:10071000F68100002DE9F04184B0044600208DF8F8
:10072000090001208DF80800A588A079A778042D7C
:10073000804669D8DFE805F068030A28440002AA69
:100740000DF10901204600F07BF85BE0002610283F
:1007500014D013280DD0142807D0152854D1E268DE
:10076000A17A208901F03CFF4CE0A06803F0C8FDAD
:1007700007E0A17A208903F0BDFD02E0207A03F0B2
:10078000B6FD8DF8086040E00026A8B1042804D02A
:10079000052806D006280AD036E0A06805F059FDE5
:1007A00033E02089E168C0B205F02CFD2AE000F0BA
:1007B00041F805F0E7FC25E0A06805F03EFD21E0EA
:1007C000062821D8DFE800F01B20140F20040A00BF
:1007D0002089E168C0B200F05FFE13E000F02AF863
:1007E00000F02BFE0EE0E168208900F004FE09E035
:1007F0002369A27BA189A06800F0D2FD02E0A06875
:1008000000F0A7FE064600E00126204600F012F99F
:100810009DF8080050B13648019033469DF8090014
:100820000090424629463846FFF7C6FD002004B036
:10083000BDE8F08161892089E268C9B2C0B2704721
:10084000F8B50D4681792B4F00240429164626D091
:10085000102910D0112912D0122915D0132922D015
:10086000142926D015292CD017292FD018290ED0BD
:1008700019290FD033E0007A05F00EFE24E0817ACA
:10088000008906F062F826E006F08AF823E006F018
:1008900073F820E0C168008906F009F80FE080686D
:1008A00002F05DFE10E0C268817A008902F064FE09
:1008B00005E0837C028AC168007A02F001FD0446EB
:1008C0000EE0008902F099FD347009E00269C16808
:1008D000007A02F0BAFDB8710120287000E001240E
:1008E0002046F2BDDA48002044430020E1480020C1
:1008F0001647002010470020020202001AFE0000E6
:100900004043002000B583B00821ADF800100190ED
:100910000B21ADF802106846DFF8741609688847A5
:100920000EBD1FB58DF806100824ADF800408DF8F7
:1009300004000624DFF858168DF808200393ADF85C
:10094000024068460968884704B010BD80B505209C
:1009500006F07FF800F0EDF90C2000F001F802BD80
:10096000DFF82C160968ADF802006846084706F063
:100970007FB803E011F8013B00F8013B13465A1E13
:10098000002BF7D170471144491E03E011F80139DB
:1009900000F8013B13465A1E002BF7D1704770B583
:1009A00004460D46A8B206F07FF8060003D02A469A
:1009B0002146FFF7DEFF304670BD10B513465A1EC4
:1009C0003BB110F8013B11F8014BA342F6D00020D7
:1009D00010BD012010BD10B5044610460A46014660
:1009E000204606F081F8204610BD03F073BCDFF806
:1009F000A425DFF8A435126A11541B7805E0DFF84E
:100A00009835DFF890251B78126AC018115470478A
:100A100010B5040001D1002010BD04F10C0080B21B
:100A200006F042F828B1002101600481FF218172A3
:100A30000C3010BD80B508B9052002BD10F8021CAD
:100A4000FF2901D0042002BD0C3806F03AF800203E
:100A500002BD38B50C46010622D5DFF838150A78F4
:100A6000FF2A08BF4D7805D0DFF82C351B78096ABE
:100A70009A188D5CFF2D02D1FFF768FF0EE000F0A1
:100A80009BF90146FF2004F8020C23460022284669
:100A9000FFF747FF48B12046FFF7CCFF012032BDEA
:100AA0002146BDE83840002200E032BD70B50D009F
:100AB0000446164618D0200648BFFFF747FFDFF868
:100AC000D81409788C4204D32846FFF7B3FF0320DB
:100AD00070BDA5F10C000168002904BF817AFF29CF
:100AE00004D02846FFF7A6FF052070BD8472012EB2
:100AF000DFF8A004294603D1001D00F055F802E0FC
:100B0000001D00F039F800F033F8002070BD2DE929
:100B1000F0410446DFF88404DFF878740068804709
:100B2000804678680026002503E005B9064650F89F
:100B30000C0C50B110F8021CA142F6D1002D08BFD8
:100B40000546F4D000F014F805E04FF400412046CB
:100B500000F0A4F825B132462946381D00F031F8DE
:100B6000DFF83C140968404688472846BDE8F08114
:100B70004FF40041204642E038B500F00FF8002164
:100B800045F80C1C216811B9256006E0114651F8A2
:100B90000C2C002AFAD141F80C5C27E10446DFF85E
:100BA000FC0300680D46004738B5FFF7F7FF2168E2
:100BB00045F80C1C2560DFF8E8130968BDE83440EF
:100BC000084770B5044600F014F8A5F10C0123683D
:100BD0000A689D420CBF226046F80C2C00220A6075
:100BE000FF228A72BDE8704002E1DFF8B4130968A1
:100BF0000847DFF8A80300680D46164600472DE9B0
:100C0000F0410446DFF89003DFF8885390F8008045
:100C100020060E462CD50420FFF7FAFE070008BF79
:100C2000042039D04FF6FF7038807E80A7F10C0683
:100C30002878FF280FBF6D78296A40440D5CFF2D8E
:100C400005D13846FFF7F6FEFFF780FE0EE020469E
:100C500000F0B2F8FF21B1723B460146002228465F
:100C6000FFF75FFEC0B13846FFF7E4FE012013E056
:100C7000444510D200F028F8DFF82813096831F84D
:100C80001420324321F81420FFF7AFFFE868FFF784
:100C900039FE002000E00320BDE8F08138B50C46A5
:100CA000BD490978884205460CD200F00DF8BD49CF
:100CB000096831F81520A24321F81520FFF795FFA8
:100CC000002032BD032032BDB4480068004730B573
:100CD000B04C0020606083B005F048FF06F095F846
:100CE000AD480578680005F0DFFE20626A00FF214C
:100CF000FFF771FE0222FF21A01CFFF76CFE06F039
:100D0000DBF800F016F81420A14D2968ADF80200B8
:100D1000684688470198206100F00BF81520ADF86F
:100D200002006846296888470198801E606100209B
:100D30003EBD0820ADF80000704730B587B00820F0
:100D4000ADF808001B20ADF80A0001200390914D7A
:100D50000FF27D008E4C21680590E8690690A86925
:100D6000049002A888470499A96108B1FFF7EEFD35
:100D700000F053F8FFF7DDFF0A20ADF802004FF056
:100D8000FF300190684621688847F1E780B500216F
:100D9000804A0A449378FF2B01D1907001E083428E
:100DA00003D141F08000C0B202BD491C0229EFD33B
:100DB000FFF7CCFDFF2002BD10B580F08004022CAF
:100DC000A8BFFFF7C3FD73482044807810BD000022
:100DD00038B50446FFF778FF05466E48C1698C4276
:100DE00004BFC068FFF78EFD4FEA0500BDE8344040
:100DF0006B490968084710B50446608850B9A07966
:100E0000FFF7C4FFFF28E07102D16FF0030010BDAF
:100E1000002010BD6FF0010010BD2DE9F04F8BB028
:100E200005F0C7FF00245FEA000B03D005F0D3FEF6
:100E30004FF0FF3B574DA868010003D0804701E009
:100E4000FFF784FD0820ADF808000720504E3168F8
:100E5000ADF80A0002A888474F499DF80E20049F6C
:100E60000978E8B9002600E0761C8E42E8D2286AAC
:100E7000805D9042F8D1F6B2FF2EE1D017F8080C51
:100E8000FFF784FF17F8061C012908BF387002D04D
:100E9000022908BFB87039463046FFF7DAFDD1E7BE
:100EA000404F3868E4B230F8140018B9641CE0B25E
:100EB0008842F5D3E0B28842DFF8E480DFF8DC90C6
:100EC0001DD2D9F8000080473968E4B231F814A087
:100ED000002200F047F8344A2C70514652F8242082
:100EE000204690478246FF202870D9F800008047AE
:100EF000396831F814204AEA020200F033F805F0AC
:100F000058FF07465F452AD007B9284F6869B8429D
:100F100038BF0746D9F8000080470446FFF709FFAD
:100F20001C20ADF80200A869316801906846884726
:100F30000821E869ADF81410401C1321E861ADF8F0
:100F40001610099006971A49A8690891079005A8F4
:100F5000316888470798A861204600F005F80BB073
:100F6000BDE8F08F21F81420D8F80010084710B51C
:100F700048B1002300E05B1CDCB2944205D2DBB236
:100F8000C45C8C42F7D0002010BD012010BD0000D1
:100F9000D8470020A444002018FE0000DC470020B1
:100FA000E0470020F0470020F0FD00008EC2F52849
:100FB000D10D0100DFF800F0F5950010DFF800F02A
:100FC00031960010DFF800F05D9600100A4610B56B
:100FD000052A18BF042A03D0062A18BF072A08D1F9
:100FE0000C24484B62431A4422F8301D90700020B4
:100FF00010BD022010BD38B50D46044628880528CE
:1010000018BF042803D0062818BF072801D1686834
:1010100008B9022032BD0121204605F096FC08B92E
:10102000142032BD4FF6FE70844207D0204605F0F2
:10103000C8FC2989884201D21B2032BD3248007881
:1010400000282946204603D0BDE8344003F08CBB7D
:10105000BDE8344003F03EBB80B52C4B00931346F3
:101060000A4601211AE070B50D4684B004461646C2
:10107000EB88AA886988288801F082FE58B1002090
:1010800002900196042000902A46214B122120460E
:1010900003F0B6FA00E0182004B070BD03F0E2FAE5
:1010A00002BD38B504461B480129017011D11A4808
:1010B0000088051DADB20120FFF77CFF94FBF5F021
:1010C00082B2284601B0BDE8304000230021FFF77E
:1010D00075BFBDE832400020FFF76CBF03B50D4877
:1010E0000078012881B003D102AA01A9FFF76AFFA5
:1010F00007BD094A001F1080034801707047064869
:10110000008870478C480020E646002069480100AE
:10111000E7480100DF480020FC460020704700003F
:101120006E490860704780B5002200920B4601228C
:101130006B4900F0BAF802BD80B50A88172A05DBB2
:10114000002200920B4603226649F2E7022002BD0C
:1011500038B50D460446A878012818BF02280DD1DD
:10116000288800281CBF6868002807D0022103F0E7
:101170005DFD00902B4605225B4931E0022032BD27
:1011800038B500F01EF81CBF6868002806D000F0D3
:1011900036F800902B460722544921E0022032BD48
:1011A00038B500F00EF81CBF6868002807D002218F
:1011B00003F03CFD00902B4609224D4910E002202F
:1011C00032BD0D46044628880028704738B500F027
:1011D00024F808B100F013F800902B460B22454983
:1011E000204600F062F832BD38B500F016F808B1BC
:1011F00000F005F800902B460D223F49F0E7012151
:1012000003F014BD38B500F008F808B1FFF7F7FF98
:1012100000902B460F223949E2E70D4604466868E4
:10122000704738B5FFF7CDFF1CBF6868002807D0AE
:10123000022103F0FBFC00902B4611223049CFE73E
:10124000022032BD80B5002100910023132270E7F7
:1012500038B50D460446A86810B1052103F0E6FC38
:1012600000902B4617222749BAE780B5002100914C
:10127000002319225DE738B5FFF7CFFF10B1032136
:1012800003F0D4FC00902B461B2209E038B5FFF791
:10129000C4FF10B1032103F0C9FC00902B461D22AE
:1012A0001949204605F0A7FF32BDF8B50446069857
:1012B000009015461E46204605F09DFF07000AD106
:1012C00006480268100006D0012D04BF3078451C86
:1012D000E9B2204690473846F2BD00000848002099
:1012E000FB6F010017700100317001008B7001006D
:1012F000CF700100EB7001004371010067710100C4
:101300006B710100A5710100D5710100DFF8581C57
:101310000870704738B5DFF8544CDFF8545C20761D
:101320002878C00005F0C0FBE061C8B1002108E0EA
:101330004FF6FF7220F8312000EBC10300225A6003
:10134000491C2A789142F3DB052000F0AFF8207E9B
:1013500001F058F8BDE83240DFF8180C05F037BA54
:1013600031BD38B50C46200418D5DFF8000C007EDE
:10137000FFF7CDFB05000ED02878B02808D128460D
:1013800000F0FDF820B1297905F1080003F01CF9FF
:101390002846FFF74FFB84F4004032BD002032BDE9
:1013A0007CB506001C460DD0ADF800108DF802206B
:1013B0000196684600F0B8FF05001AD1CCB17689D5
:1013C000300001D1022514E00C2005F06DFB08B9B6
:1013D00013250EE00021016086808460DFF8981BF1
:1013E0000A6812B9086004E00A4611680029FBD1B6
:1013F0001060284676BD30B50C46DFF87C1B0546EC
:10140000086883B0002201E00246006898B1838832
:10141000AB42F9D10368002A0CBF0B60136005F0E2
:1014200050FB6946284600F0CDFF010002D10CB107
:10143000019921603EBD01203EBD70B550BB012920
:1014400026D1DFF8280BC169002300E05B1CDFF820
:10145000204B2478A34217DA31F833404FF6FF755A
:10146000AC42F3D0002400E0641C467EE5B2B542F5
:10147000ECD201EBC305E4B26D680C266643AD5BAC
:10148000002DF1D0012070BD1078BDE870400DE056
:10149000182070BD022070BD0022002803BFDFF8B5
:1014A000CC0A407E08700222104670472DE9F843AE
:1014B000DFF8B87A0446002078760C25F869DFF862
:1014C000B06A406805FB04F870B105F0FAFA002034
:1014D00006E0F969C0B201EBC00100224A60401C7D
:1014E0003278C1B29142F4D3307808FB00F080B278
:1014F00005F0DAFA5FEA000928D0307808FB00F23C
:1015000000214846FFF767FA00200FE0516805FB0D
:101510000CF34FF0000E21F803E019440CF1010C1C
:10152000C1F808E0A445F1DBC144401C3278C1B2E7
:10153000914208D2F969C0B201EBC0024FF0000C31
:10154000C2F80490EEE77C76002000E01320BDE8AE
:10155000F28301460020C90705D50023102201218E
:10156000DFF8180C1CE77047DFF80C1A096821B186
:101570008A888242FAD188687047002070472DE936
:10158000F04186B004460020ADF8100001208DF82F
:101590001200DFF8D859286A38B9FFF7B0FD05F016
:1015A00083FA0028286200F0E280182200212846F1
:1015B000FFF711FA2079461C02284FF6FF7817D062
:1015C00006282CD008282FD00A2833D00C2857D032
:1015D0000E2800F08B80102800F08D80122800F07B
:1015E0008F80162800F09380182800F09780BBE0C9
:1015F000FFF785FD288029466088FFF79DFD0028BC
:101600002189288804D0814228BF01462980A0E092
:10161000814228BF0146608802F045FFA4E004A98A
:10162000204600F0AEF87DE004AA0021204600F03C
:101630002CF977E000F0A0F8070052D0608805ABE5
:1016400042460B2102F084FF03006B6024D0207916
:10165000BDF81620039000953946BDF8140002909D
:101660000020019000F026FA070004D16088294686
:10167000FFF7ACFD29E0162F686808BF00272BE0B4
:1016800000F07AF807002CD0608805AB42460D21A7
:1016900002F05EFF686020B92089ADF810001127C4
:1016A00045E02179BDF8162003910346BDF81410DA
:1016B0000291618901910095394600F0FBF907001C
:1016C00006D160882946FFF78FFD002841D12AE026
:1016D000162F686808BF002703F083FA380001D18D
:1016E00021E001272089ADF810001CE004A9204664
:1016F00000F06EF916E004A9204600F0E9F911E0C7
:101700000DF1120204A9204600F086FA0AE00DF15C
:10171000120204A9204600F0C0FA03E004A9204602
:1017200000F029FB0746380011D0162F11D0607841
:1017300014280CD0207928702F712946BDF810008C
:1017400068806088FFF7EFFC08B1012601E0162FE2
:101750000AD160882B46F2B2162102F09AFE18B127
:10176000F1B2284602F030FF204602F0C9FD9DF894
:10177000120006B0BDE8F08120890DF1160100F0DD
:10178000B9BE2DE9FA47044686B06088DFF8DC5719
:1017900005F0C5FD80460DF1120000F0D4F80027D9
:1017A00081464FF0FF0AB9F1000F5BD009E0BDF8A8
:1017B00010304354BDF81000696892B2000A885492
:1017C000571CBFB2A8F1050087424BDA207903907D
:1017D0000026A8F1070080B20290019605F11A00D8
:1017E00000902B6ABDF812206088494600F0CCFBBF
:1017F000002802BF6A8B208A904214D1296A60694E
:10180000FFF7DBF878B1686858B900F055F907219F
:1018100002F09EFE686020B9069920890880112098
:1018200030E0B9F80A60BDF81220618904AB48467F
:1018300000F086FE002E8146B5D06868C655781C3B
:101840006A6880B231121154411C4A1C6868B9F1AF
:10185000000F89B2ABD100F801A092B2686800F81D
:1018600002A0571CB8B248B13F04B80C28802946E2
:101870006088FFF785FC28B1162003E006992089CF
:1018800008800A2008B0BDE8F0872DE9F04304463F
:1018900085B060888846914605F041FD851EADB251
:1018A000DFF8C87601E0401C2081A81E39898842F3
:1018B0002FDB5FEA08002CD104A800F044F80600F2
:1018C00027D070892081BDF81020317A608800F01F
:1018D0009DFD5FEA00081CD120793B6ABDF810200D
:1018E00003903146A81E80B200F0EBF800F0E2F859
:1018F0005FEA00080DD173897A8B396A608800F03D
:101900002AF85FEA000804D120894FF6FF71884267
:10191000C9D1388901000AD0798890FBF1F038806C
:1019200039466088FFF73CFC50B1162008E05FEABA
:1019300008002089A9F8000008BF4FF00A084046B7
:1019400005B0BDE8F0830090237B6189208904F114
:101950000D0200F0A0BD2DE9F846824689461546E5
:101960001E4605F0DCFCDFF804460746208990B9E6
:1019700000F0A3F80921504602F0EAFD606008B9C2
:10198000112023E0A81C60803A1F208901466B18B3
:101990009A4206D203E06088A91C8842F4D0012054
:1019A00014E0401C2081606846542089411C21813C
:1019B000310A62681154606823892A4649461844EE
:1019C000FEF7D7FF2089281820810020BDE8F28685
:1019D0002DE9F047044686B06088DFF890750D4623
:1019E00005F09DFC0026A0F10109A0F1010814E01A
:1019F0003888798B0346C9188845BCBFA9EB00001D
:101A0000788378687A8B396A1844FEF7B2FF388891
:101A1000798B0818761C3880B6B2A0898642BCBF84
:101A20003888404534DAA06810F8162000EB4600EC
:101A300004A9407802EB002080B200F05BFD0100B9
:101A400009D14FF0010A00F02BF8786808B103F0D3
:101A5000C8F85046DDE02079BDF8102003901FFA49
:101A600089F000F02EF83B6A00F024F80028824646
:101A7000E9D178680028BBD100F01EF80F2102F0F0
:101A800067FD00287860B3D100F00AF81120E1E783
:101A900060883946FFF7B6FB0028DBD01620D9E76F
:101AA000A06810F8161000EB4600407801EB00200B
:101AB00028807047608867E2608800234FF6FF72D5
:101AC000704702900020019007F11A0000907047C3
:101AD0002DE9F047044686B06088DFF890548946C7
:101AE00005F01DFC059004F10D0204A80090237B75
:101AF0006189208900F0CFFC0026B24607464FF0EE
:101B0000FF0810E0696801F8068080B2696801F892
:101B10000080461C68686A8B296AB6B28019FEF795
:101B200028FF688B8619B6B2FFB1BDF81020397A4C
:101B3000608800F06BFC5FEA000A13D12079BDF8E1
:101B40001020039039460598801F80B20290002033
:101B5000019005F11A0000902B6AFFF7ABFF5FEAD6
:101B6000000A10D07889A9F80000002E48D06888B3
:101B700096FBF0F0288029466088FFF752FB00288A
:101B800047D0162045E07EB9FFF796FF112102F0FD
:101B9000DFFC686020B97889A9F80000112038E0DE
:101BA000688B001D688009E0688B6988021D91427E
:101BB000DDD10599891F80198142D8DB6968788950
:101BC000885579896A68701C80B2090A1154461CCC
:101BD000BDF8102061890DF11203384600F0B0FC09
:101BE0000746701C002FB6B28CD06A68BDF8121080
:101BF000915580B2BDF812106A68090A115488E73D
:101C00005FEA0A002089A9F8000008BF4FF00A0A1D
:101C1000504606B0BDE8F087FEB504460D46208963
:101C2000164602A900F066FC07002ED0387A80061E
:101C30000BD5BDF8080000F0A1F903000BD06088B7
:101C4000122239469847070020D1607C002814BF33
:101C50005220207901E00E2718E00190002000902A
:101C60006389E2682189608800F08AFA070007D159
:101C7000607C68B96088FFF7E5FA48B11620FEBDC0
:101C8000162F03D10027377002E001272089288012
:101C9000607C00B100273846FEBD2DE9F0410446C6
:101CA00082B00D4660889046012104F04EFE002768
:101CB00018B9142060700E205BE02089694600F09E
:101CC00019FC060051D0307A80060BD5BDF8000013
:101CD00000F054F9030013D060881222314698476F
:101CE000070043D16688304600F008F928B94FF65E
:101CF000FF7000F003F9A0B3068000219B4E02E0C4
:101D00000E2733E0491C737ECAB29A4229D2426838
:101D1000C9B20C234B4313441A88002AF2D10C2277
:101D200004F108011846FEF724FE002088F80000A0
:101D30000C2204F108013046FEF71BFEA2896088E0
:101D40000023172102F004FCB06060B1A289216970
:101D5000FEF70FFE60883146FFF77AFA40B1162091
:101D600007E0092702E0112700E0012720892880E9
:101D70003846BDE8F6812DE9F043044683B060881B
:101D8000894600F0BBF800265FEA00084CD0207AB4
:101D9000012845D1414604F1080000F051F8A0B1F6
:101DA000D8F804701820019078880090BB88BA6831
:101DB0003988608800F0E4F90646162E02D100202A
:101DC000B8602DE060B3388828E000270EE001906D
:101DD00068880090AB88AA68608800F0D1F9064650
:101DE000162E18D10020A8607F1CFFB25F48407EED
:101DF000874215DAD8F804100C227A430A441546B3
:101E000029880B000CD07B1C83421DBF90890028C1
:101E100016201820DBE7002EE6D02888A9F800005D
:101E2000404600F080F82EB96088FFF71EFA20B116
:101E3000162003E0162E08BF00263046BDE8FE83BC
:101E40002DE9F84F0C460020002700264FF00C0B20
:101E500046490DE0984202BFBCF8025093B2AB4233
:101E600024D1BCF80430DF19BFB29A1892B2761CA4
:101E70004B7E9E420FDA63680BFB06FC9C44BCF869
:101E8000003043B10028E5D1BCF80470BCF8022052
:101E90001846BA18EAE7022E2DDB38004FF0000989
:101EA00004D002F087FE5FEA000801D1002023E0A1
:101EB000CA461AE00BFB0AF14518A96859B1AA886D
:101EC00008EB0900FEF755FDA88848441FFA80F981
:101ED000A86802F086FEBAF1000F04D00C2200219F
:101EE0002846FEF778FD0AF1010AB2456068E1DB99
:101EF000C0F8088087800120BDE8F28F10B51B4A2A
:101F0000D269002100E0491C194C2478CBB2A342CD
:101F100007D2C9B232F831308342F4D102EBC100AA
:101F200010BD002010BD70B5044600250BE0B06860
:101F300008B102F056FE0C2200213046FEF74BFDA0
:101F4000002030806D1C0949497EE8B2884207D2E2
:101F50006068EDB20C216943461830880028E6D14C
:101F60004FF6FF70208070BDFE4600201C48002008
:101F700054480020272201004048002080B5FFF788
:101F8000F3FA00B1806802BD2DE9FE4F0D46804690
:101F9000287AC00693461E464FF0000A0CD55846D4
:101FA000FFF7ECFF030000F0E4800A2229464046D8
:101FB00098470028824649D128780C9F0D9CDDF86F
:101FC0003890022816D100F018F94FF42051401A29
:101FD000012810D9801E3AD0401E14D0FD3876D08A
:101FE000401E00F07D80401E6AD0401E6FD0401E13
:101FF00000F09180A7E0002C2AD1E86801783980B0
:102000000278416883E0002C22D101203880002131
:10201000E868007830706889401C80B200F06AFA85
:10202000398860B10278921C5118398041897170E9
:102030004189090AB17002784168F01C68E0081D06
:10204000388004220021701CFEF7C5FC93E0002CB0
:1020500062D1E8680488042038803470200A7070E7
:102060000DF10201204600F045FA05001ED0EC6893
:10207000BDF802204FF6FF786B46414600F060FA4B
:1020800040B92B786A688B48022105F0F7F808B947
:10209000ADF80080207802280AD161680222301D44
:1020A000FEF767FC3888801C388001E0ADF80040FE
:1020B000BDF80000B070BDF80000000AF0705AE0F2
:1020C00054BBE8680168404605F05CF902E01CBBBF
:1020D000E8680088022139803070000A70704AE098
:1020E000E868FEF744FC82B2A242B8BF4FF0070A8C
:1020F00041DB944208BF002206D009EB0401914263
:10210000B2BF4A46121B92B23A80E9682144304677
:10211000FEF72FFC2FE014B14FF00B0A2BE0E8681C
:102120000721398001783170417871704188B17030
:102130004188090AF17001793171C1887171C088D3
:10214000000AB07117E05846FFF70EFA00281CBFCE
:10215000D0F800C0BCF1000F0BD00F980290CDF862
:10216000049000943B46324629464046E04782466A
:1021700001E04FF00E0A5046BDE8FE8F08460020F1
:102180002DE9FE438046894617461E4602A9484669
:1021900000F0B0F905002CD0BDF80800FFF7E4F915
:1021A00000281CBFD0F804C0BCF1000F1FD00A9853
:1021B0000B9C0090019433463A4629464046E0473E
:1021C0000646B8B9FE2C15D02878022812D100F0A6
:1021D00014F842F6021188420CD13878797800EB75
:1021E000012082B24946404600F047F802E00E2640
:1021F00000E001263046BDE8FE836868017840783B
:1022000001EB002080B27047E0B58DF80820022372
:10221000120A8DF80920FE2201920022009202AAE1
:10222000FFF7AEFF0EBD7CB50129044605D002299B
:1022300022D1012104F089FBF0B92046FFF75EFEB0
:1022400008B1FFF770FE01A800904FF6FF7502235A
:10225000194A2946012000F01EF90BE0F0680168D8
:10226000204605F075F8BDF80420002329463046C5
:1022700000F066F90600F1D173BDF8B50F4F0446C2
:102280003878FF280D46164611D00A20FEF7C0FB0D
:1022900068B1B12101704480002141700171C58095
:1022A000068101463878BDE8F440FEF7D2BBF1BDA7
:1022B000000000009CCC0100A4CC0100FE460020E0
:1022C00070B5DFF8385A28780624604304F0ECFB38
:1022D000DFF82C1A086008B9132070BD0020FF2217
:1022E00006E03380401C0023F270B2703371C0B23C
:1022F0002B7898420ADA0B6804FB00F61E4400288B
:102300000CBF4FF6FE734FF6FF73EAE70FF2514032
:1023100001F0EAFF0FF61510FEF702FF0FF6551059
:1023200004F055FA002070BD70B50446208868B1ED
:1023300060680378426800F040F948B96068037843
:102340004268DFF8C00900F03AF908B9022070BD10
:10235000A078C01F0A2801D3182070BDDFF8A85943
:102360002888010004D02188C0F58030884201DA35
:10237000012070BD0C2004F097FB060001D1132052
:1023800070BD002008E06268298880B202EB00126C
:10239000401C5181491C298081B222889142F2D38C
:1023A0000020306008222146301DFEF7E2FA6868FE
:1023B00010B96E6004E0084601680029FBD1066090
:1023C000002070BD38B502460846DFF83C194C685D
:1023D000002301E02346246894B1A5686D899542E5
:1023E000F8D12268002B0CBF4A601A6018B108228D
:1023F000211DFEF7BEFA204604F063FB002032BD2B
:10240000012032BDDFF804190870704710B504468A
:1024100010461422114203D000F0DAF8012204E041
:102420004A0608D500F0D4F8002201462046BDE84F
:10243000104004F0CCBAC80701D4022010BD00201F
:1024400010BD70B505460E46B0061C4609D51046AF
:1024500000F0BEF801462846BDE87040012204F0B5
:10246000B6BA8820064210D0104600F0B1F80146F6
:1024700006F00802284604F0AAFA010009D0617AA1
:1024800041B1217A012904D070BDB00701D40320E5
:1024900070BD002070BD2DE9F0478146DFF8680867
:1024A00044688A4690461E4600E02468FCB1002736
:1024B00000E07F1CA188B8B28842F6D2A068BFB203
:1024C00000EB07156889484528BF8245F1D33EB126
:1024D000297868683346424604F0D0FE0028E8D0E8
:1024E000089810B1A16849890180284600E00020C1
:1024F000BDE8F087F0B5DFF81028546800E02468E4
:10250000E4B1A5686E89B042F9DBA788BA19904298
:10251000F5DA4FF0000C01E003F1010C1FFA8CF228
:10252000BA42ECD21FFA8CF305EB0312B2F80AE0C0
:102530008645F1D101B10E801046F0BD0020F0BDFE
:102540002DE9FC4104460027ADF804704FF6FF78F2
:102550006089404515461E4608D001AA0092401CDD
:102560002378626880B2FFF796FF07462378626897
:1025700000F023F830B923786268DFF8880700F0AC
:102580001EF808B160890CE023786268DFF88007E4
:1025900000F015F858B11FB1BDF80400A84203D0EF
:1025A000284600F0D2F803E07889404400E06089D2
:1025B00006B130803846BDE8F681DFF858070221C1
:1025C00004F05CBE80B500F0F3FA00B1008802BDF3
:1025D00080B500F0EDFA08B1807802BD102002BD90
:1025E00070B5012982B00446154616D0032918D0CB
:1025F000052925D0072927D0092929D00B292BD037
:102600000D292DD00F292FD0112931D0132933D0E6
:10261000172934D0192936D039E02946FEF783FD31
:1026200033E0FEF76CFDADF8000069462046FEF78A
:1026300083FD06002CD12988204601F034FF27E0D5
:102640002946FEF785FD20E02946FEF799FD1CE0AE
:102650002946FEF7A5FD18E02946FEF7B7FD14E070
:102660002946FEF7C1FD10E02946FEF7CBFD0CE040
:102670002946FEF7D6FD08E0FEF7E4FD05E0294611
:10268000FEF7E6FD01E0FEF7F0FD064600E002265B
:10269000304676BD2DE9FC410E46054617461C46E0
:1026A00001A900F092FA804638BB380014D000200F
:1026B000ADF8000069463088FFF71CFF012FBDF818
:1026C000000018BF0027FFF783FF01463A4628465F
:1026D00004F07DF9804680B931462846FEF7D6FDE4
:1026E000804650B9019DFF2C07D0AB1C1E22294605
:1026F0000FF2555001F0B9FEEC704046BDE8F6818E
:102700007CB50D460446164601A900F05EFA17286E
:102710001AD0300014D00020ADF800006946288897
:10272000FFF7E8FE012EBDF8000018BF0026FFF7F6
:102730004FFF01463246204604F049F9010003D11B
:1027400029462046FEF797FD76BD10B50446FFF7F3
:1027500039FF01001CBF611E0C18A0B210BD0000A3
:102760002DE9F0430D4689B08146A87800261E2841
:10277000174614D1484600F03CFA06001EBFB07858
:10278000FE28FF2822D0002000900022AB78F078AD
:10279000494601F03FFE304600F040FA16E01228AC
:1027A00004BF6878012813D0484600F022FA0600DA
:1027B0000ED0327910000BD0100607D4A978484605
:1027C00001F084FE307940F080003071002069E033
:1027D000DFF838452078FF2812D0A878811E172905
:1027E0000ED200F08AF958B1A87800F0B3F938B1E8
:1027F000287810B96878012804D1A878122801D067
:1028000006204FE0A87800F078F9844602A80090EE
:10281000AB88AA6869782878E0470028804640D1CC
:10282000A87800F097F9024602A9484690478046EA
:10283000D8B9AB78042B34D002A8009000222078BD
:10284000494601F0E7FD804658BBA97802A801F08F
:1028500055FE08B100203870A878122804BF6978A6
:1028600001291ED0EEB130711BE06878C8B9A87894
:102870008DF800008DF804806946A878042818BFF8
:102880000628BDF80800ADF802004846FEF74BFCEC
:1028900028B16B4601221621484601F0FAFD4FF09F
:1028A0000008404609B0BDE8F083002070472DE9DC
:1028B000FE430D46804628886988814201D3010085
:1028C00001D101206DE00021ADF8041002914FF616
:1028D000FF7900E0401C002100910023698800225C
:1028E00080B2FFF7D8FD070037D0BDF804000028FC
:1028F00038D16B464A460521404601F029FE0400C6
:1029000001D111204DE002943878022806D101202F
:102910008DF80600BDF80000860827E002208DF83B
:1029200006001221BDF8000090FBF1F6387810285F
:1029300013D1788904F8010B102200F034F8103418
:10294000BDF80400401CADF80400B1B2BDF80400AD
:10295000884202D278894845BCD1BDF8040080B9CC
:102960000A201EE09DF806000128DFD138780228F1
:10297000F3D1788904F8010B022200F014F8A41CAA
:10298000DEE701A94046FEF7E3FB48B101AB0522B3
:102990001621404601F07DFD10B1029802F021F9A8
:1029A0000020BDE8FE837889000A04F8010B204668
:1029B0007968FDF7DEBF10B582B04C880888844284
:1029C00001D3020001D1012016BD00F016F808B9AC
:1029D0000A2016BD002016BD10B582B04C880888AC
:1029E000844201D3020001D1012016BD00F005F898
:1029F00008B90A2016BD002016BD002200924A1D0B
:102A00000B79214647E510B5044682B00846694671
:102A10000088FFF76FFD08B9012016BD017ABDF8E7
:102A200000202046FFF7F2FC16BD70B582B00646C6
:102A30000D46002401E0641CA4B2A888844229DA6F
:102A4000286810F8142000EB44006946407802EB37
:102A5000002080B2FFF74EFD50B9286810F814101E
:102A60000170286800EB440149784170012076BD6F
:102A7000017ABDF800203046FFF7C8FC0100DAD02B
:102A8000296811F814200A70296801EB4402527871
:102A90004A7076BD002076BD10B50C4682B0208805
:102AA0006188814200D308B9012016BD2379994875
:102AB000621DFFF784FD08B9102016BD00200090AC
:102AC000237961882088621DFFF7E5FC08B90A2098
:102AD00016BD002016BD38B504460D466946288847
:102AE000FFF708FD08B9012032BD017ABDF80020CA
:102AF0002B462046FFF7A5FC32BD022814D004283F
:102B000014D0062814D008281AD00A2812D00C286D
:102B100012D00E2812D0102812D0122812D0162847
:102B200012D0182812D013E07B4870477B487047BA
:102B30007B4870477B4870477B4870477B487047AD
:102B40007B4870477B4870477B4870477B4870479D
:102B500000207047022814D0042814D0062814D06E
:102B6000082814D00A2818BF0C2812D00E2812D01A
:102B7000102812D0122818BF162810D0182810D0EC
:102B800012E06F4870476F4870476F4870476F4852
:102B900070476F4870476F4870476F4870476F487D
:102BA00070470FF2090070470020704700207047FF
:102BB0005549496800E0096829B18A68528982420A
:102BC000F9D1081D70470020704710B50C4600F081
:102BD00010F860B104B120608078FE2801D1172080
:102BE00010BDFF2801D1002010BD162010BD02200D
:102BF00010BD10B5424A1268002100E0491C3F4C4C
:102C00002478CBB2A34207D2C9B206234B43D45A8D
:102C10008442F3D1D01810BD002010BD10B5044679
:102C2000A01C01F02AFCFF20E07010BD10B50C467E
:102C3000FFF7DFFF30B101794A1C944204BF01F075
:102C40008001017110BD000010B582B004001EBFEC
:102C5000A078FF28FE280BD0002000901E2321889A
:102C6000E078172201F0D6FBFE20A070FF20E07074
:102C700013BD000070B504464FF6FE70844282B06A
:102C800037D008004FF6FF760AD12046FFF7B1FF94
:102C900078BB3046FFF7ADFF05002AD0048073BD36
:102CA000012906D12046FFF7A4FF050021D02E8080
:102CB0000BE002291DD10121204603F046FEC0B9D8
:102CC0002046FFF796FF050013D0A878FF280ED006
:102CD000FE2807D0002000901E23E8781422214609
:102CE00001F098FB2846FFF799FFFF20A87000200D
:102CF000287173BD0448008870470000DD4800203B
:102D00004C4800209CCC01001846002000470020C1
:102D1000A0CC010098CC01000D70010027700100CB
:102D200049700100D17001001F710100477101005D
:102D300093700100EF7001007D710100C37101000B
:102D4000AB280100AF280100B7290100D9290100F3
:102D5000072A01002B2A0100992A0100D72A010025
:102D6000DFF800F0DD8A0010DFF800F0A18B001022
:102D7000DFF800F0D5700010DFF800F09D5800106B
:102D800030B540F67B44851FA5423CBF8D1FA54250
:102D900012D2814210D3B2F5FA7F0DDAA3F10A0004
:102DA00040F67744A04207D2501C49004843B0EB9C
:102DB000C30F8041C00F30BD002030BD80B505F08D
:102DC0005AF88DF8000005F0ABFE77490020087036
:102DD0006A4676490880012140F6034063E080B5E9
:102DE0000FF26022412141F20200FFF7B9FF0020FB
:102DF00002BD7CB5002808BF00294FF620442DD124
:102E000062BB01A805F0C7FD9DF8040000EBC000FF
:102E1000451DEDB2284603F047FE060018D02020DD
:102E20003070042070700020B0709DF804000028FD
:102E30000CBF0022721D311DF01C05F099F83246BE
:102E40002946204606F08AF8304603F03AFE15E09F
:102E500004218DF801102020072106E005F088F8F4
:102E600004218DF80110202000218DF800008DF83C
:102E700002106A460321204606F070F8002076BD55
:102E800080B500208DF800006A46494800788DF82A
:102E90000100042100208DF80200464800788DF8DA
:102EA000030042F20200FFF75BFF002002BD012099
:102EB00070470120704738B5044642F2160529468E
:102EC0000020FFF751FF204605F0E9F88DF80000DB
:102ED00020B16A4601212846FFF742FF002032BD9B
:102EE00080B5012305F0B5FA00F01BF842F21E0090
:102EF000D9E780B5012105F069FB00F012F842F234
:102F00001D00D0E780B530B1014608222A48FDF700
:102F100030FD002000E0122000F003F840F663408E
:102F2000C1E78DF800006A460121704780B542F282
:102F300013010C20FFF718FF002002BD80B51D21F2
:102F40008DF8001004218DF8011010B9FFF710FF63
:102F500000E011208DF802006A4603214FF61D4063
:102F60000DE080B51C208DF800006A4604208DF825
:102F7000010003210C208DF802004FF61C4005F0E3
:102F8000EDFF002002BD05F03FBD80B530B10B491B
:102F900002780A7040784870002000E01220FFF7A5
:102FA000C0FF42F201007EE7244F0020264F0020A0
:102FB000284300202A430020C4480020BC480020A9
:102FC00000B585B06A460DF1020101A8FFF7D4FEF5
:102FD0008DF80800222107208DF8090002AA02A816
:102FE000817002218DF80B109DF804108DF80C10E3
:102FF000BDF802108DF80D10090A8DF80E10BDF8FD
:103000000010C171090A017241F201000921FFF7A4
:10301000A7FE002005B000BD10B582B004460DF13A
:10302000030105F0BEFC8DF800008DF80140200A78
:103030008DF802006A46042141F20540FFF790FE38
:10304000002016BD000000800000C000000000E469
:103050000000002822000000000000040000F7C368
:10306000B37E00000000000000000000000000002F
:103070000000000000000000000000000000000050
:1030800000000000000000007CB5164600244FF44C
:103090008063C21ADFF8105C21D0521E26D0521E67
:1030A00029D0521E2ED0521E33D0521E38D0521E5E
:1030B0003FD0521E44D0521E47D0521E4ED0521EF8
:1030C00074D0521E79D0521E00F07E80521E00F045
:1030D0008380D21E4DD0083A00F08A8090E001290A
:1030E00011D1307803280ADA687393E002290AD1F3
:1030F000308828858EE0012905D1307802287DDAD4
:10310000A87387E0012979D13078052876DAE87349
:1031100080E0012972D1307802286FDA287479E0D2
:1031200010296BD11022314605F13C00FDF721FC3E
:1031300070E0012962D1307802285FDA687469E0B2
:1031400001295BD13078287564E0042956D13068B4
:10315000DFF8B01C884251D2E8625BE000294DD113
:1031600003F00CFA10B900F076FC17E00120E875C6
:1031700050E0072942D10622711C6846FDF703FC86
:1031800030780022694600F060F906460A2E40DADF
:1031900003F0F4F930B9304600F069FC502001F03A
:1031A00089F822E0A9190120087733E0012925D107
:1031B0003078022822DAA8742CE001291ED1307858
:1031C0000A281BDAE87425E0012917D13078C11FDD
:1031D0000A2913D268751DE001290FD1A97D307825
:1031E000A875002908BF012814D100F0D8FB11E010
:1031F000012903D116B1307868760BE0182409E074
:10320000282806DA022904D1318802F073F804462E
:1032100000E00224204676BD38B500244FF48063D8
:103220000D46C21ADFF8801A1CD0521E1CD0521E46
:103230001CD0521E1CD0521E1CD0521E1CD0521E1E
:1032400020D0521E20D0521E20D0921E21D0521EBD
:1032500021D0521E21D0521E21D0521E21D00A3A16
:1032600022D024E0487B20E0088D24E0887B1CE00D
:10327000C87B1AE0087C18E010223C312846FDF794
:1032800078FB1BE0487C10E0087D0EE0C86A2860EF
:1032900014E0887C09E0C87C07E0487D05E0887D73
:1032A00003E000F0C5FB00E0487E287006E0282817
:1032B00003DA02F02CF8288000E00224204632BD18
:1032C0002DE9F04F93B0914698460AAA0023C2E92F
:1032D0000033DFF8D47900F0B8F88246BAF10A0F6B
:1032E00071DA4FF0060B0BFB0AF404F1200000F03A
:1032F0007FF80028787B0CBF9DF80D500025022830
:103300000CBF01260026B8F1080F0BFB0AF004D110
:10331000290758BF00F1220B01D500F1210B1C2217
:1033200000210CA8FDF757FB0CAA1C215FFA8BF0BB
:1033300000F0A2FF05F0010558B99DF84A00C01F32
:103340000A2806D200960CAB00222946484602F015
:10335000F4FA1422002101A8FDF73DFB04F124003A
:1033600001AA00F0D1F880B91022FF2101A8FDF7D1
:10337000FEFD50B904F1250005AA042100F0C5F8AE
:1033800001AA2946484602F017FA0AF1700006AA77
:1033900000F0BAF8A0B906A800F040FA002406AD83
:1033A000204635F8201041B106A901EB80018A784A
:1033B00035F820104846FEF727FF641C042CEFDB8D
:1033C000504600F010FBB8F1040F04BF787B0228D0
:1033D0000AD1797C002001B10120B97B01B104211F
:1033E0000143484602F046FE002013B0BDE8F08FCE
:1033F0006A460E21C0B200F03FBF70B503F0BEF8C0
:1034000010BBDFF8A448E07D01280AD100F023FBBF
:103410000020E0750A22002104F11C00FDF7DBFA10
:103420000CE000256619307F012804D1284600F001
:103430001EFB002030776D1C0A2DF3DB502000F0BE
:1034400039FFBDE87040AAE270BD2DE9FF41164684
:103450000D460A246A79022102F0C002C02A08BF80
:10346000002102D0402A08BF0121020018BF022813
:1034700003D0032818BF00290DD1284600F07AFA9E
:1034800004460A2C3CDA002E3AD006222946304661
:10349000FDF76FFA34E0022910D10027DFF88089A8
:1034A0000E207843404406222946C01DFDF785FAC8
:1034B000F0B97F1CFFB20A2FF2DB21E001291FD1F6
:1034C00000270620784323306A4600F01DF850B9E3
:1034D0001022FF216846FDF74AFD20B929466846BB
:1034E00002F070FD20B17F1CFFB20A2FE9DB07E07C
:1034F0000A2F3C4604DA1EB13146204600F023FA7A
:10350000204604B0BDE8F0811021C0B200F0B4BE86
:10351000F8B50C4615264FF6FF71884215460BD1BB
:1035200000272A462146384600F021F900B100263E
:103530007F1C0A2FF5DB10E003F0D9F960B1811D83
:1035400040790022FFF781FF0A2806DA2A46214641
:1035500000F00DF9002600E014263046F2BD10B54B
:10356000DFF84447217B2063262001F0C3FE207B47
:10357000BDE81040FDF7CABE38B504460025080076
:103580000DD1DFF88008DFF87C38B2FBF0F021467F
:1035900003FB102002F0ABF9050003D00121204607
:1035A00002F07CF9284632BDF0B585B0DFF8F85658
:1035B0000446A178286B062900F0CB80092900F089
:1035C00088800A2920D00B2905D00E2979D00F290F
:1035D00000F08E80C0E050B10668300007D020694E
:1035E0000090637B227B6189E01CB047B4E02069D6
:1035F0006189002814BF0120E86A02F078F90028E8
:10360000F4D06089012191E060780026002846D13D
:10361000A079C00743D5686B002840D10E2200F086
:10362000A2F8A08803F063F90600DFD06769CFB184
:10363000387C8DF80600062207F111016846FDF777
:1036400098F90622B11D06F10C00FDF792F9062249
:1036500007F11101B01DFDF78CF9387C40F0020034
:10366000707107E070798DF806000622B11D68467A
:10367000FDF77FF9A1799DF80D00890801F001019E
:1036800008438DF80D002146684600F0D6F828B9A9
:10369000287B0221FDF7B3FA00205EE01526286B97
:1036A000002859D04368180056D06278A0880121BC
:1036B0009847300050D02B6BA0885B6832460321BE
:1036C00045E0002848D04368180045D062780221C0
:1036D0003CE0E0780022211DFFF7B7FE0A283BDA24
:1036E00006235843253004F10C0200F038F833E08B
:1036F000A088A97C09B1E97C18E0697B09B905219A
:1037000014E003F0F4F8060026D0A07AC00710D524
:10371000707901000DD0E168C1F3402149B96A46D2
:10372000B11DFFF792FE20B9A088032102F0B6F880
:1037300012E07179A08804F1080200F0E1FA286B28
:1037400050B14368180007D000220021A088984794
:1037500002E0A088FFF751FE012005B0F0BD042172
:10376000C0B200F099BD00216846FDF734B970B5CC
:1037700006460620704388B00C461546203004AA41
:10378000FFF737FE002838D10622FF2104A8FDF7F5
:10379000EEFB90BB70366A461021F0B200F06CFD73
:1037A00048BB684600F03AF8200009D110220021F9
:1037B0006846FDF7DCFBF0B91022FFF7D4FF12E0FA
:1037C000694600F01DF838B9280016D06946002077
:1037D00000F016F888B104808178A9420BD085707A
:1037E0000DB900210180684600F018F86A461021E2
:1037F000F0B200F051FD012000E0002008B070BDE3
:10380000002231F82230834202D101EB820070475E
:10381000521CD2B2042AF4DB00207047002130F899
:103820002120D24320F8212000EB8102491C93780B
:10383000DB4304299370F2DB70472DE9F043DFF896
:103840006844DFF8DC958046606B85B00F460E2635
:10385000E8B9B8F1000F18BF002F70D0404600F053
:1038600089F80A28207612DB002506FB05F00622DF
:10387000FF214844FDF77BFB40B96D1CEDB20A2DDA
:10388000F3DB607E002814BF25780A252576207E8C
:103890000A2854DA0625616B6843C9B920304246CC
:1038A0000E21FFF75DFF207E00F09DF81022FF2122
:1038B000FFF75AFF207E703000F046F9207E7043FB
:1038C0000E2241464844FDF754F86763002037E074
:1038D0008A683AB121301C21FFF742FF616B00205A
:1038E0008860F3E70A693AB122301C21FFF738FFFC
:1038F000616B00200861E9E74A693AB12330102181
:10390000FFF72EFF616B00204861DFE7CA6882B1D4
:1039100024301021FFF724FF606BC06800F1100213
:10392000207E68432530FFF71AFF616B0020C860D6
:10393000CCE7A07D08B100F04CFA00F0D2F90120EC
:1039400005B0BDE8F08330B50A2885B00C4600DA32
:103950000CB902200CE0062358432030FFF748FD45
:10396000050004D1062269462046FDF702F82846E4
:1039700005B030BD70B504460025DFF8A4640E2004
:103980006843062221463044FDF717F808B128465F
:1039900070BD6D1CEDB20A2DF1DB0A2070BD38B58B
:1039A000002400F029FA0620604320302A460E2128
:1039B000C0B200F061FC58B10622FF212846FDF795
:1039C0000AF80622FF21E81DFDF705F800206873BC
:1039D000641C0A2CE5DBB448807D08B100F0F9F9DD
:1039E000BDE831407DE138B50A210A23AE4A5C1EAC
:1039F000DBB2134413F8013C834201D1214603E0BA
:103A00002346E4B2002CF2D1C9B2084605E01418EE
:103A1000135C657815546370401C0928F7DB09298D
:103A200005DABDE838400A21052000F035BC31BD7B
:103A300070B500240025DFF8E8630E2068430622F5
:103A4000FF213044FDF793FA00B9641C6D1C0A2D68
:103A5000F3DBE0B270BD10B50024204600F007F89B
:103A6000641CE4B20A2C01DA0100F6D010BD2DE985
:103A7000F0478D4D297E884290B0814609D1287B40
:103A80000121FDF70BF9287B0221FDF707F900F072
:103A9000BBF9062000FB09F505F1200607AA0E2157
:103AA000F0B200F0E9FB002845D10622FF2107A86B
:103AB000FDF75DFA00283ED11C22FF21FFF754FEDE
:103AC0001022FF210BA8FCF786FF0E22FF2107A87A
:103AD000FCF781FF07AA0E21F0B200F0DDFB0646DD
:103AE00005F1210000F02BF8824605F1220000F0DC
:103AF00026F8804605F1230000F026F8044605F17B
:103B0000240000F021F8074605F125006A4604214B
:103B1000C0B200F0C1FB48EA0A012143394340EA40
:103B2000010509F170000BAA1021C0B200F0B4FB2E
:103B30002843304300E0002010B0BDE8F0876A461B
:103B40001C21C0B200F0A8BB6A461021C0B200F030
:103B5000A3BB10B5B34C207304F14C0002F0FBFD85
:103B6000FFF71DFF22460A21052000F085FB30B13A
:103B70000020C0F109012154401C0A28F9DB10BDC6
:103B8000F0B50D46280485B0474C25D5207BFCF7C1
:103B9000BEFF04001DD021780120B0290FD0B1292B
:103BA00005D0D02904BF2046FFF7FEFC0DE02079A8
:103BB00060B92289E1886088FFF7AAFC06E02179D4
:103BC00004F1080000F000FD00E010B12046FCF711
:103BD00031FF85F4004065E0A80709D500210020E9
:103BE000FFF72BFE002885F0020550D102214FE09F
:103BF000E80752D5606B8688A06B4FF6FF7748B90F
:103C000004F12A0000900223874A39460120FEF77A
:103C100042FCA06385F00105A16B21B3FF20039056
:103C200002200290002001900DF11200009004ABE0
:103C3000628D3046FEF7A8F968B99DF810009DF82E
:103C4000111000EB012290B228B1A06B418992B211
:103C50003046FFF75DFC628DA06B00233946FEF70E
:103C60006FFCA06398B9206B70B1436818000BD04B
:103C7000606B8088002201219847606B236B8088ED
:103C80005B6800220321984700F0BEF803E00121A1
:103C9000207BFCF7B4FF284604E068074CBF85F0A2
:103CA0000400002005B0F0BD4844002010B52038C5
:103CB000062390FBF3F30624012204FB13000528DE
:103CC0000DD8DFE800F00305050707090E2904E019
:103CD0001C2902E0102900E0042908BF0022104638
:103CE00010BD80B5FFF7A4FE0228ACBF02200A2059
:103CF0008DF800006A460121052002F043FA01BD5B
:103D000070B5AAB006460C46154602F0F0FD08B99B
:103D100014205CE0A422FFF726FDADF80060414EC0
:103D2000F07B317D8DF8040001F00102707D8DF88B
:103D3000A0002798400842EA400020F0020248080C
:103D400000F0010042EA400020F48072080900F00F
:103D5000010042EA002020F40072480900F001004E
:103D600042EA402020F48062880900F0010042EA23
:103D70008020890820F0040001F0010140EA810060
:103D8000279001A9307C020008D04870102206F16B
:103D90003C010DF10600FCF7ECFD01E0002048704D
:103DA000707C28B11CB1279840F0020027900120B8
:103DB0009DF899100843B17B8DF8990001B1042159
:103DC00008438DF899002946684601F019FD2AB08C
:103DD00070BD38B5FCF778F8002400F00DF8062225
:103DE000FF212846FDF7C3F810B92946FCF770F803
:103DF000641C0A2CF1DB31BD0E21094861434518D2
:103E00007047000040420F0010B5064C606B18B1BF
:103E1000FCF710FE002060630A20207610BD000031
:103E20004847002048440020A4CC0100002010B5E1
:103E3000DFF828446070207082B000F004F900219F
:103E400000F0FEF80098B0F5801F02D100F0E3F812
:103E50000BE020B900F0DFF800F01DF905E000F0FC
:103E6000BDF800F0ABF804206080607816BD38B56E
:103E7000DFF8E8432578290001D0012032BD6188B0
:103E8000C1F5805189B2814200D350B900F09EF84B
:103E90000020607000F0FFF818B96578280008BFAE
:103EA0000125284632BD13B5DFF8B003BDF8021076
:103EB00040881C46C9B200F0CBF8010009D0DFF8F9
:103EC000A003049A0003A3B2000E05F0C1F800207D
:103ED00016BD012016BD2DE9FB43DFF8806382B0DB
:103EE000002070701746BDF80A90708898465FFAF7
:103EF00089F100F0ADF80446B8B1002501E0641C7A
:103F00006D1CEDB2B9B28D420CD2D548000301232D
:103F100001AAA1B200F094F89DF8040018F8051069
:103F20008842ECD0B8B285423ED0BFB2F81C4110F6
:103F300000EB9170801087007088BFB23818001DA8
:103F4000B0F5805F03DD00F041F800F0A4F874885C
:103F50004FF6FF70ADF800003D1947F4004000F047
:103F600027F8BDF80200C0F30E0000F021F8BA05F2
:103F7000120E4146204600F016F95FFA89F141F42D
:103F80000040ADF8000000F015F8BDF80000C0F3E7
:103F90000E00ADF8000000F00DF87078010004D1BB
:103FA0007088391D08187080002005B0BDE8F083C6
:103FB000ADF8020001226946A8B2F4E080B54FF4E2
:103FC0008010009001226946002004E080B50020A6
:103FD00000900122694600F0E6F801BD70B5A148E5
:103FE00000688047044600F023F905469C4800031A
:103FF0000021000E05F04DF805F056F8064628465B
:1040000000F00EF90EB100F006F92046BDE8704050
:1040100095490968084710B582B040F6FC7400F075
:1040200012F8214600F00CF8009810F1010F03D1AE
:10403000241FA4B2042CF2DA8849201D488013BD45
:10404000000E05F005B88648000304236A46704751
:1040500038B50C46051F00E02D1FADB2042D18DB4E
:10406000FFF7F1FF2946FFF7EBFFBDF80010BDF8A1
:104070000200A14203D1C0B2281A80B232BD0104AD
:10408000EAD4011D8D42A8BF281AE3DA002002F00D
:10409000E0FC002032BD2DE9F04F83B000F0C8F8FD
:1040A0006E4FDFF8BC9183467888041F4FF0FF08FD
:1040B0000025A4B24FEA193A2DE04FF0885081193B
:1040C000042201A805F006F8BDF804005FFA88F1A3
:1040D00088421BD0BDF80600301A061FB6B2301F4A
:1040E00040F6FC718842E8D3BDF802004FF08851D9
:1040F0004A19031D211A9BB289B25FFA8AF004F0B3
:10410000A7FFBDF802004019051DADB2BDF80200C1
:10411000201A041FA4B2042C2ADB04236A46214679
:104120005FFA8AF004F094FFBDF800004FF6FF71CB
:10413000884218BF002810D1BDF80200010448BF12
:10414000241FE7D4001D8442E0DA002002F081FC45
:10415000584600F065F8002023E00004D6D4BDF8EE
:1041600000005FFA88F18842D0D080462E1FB5E764
:10417000FFF734FF45B12A464FF0885109F104009A
:1041800004F082FFFFF71AFF584600F049F87878EC
:1041900028B9281D7880C5F5805080B201E0002044
:1041A0007880BDE8FE8F2DE9F04705462C480E4685
:1041B000040B82B017462946E0B204F06AFF81463C
:1041C000284800688047804600F032F88246BA00EE
:1041D0003146484604F058FF504600F021F801E00F
:1041E0002D1D361D3846471EC0B270B104236A46E5
:1041F000A9B2E0B204F02CFF04223146684604F074
:10420000A5FF0028ECD000F006F8404616490968E2
:104210008847BDE8F387114801214170017070475C
:1042200028B1124A1248126852680121104770479B
:1042300038B50F4C204604F0BBFF0546C0B250B164
:104240000A4A12685268002120469047204604F02E
:10425000AFFF0028FAD1E8B232BD0000F8460020D6
:1042600000E00100DC470020E0470020D8010010FA
:10427000004003400020D9E5E0B5ADF806000B464C
:104280000020ADF808008DF804000092DDE901017E
:104290000022FFF708FE0EBD82B01346ADF8020003
:1042A0000A460020ADF804008DF80000DDE90001A9
:1042B00002B010E6652807DA0003642190FBF1F0F4
:1042C000C0F5805080B2D2E504207047DFF800F0DE
:1042D0000158001080B502216846FFF7F7FFBDF8CE
:1042E000000002BD704770478149086070478149EE
:1042F00008707047032290FBF2F080B2FCF7D1BE49
:104300000178B02904BF417800290CD10179122924
:1043100003D1417C012906D101E01B2903D140884A
:104320000121FCF7DBBE704710B5734C607002F0E2
:1043300037FB401C207004216078FCF747FEBDE885
:104340001040FDF7BDBF38B50C46200411D56A48B2
:104350004078FCF7DCFB050008D02878A02804BFD3
:10436000284600F008F82846FCF764FB84F4004077
:1043700032BD002032BD30B587B0044601208DF833
:10438000000001A9204602F00BFE05002AD19DF88D
:1043900006105748C9070AD54368180005D0608839
:1043A0006A4601A9984705461CE006251AE00368FD
:1043B000180006D060886A4601A99847050001D117
:1043C00010E006259DF8050060B99DF806008DF8FF
:1043D00010008DF814500020ADF8120004A9608878
:1043E000FCF7A1FE9DF8000000281EBFA068002871
:1043F00000F0F7FB45B99DF80600122806BF9DF8AE
:10440000051001291B2803D060880121FCF766FEF6
:1044100007B030BD2DE9F0410446FF2C0D4616468D
:1044200098461FD02020FCF7F3FA070018D0B020E0
:1044300038707E707D8087F80480069929B1182233
:1044400007F10800FCF795FA04E0182207F10800CC
:10445000FCF7C1FA39462046FCF7FBFA002002E0DF
:10446000132000E00220BDE8F08110B54FF47A740B
:104470006243BDE8104004F0EABE10B504001EBF60
:104480002078FF28FE2803D004F0E9FEFF202070EA
:1044900010BD80B5009313460A46014615480078C2
:1044A000FFF7B8FF02BD30B583B004460D4602F0F9
:1044B00021FF50B901A80090ADF804507F230D48AA
:1044C000007800222146FFF7A5FF37BD00B583B075
:1044D0007E238DF804108DF8052001A9009100229B
:1044E000014604480078FFF795FF07BD0000000073
:1044F00044480020FF460020DD480020052923D045
:1045000006291BD0072918BF09291DD00B2918BF60
:104510000D2919D00E2913D00F291CBF11291229DA
:1045200012D0162918BF17290CD01B2918BF1D2916
:104530000AD0522918BFD22906D007E0C0687047B8
:104540000068704780687047406870470020704777
:1045500070B5052914461D4616D0062912D0092922
:1045600018BF112910D0122912D0162918BF1729E7
:104570000CD01B2918BF1D290AD0522918BFD229D7
:1045800006D007E0072606E0022604E0052602E042
:10459000032600E001264FF6FF72944203D102F099
:1045A000BEFE841B02E0D22908BF0C34301980B251
:1045B00000F0F2FA38B105B12C807142BDE87040CC
:1045C00009B200F033BB70BD80B5FFF797FF18B19B
:1045D000BDE8024000F005BB01BD0000DFF800F0BF
:1045E000E9940010DFF800F0A19400100A7802703E
:1045F0004A7842708A78C97802EB0121418070477D
:104600002DE9FC410D4616461F460A9A09990446B3
:1046100001AB00F0F0F9804608BB019908980870DA
:104620003346DFF858050178491CCAB2002A06BF94
:10463000012101220A460170294601980271009762
:1046400001980279204600F00DF8804620B90198C3
:104650001E2100F015FA02E0019800F0F5F940463D
:10466000BDE8F6812DE9F041044684B00E461746B8
:104670009846172000F090FA050026D00A9A1000FC
:1046800003D04146281D904700E00020010A2E700B
:10469000E9706F70A8700521001DADF80800ADF835
:1046A000001001956946DFF8D804007800282046FC
:1046B00002D000F059F801E000F00CF804462000A8
:1046C00004D0284600F08DFA00E01324204604B000
:1046D000BDE8F08110B50B88DFF8A8240C246343F3
:1046E0001A44303A536833B94B6853600989508192
:1046F0001181002010BD162010BD80B5052000F0EE
:104700000FF858B9062000F00BF838B9042000F073
:1047100007F818B9072000F003F800B1012002BD26
:104720000C2210B5DFF85C1442431144A1F13004AF
:1047300084B06168A9B1DFF8482412787AB1ADF885
:104740000000019169462089ADF80800608900F0F9
:104750000BF810B1606800F044FA0020606001209E
:1047600000E0002004B010BD70B50D460446288955
:10477000010004D0DFF810140988814201D21B2007
:1047800070BD6868042100F051FA0646288930702F
:104790002889000A70702888B0702888000AF07094
:1047A0002889051D4FF6FE70844213D10C20FCF7BA
:1047B0002FF901000CD0902008704C800220087165
:1047C000CD808E60DFF8C4030078FCF742F918E072
:1047D000132070BD3346AAB200212046FFF7FEFE2B
:1047E000010007D002280ED0072810D012280CD0C4
:1047F0001F280DD1DFF8880301780A001CBF491E6D
:104800000170002070BD142070BD022070BD042016
:1048100070BD38B50446002060600879022821D1B7
:10482000CA88042A1EDB886801784378C57801EBC2
:104830000321837889B203EB05230D1D95429BB2BA
:1048400010D1052B18BF042B03D0062B18BF072B44
:1048500008D1218123806FF0030100F0E7F9606047
:10486000002032BD012032BD0B88037002220B886C
:104870001B0A43700B88012B06D14A8882700422E0
:104880004988090AC1700CE0022B0AD14A8882705B
:104890004A88120AC2708A88027106228988090A27
:1048A000417110467047022A1BDB0A784B7802EBF5
:1048B000032202800288012A05D18A78C97802EB96
:1048C000012141800BE0022A09D18A78CB7802EBE2
:1048D000032242800A79497902EB0121818000207C
:1048E0007047012070470A8802700A88120A4270D5
:1048F0004A8882704A88120AC2708A8802718A883D
:10490000120A4271CA888271C988090AC1710820D5
:104910007047082A18D10A784B7802EB03220280EC
:1049200011F8022F4B7802EB0322428011F8022F7C
:104930004B7802EB0322828011F8022F497802EBB8
:104940000121C1800020704701207047022A00D158
:1049500001E0012070470A78497802EB01210180CB
:1049600000207047F8B504460D4616461020FCF7A7
:104970004FF8070016D0A02038707D800020787096
:104980002EB10C223146381DFBF7F3FF04E00C2258
:104990000021381DFCF71FF839462046FCF759F86E
:1049A0000020F2BD0120F2BD2DE9F04180460D4608
:1049B00016461F462020FCF72BF8040019D0A22031
:1049C000207066706580069820716771079929B11B
:1049D000182204F10800FBF7CCFF04E0182204F1D0
:1049E0000800FBF7F8FF21464046BDE8F041FCF720
:1049F00030B8BDE8F08170B51E0004460D4621D0E8
:104A0000012101F0A2FFD8B161480078002100E047
:104A1000491CC9B2814211DA5E4B1B6803EB0112DB
:104A20005388002BF4D10020107001F14000508019
:104A300022B1D48015723260002070BD152070BD87
:104A4000142070BD012070BD10B504461022002155
:104A5000FBF7C1FF23E0002200E0521C4C4909781B
:104A60008A420BDA4B49096801EB02114B88002B93
:104A7000F3D00B798342F0D108467047002070478D
:104A80004FF47A724A4300F1090301460FF219000C
:104A900004F0DDBB10B50446607A04F0E0FBFF20B3
:104AA000607210BD0000000010B504001CBF6088DB
:104AB000002807D01721204600F005F82046BDE861
:104AC0001040C1E710BD1CB50446207804280FD162
:104AD0000020019000900A46E188207A1323FFF716
:104AE00063FFE18802B0BDE81040122205202EE0ED
:104AF00013BD072170B50446002539BB18E02548D1
:104B00000068EDB200EB0516307800281CBF707A03
:104B1000FF280CD0F088A04209D13046FFF7BAFF39
:104B200014213046FFF7CFFF3046FFF78DFF6D1C95
:104B300017490978E8B28842E1D30425FF222146CB
:104B4000284600F004F86D1C082DF7DB70BD10B589
:104B50000C240C4B60431844A0F130046089884257
:104B60000AD1606840B1FF2A1CBF0178914203D18D
:104B700000F037F80020606010BD0000E048002021
:104B8000E64600208C480020FC460020E446002039
:104B9000E5460020E846002080B5001D80B2FFF702
:104BA00021FD28B1BDE804406FF0030100F03EB8DC
:104BB00002BD000070B500F035F8054604F10800AC
:104BC00080B201F071FF060005D02A48B480016868
:104BD000316006600836284909682846884730460B
:104BE00070BD38B500F01EF8224A05461068002155
:104BF00001E00146006878B100F108039C4221BF42
:104C00008388C3180833A342F3D3036800290CBF79
:104C100013600B6001F055FF2846BDE8344016498B
:104C200009680847044615480068004738B5044637
:104C30000D4600F00FF801000AD06842204401F14F
:104C40000803984221BF8B88C9180831814200D2DD
:104C5000204632BD0749096841B101F1080290427E
:104C600021BF8A888A1808328242F4D308467047E6
:104C700000000000E4470020E0470020DC4700205F
:104C800038B50225012918BF04291C4610D100F0AF
:104C900047FB05000CD10599049800F055FB204610
:104CA00000F05FFB00F03DF901F001FA04F05AFB5F
:104CB000284632BDDFF800F0A1980010DFF800F0C0
:104CC000BD980010DFF800F0D9980010DFF800F070
:104CD0006D98001070B5DFF8F065054630680C4639
:104CE00008B1112070BD00F0E7F801D1122070BDAD
:104CF000DFF8D805806800281CBF0078002801D1A3
:104D0000102070BD0C2001F0CFFE306040B30120B8
:104D100001F095F9306805700021306841700A2271
:104D20002146801CFBF725FE00F0C4F9040002D0E8
:104D300000F0A9FA15E0DFF898050078032810D1F3
:104D40001D2000F0E4FADFF88C15088048B1DFF888
:104D5000880500784EF66022042101F07BFF00E018
:104D60001324204670BDF8B50C46DFF8701509789D
:104D70001546052211421E4627D0012CDFF84C159E
:104D800002D18F680FB301E0CF68F7B1202D02DAAE
:104D90002A0002D00EB90220F2BD08701F220021A5
:104DA000781CFBF718FE2A463146781CFBF7E1FD1C
:104DB0003D70284624B1791CBDE8F440FFF77ABF66
:104DC000791CBDE8F440FFF779BF1220F2BD38B579
:104DD000DFF8F444216809B9122032BD0978814214
:104DE00001D0032032BDDFF8F0542878022101F011
:104DF0004BFFDFF8D814002048800421287801F008
:104E000043FFDFF8D0140020088003202168487099
:104E10000020BDE83240FFF755BFF8B5044600F06A
:104E20004BF801D11220F2BD1CB1207801F0D3F86B
:104E300008B90220F2BD6078801C202823DA20788F
:104E400000F0A3F908B11820F2BDDFF880546B68B8
:104E50000021002202E0B61C71181B685BB15E687D
:104E6000767828B9C9B27718BF1C202FF3DB012050
:104E7000B61CB218F1E7D0B238B16078D2B280185F
:104E8000801C202801DB0B20F2BD082001F00CFE65
:104E900006000FD0082200F07CF8686830B100E00E
:104EA000084601680029FBD1066000E06E6074606E
:104EB0000020F2BD1320F2BDDFF8200400780521A8
:104EC0000842704710B500F01CF801D1002010BD59
:104ED000DFF8F8335968002201E00A46096869B131
:104EE0004C6824788442F8D14C680868002A14BFC2
:104EF00010605860084601F0E4FD00E00024204600
:104F000010BDDFF8D8130978052211427047DFF889
:104F1000CC0300780521084218BF00F043B91220E5
:104F2000704770B5DFF8A443A06818B101F0C9FD5F
:104F30000020A060E06818B101F0C3FD0020E0602F
:104F40000521DFF89853287808421CD004F110009E
:104F500001F0FEFB287800260521084211D000F060
:104F600077F9A06060B100F013F800F071F9E0602B
:104F700010B100F00DF804E0A06801F0A2FDA660F9
:104F80001326304670BD002001F0E2FB002070BD0A
:104F900020220021FBF71FBD2DE9F0478288DFF8B2
:104FA0002863DFF82853316842F20607D31B4FF01D
:104FB000010805D09B1E012B60D99B1E0FD00BE072
:104FC0008068007841B1020003D101204870FFF7EA
:104FD00079FE01006BD038E04FF0000867E0806890
:104FE00007780029F8D04878BD4C012833D100F06B
:104FF00058F9DFF8E492B0B1012000F088F9824658
:10500000BAF1420F0AD399F800004EF6602202214D
:1050100001F020FEAAF13C00688010E04FF47A70A5
:1050200000FB0AFA02E000F072F98246BAF1000FC2
:1050300005D099F800005246022101F0F3FD3168D5
:1050400002204870207818B9384600F004F92EE0A4
:10505000002020702BE0207848BB0320FBF7D8FC11
:1050600048B1D02101704770042181700146306839
:105070000078FBF7EEFC00F006F918E0806807788E
:10508000287842F208018A420CBF01260026FF2838
:105090000DD00420FBF7BCFC010008D0D020087024
:1050A0004F7002208870CE702878FBF7D2FC404603
:1050B000BDE8F087F0B5844F386885B070B3847868
:1050C00001F05CFA28B10A2000F021F905460B2016
:1050D0000DE000F0E6F828B1062000F018F90546CA
:1050E000072004E0082000F012F90546092000F02E
:1050F0000EF906467648007800F01BFA3968CA7A3D
:10510000039203468A7A029228460A1D0192224699
:10511000C97800913146FFF7D9FD00E0012005B0C4
:10512000F0BD38B5014668486B4D02682878674C79
:1051300001291ED161880B0002D0694B1B7823B175
:1051400012B31078BDE8324041E63C29A8BFA1F176
:105150003C000CDA022101F097FD60884FF47A716F
:1051600001FB00F22878022101F05CFD0020608044
:1051700031BD4AB159490978490705D5022101F0E5
:1051800083FD002060807CE031BD5049496800E02B
:10519000096829B14A6812788242F9D108467047F5
:1051A00000207047F8B54D480078002405210842DA
:1051B00001D11220F2BD454DA86810B900F048F8A1
:1051C000A860E86810B900F043F8E860A868002813
:1051D0001CBFE968002901D11320F2BDFFF7D8FEFA
:1051E000E868FFF7D5FE6E6812E09B1C501859184E
:1051F000401C117071684978491C01707168097808
:105200004170801C71684A784968FBF7B2FB3668C8
:10521000AA6896B13CB97068117843785F18BF1CD2
:10522000202FE2DB01247368E9685B780A789B1C15
:1052300088189A18401C0A70DCE71078511CFFF798
:1052400039FDE868411C0078FFF738FD0020F2BD09
:10525000202001F029BC38B51B4D0446286878B1E0
:105260000320FBF7D5FB48B1D02101704470032126
:105270008170014628680078FBF7EBFB04B100E081
:1052800031BDBDE8314010B50F4C206840B101F090
:1052900018FC002020600120BDE8104000F0D4BEC2
:1052A00010BD80B50948806858B10278431C694632
:1052B000012000F09AFE20B10078C00701D501203E
:1052C00002BD002002BD000018480020DC4500207F
:1052D0007E45002080450020F84500207D450020C7
:1052E0007F450020DFF800F049980010DFF800F05B
:1052F000C9560010282808DA4FF6FF72914204D0F0
:10530000CA4A22F81010002070470220704728284F
:1053100003DAC64931F8100070474FF6FF70704746
:1053200070B504460D46C24E1C2200213046FBF7E4
:1053300052FB34777577FAF7B7FD01000EBF0121F4
:1053400000211220317070BD10B5B94CE160A06031
:1053500010220021FBF70BFE012801D1A0680CE010
:1053600010BD10B5B24C606010220021FBF7FFFDAC
:10537000012801D1606800E010BDBDE81040102197
:1053800004F0B3BBAA48406870472DE9FC41A84D22
:105390000446002695F81E80042C0F4624DA28784F
:1053A000032818BF102054D101F0E8F828B900F004
:1053B0000BFE10B900F00AFE08B1122049E0012CE2
:1053C00018BF022C1DD1BFB1062200216846FBF791
:1053D00002FB00F040F838B90622FF216846FBF7CF
:1053E000FAFA00F038F808B1022032E00622394615
:1053F0006846FBF7BEFA0BE00621684604F075FB31
:1054000006E0032C04D16868694604F067FA064692
:10541000884FAC770421387801F036FC00202884CE
:105420009EB9ACB1684600F05BF8064668B9032C3B
:105430000ED11D20FFF76BFF288448B138784EF657
:105440006022042101F006FC02E00EB185F81E8006
:105450003046BDE8F681062269463846FBF7ADBA0C
:1054600070B5044600252000714E05D121B10622F9
:1054700006F11000FBF77DFA307801280CD10125E8
:10548000200004D102203070FDF7FAFC04E0002077
:105490003070204600F0A8F8284670BD38B50024CA
:1054A000E0B10578624A290006D14178837801EBA2
:1054B0000321D182C0781076107802280ED1012401
:1054C000280006D103201070117ED08AFBF711FE50
:1054D00001E000201070284600F086F8204632BD1A
:1054E00010B5534CA17F81B10146062204F124007E
:1054F000FBF73FFAA07F04F1240100F008F804F163
:105500002400BDE81040FFF7EDBE002010BD79B1CA
:1055100002000DD04A79012808BF42F0C00006D031
:1055200002F03F0203284A7102D142F04000487164
:105530007047010018BF01210846704770B53C4D07
:105540000446287FFF2815D00A20FBF761FA0600E1
:1055500010D0D020307074700820B0700622A87F60
:10556000F07005F12401301DFBF703FA287F314666
:10557000FBF76FFAE87F01280FD12F48006818B1B8
:105580008068010018BF8047BDE870402948007856
:105590004EF66022042101F05DBB70BD2448806896
:1055A00070472348C068006870472148C1680A688E
:1055B000521C0A60007FFF281CBF4FF48041FBF79C
:1055C0001EBB70471A48807F704738B50446184D97
:1055D00005F11000FFF78AFE05F110001CB9A97F44
:1055E00009B105F1240032BD70B5114D0446287F84
:1055F000FF2819D00E20FBF70BFA060014D0D0209C
:10560000307074700020B070062205F11001F01C9B
:10561000FBF7AFF9E88A70813146287E3073287F26
:10562000BDE87040FBF715BA70BD00008C45002046
:1056300060450020F8450020FC450020DFF800F020
:10564000259500102DE9F041044688461227404672
:105650004FF6FE7188421646DFF84C5908D1A8690A
:1056600050B30268100027D041462046904720E002
:105670004FF6FF71884212D1A86938B10268100054
:1056800004D0414620469047070005D031462046C9
:1056900000F0BDFA07000FD12C706E700CE001F025
:1056A00026F948B10078A04205D131464046FFF7BF
:1056B000C5FF074600E003273846BDE8F08110B576
:1056C000044684B000F072F808B9022029E020886E
:1056D000012101F03AF908B9142022E0208801F0F4
:1056E00045F9042812D1DFF8C00881894FF6FF720E
:1056F000914218BF112014D1218881816188818055
:10570000A188C180E1880181218941810020029026
:10571000019020890090E388A28861882088FDF7A5
:1057200005FC04B010BD30B5044685B0208840218A
:1057300001F00BF9002836D02088ADF8040000F005
:1057400035F8002500281CBFA07A002807D10021C9
:10575000684600F0B1F9A07AF0B102251CE0912072
:105760008DF800008DF803503E208DF801000121D6
:1057700006208DF80200A088ADF808006088ADF81A
:105780000600E088ADF80A002089ADF80C008DF81D
:105790000350684600F090F920880022402101F073
:1057A00072F8284600E0122005B030BD2389E28857
:1057B000A1886088FDF7E4BA70B50C46DFF8EC17F5
:1057C0000978022918BF0129154601D1122070BDA0
:1057D0000DB9022070BD01F08AF8060001D1142035
:1057E00070BD1CB1307940F00200307110222946A2
:1057F00006F11800FBF7BDF82869B062002070BD03
:10580000F8B506000C4601D10220F2BD308801F047
:105810006EF8050001D11420F2BDDFF89007007882
:10582000022818BF012803D0A87C082802D10CB197
:105830001220F2BDDFF87077786908B11120F2BD4F
:10584000B02001F031F9786108B91320F2BDB0221F
:1058500000F0A5FA786931884180A022311D001D31
:10586000FBF787F8796902200870A87C796932888B
:1058700008280CBF012000200B1DDFF83417097821
:1058800004F040FB06461CB12146284604F00FFDFB
:10589000300018BF00F038FA3046F2BD38B5044683
:1058A0000D4601F024F808B9142032BD8DF80050DF
:1058B0006946204604F02EFC32BD38B50022A0B166
:1058C00001230624E4B2051915F8015C303D0A2DC8
:1058D0000BD203FB05220A256B43641EE5B2002DA3
:1058E000F0D11046BDE8344001E0022032BD30B5B1
:1058F00005460C4685B0204600F0F9FF08B9122095
:1059000019E0DFF8B006854228BF022013D210222A
:1059100000216846FBF75FF8280A8DF801008DF832
:105920000050280C8DF802002146280E8DF8030047
:10593000684604F02EFB05B030BDF8B50546DFF82B
:105940006C060078022818BF01280C461F4601D1BA
:105950001220F2BD0FB90220F2BD284600F0C7FFA9
:10596000060001D11420F2BDF06A08B101F0A9F8D7
:105970001C213846FBF713F80100F16201D1132016
:10598000F2BDB07C08280AD1069840B1887E00900C
:1059900001F112030A8A284604F0B4FC00E000205A
:1059A000317941F004010CB141F002013171F2BDD5
:1059B0002DE9F0410D4600F09AFF04001FD0A562CA
:1059C00000F0EAF90546C0B200B92578A66A94F855
:1059D00005801020FBF71CF8070010D0D02038708D
:1059E000062200207870A11D0920B87087F8038076
:1059F000381DFAF7BEFFFE603946E8B201E0BDE8A7
:105A0000F081BDE8F041FBF724B8F0B50C0087B099
:105A100050D0A079DFF89065002830690CBF0825C8
:105A2000042508B9DFF890050778042D08D1DFF8C0
:105A30008C05006820B1416808001CBF0020884721
:105A4000207D059004F10803608A04903946208A7D
:105A50000390E08902900195A0880090E279E078B7
:105A600000F071F8E07880B9172004900122E089F5
:105A7000039002950020019004F108000090E37962
:105A8000A188384600F0B2FEE070306908B100F03D
:105A900056F9307801000DD0717800F0B8F848B1AF
:105AA000E378312B04D0A2883178184600F079F8D9
:105AB0000020307007B0F0BD10B5044684B0A08857
:105AC00051B1002102910191A1890091638922893C
:105AD000E188FDF7ECF91FBD04B0BDE810403B21A3
:105AE000FDF7E7B970B504460026A08800F0FFFE78
:105AF00018B10678A08800F0ACFEDFF8AC54287826
:105B0000010007D0864205D1697800F080F848B1DD
:105B100000202870300005D0A379A288A0783146F3
:105B200000F03FF8686908B100F0EEF8A08800F0D6
:105B30001DFF042802BFA088A989884204BF4FF630
:105B4000FF70A88170BD2DE9F041064688461746D2
:105B50001C461620FAF75CFF050020D0D0202870E4
:105B60006E700520A870EF702CB106222146281D0A
:105B7000FAF7FFFE04E006220021281DFAF72BFFAA
:105B8000069868812946079828730898E88109983B
:105B900028820A9868820B982875404631E7BDE84C
:105BA000F081F8B504460D4616461F460820FAF760
:105BB0002FFF48B1D021017044700621817086808A
:105BC000877101462846EDE0F1BD2DE9F04105461B
:105BD0000E46174698460C20FAF71AFF040014D018
:105BE000304600F084FE08B9DFF8CC030078D021FD
:105BF000217065700721A170E570A680E780A4F888
:105C00000880069961812146FBE6BDE8F08110B568
:105C10000C4600F081FE28B140882146BDE81040C6
:105C2000FFF70CBD122010BD2DE9F84F074689463D
:105C300092461C46484600F05AFE5FEA000B1EBF23
:105C4000DFF86453696900295CD051F8A42F18204B
:105C500002B134208A6802B1143004B11C304968A2
:105C600001B1173080B2FAF7D3FE06004AD01822ED
:105C700000F095F800F090F85FEA000808BF9BF884
:105C80000080D020307077700A20B070A6F80490A1
:105C900086F806A006F118076969D1F8A40040B19A
:105CA000B7603846D1F8A41000F11C071C22FAF79F
:105CB00060FE6969D1F8AC0040B1F7603846D1F8B0
:105CC000AC1000F114071422FAF753FE3CB137610F
:105CD000384600F11C071C222146FAF74AFE686983
:105CE000D0F8A81031B177611722D0F8A810384643
:105CF000FAF73FFE31465FFA88F0FAF7AAFEBDE8F0
:105D0000F14F01E0BDE8F18F10B5A74C6069A8B173
:105D1000D0F8A40008B100F0D4FE6069D0F8A80063
:105D200008B100F0CEFE6069D0F8AC0008B100F018
:105D3000C8FE606900F0C5FE0020606110BD10B5AE
:105D4000994C206940B100F0BCFE00202061042085
:105D5000BDE8104000F078B910BDF8B504460D4616
:105D6000284600F0C4FD060015D000F015F8070025
:105D700008BF37780620FAF74BFE06000BD0062244
:105D800000F00DF8D020307074700E20B070B58027
:105D90003146F8B206E0F1BD2620FFF7B8BA00217F
:105DA000FAF719BEBDE8F440FAF753BE2DE9F843FF
:105DB00005460E4617469846304600F098FD5FEAC5
:105DC00000091ED01020FAF723FE040019D010227B
:105DD000FFF7E5FFFFF7E0FF08B999F80000D021D1
:105DE000217065700F21A170A680277284F8098048
:105DF000C0B20899A1720999E1720A99E16021463D
:105E000031E0BDE8F1832DE9F84304468846914628
:105E100000F06DFD070024D01420FAF7F9FD05000D
:105E20001FD0FFF7B9FF060008BF3E78D0202870CA
:105E3000062200206870B91D0B20A870E81CFAF734
:105E400098FD6C8118F00101C5F8109018BF012170
:105E50002973F0B218F0020118BF012169732946B5
:105E600001E0BDE8F183BDE8F443FAF7F2BD2DE9A6
:105E7000F14F90460D469946404600F038FD070028
:105E80000A9EDDF82CA0DDF830B00D9C3ED09DF8C8
:105E9000000000283AD1387940F010005FEA4971DB
:105EA0004CBF40F0020000F0FD00002E08BFBAF128
:105EB000000F08D1BBF1000F08BF002C03D100F088
:105EC000FB00387122E040F0040038713CB12069D9
:105ED000B8621022214607F11800FAF74AFD3EB1D8
:105EE00035B9F86A08B100F0ECFD1C2130460AE033
:105EF000BAF1000F0AD0012D08D1F86A08B100F0FC
:105F0000E0FD1C215046FAF74AFDF862264D68690B
:105F1000002842D086B1D0F8A40028B91C2000F097
:105F2000C3FD6969C1F8A4006869D0F8A40018B17C
:105F30001C223146FAF71DFDBBF1000F11D0686934
:105F4000D0F8A80028B9172000F0AEFD6969C1F8A3
:105F5000A8006869D0F8A80018B117225946FAF7C6
:105F600008FD8CB16869D0F8AC0028B9142000F0A5
:105F70009BFD6969C1F8AC006869D0F8AC0018B144
:105F800014222146FAF7F5FC9DF8000053464A46D4
:105F9000414601B0BDE8F04F46E6BDE8F18F084943
:105FA0000860704700000000444500207D45002047
:105FB000F845002040420F007C450020FC450020B1
:105FC0000C48002003F0A6BC264800E026480068E4
:105FD00000B101207047010001D0172801DBFF2824
:105FE00001D101207047002070472DE9F04D0D468A
:105FF00093460024BBF1200F80461F462C7003DB24
:106000000020BDE8F08D0419E0B25845F8D2E4B2A2
:106010003E5D641C002EF3D0E4B231198B45EFDBFA
:1060200017F804A05046FFF7D6FF641C0028E7D0FD
:10603000701EC2452870E6D1E4B23819E1E70B4979
:106040000A7810430870704708490A7832EA00005D
:10605000087006D10648006818B14068010018BFF2
:10606000004770471848002014480020DC480020F2
:106070001048002038B504460D4600F038FCA0B1A9
:10608000807C042801D0122032BD3748006808B156
:1060900090F899502946684603F053FD334B6A4601
:1060A0000221204604F0C5FC32BD142032BD80B56B
:1060B0002F480078400707D52E48FFF770FF2E497C
:1060C0004FF6FF70088001BDBDE802400020FFF7D9
:1060D00066BF7CB5012403280D4610D042F213019F
:1060E000884204D04FF6FF7188421ED02AE0A8787B
:1060F0000C2818BF112826D100F027F823E0E878F3
:10610000A9881D4E1A2804BF33889942F4D06A89A1
:1061100000922B89EA88FFF758FDA88831888842C9
:1061200011D14FF6FF7030800DE0687900241228FD
:1061300009D1ADF80040297968886A46FAF78CFFE2
:10614000012400E00024204676BD38B50A4C2088A2
:106150004FF6FF75A84205D008490A780849FAF7B2
:1061600082FF258031BD000058450020FBA90100B9
:106170007D4500200446002050450020F8450020C1
:1061800048450020F8B5144600250E46BC4FBD4BCF
:1061900040B1012815D0042818D006281ED00728A1
:1061A00022D02CE0162928DA1622002107F10C0053
:1061B000FAF711FC3246214607F10C00FAF7D9FB39
:1061C0001EE0022E19D12088388119E0082E14D142
:1061D00038462146082202F07DFF11E0012E0CD145
:1061E000DA6903F1280104E0012E06D1DA6B03F12C
:1061F0004801207800F030F802E0182500E0022580
:106200002846F2BD10B50B4600249D4920B1012857
:1062100008D0042809D00DE015220C311846FAF7F1
:10622000A8FB08E00889188005E01846082202F05B
:1062300051FF00E00224204610BD01460020C9079E
:1062400006D50FF248238F4810220721FBF7A8B884
:1062500070478D490860704710B50B7884074CBFB4
:1062600043F0020303F0FD0304064CBF43F0800338
:1062700003F07F0304074CBF43F0080303F0F70368
:1062800084064CBF43F0200303F0DF030B70AA2108
:10629000084203D0107840F00C0003E018B91078E1
:1062A00000F0F300107010BD2DE9F0410F461546C7
:1062B000387802281E464FF000085ED178680178D1
:1062C0004078069C01EB002080B221001CBFB0F595
:1062D000285F0B2056D14FF42851401A08D0401E99
:1062E0001AD0401E28D0401E1ED0401E2AD044E0A6
:1062F000F868FAF73CFB079A80B2031B9342B8BFD9
:10630000021B92B21019162803DA3280F8680119BC
:106310000EE04FF00D0834E0F8680088022131806B
:106320002870000A68702CE0062030800622F96888
:106330002846FAF71EFB24E001203080F868007838
:1063400028701EE0F868B0B10821318001882970FA
:106350000188090A69704188A9704188090AE970B1
:10636000818829718188090A6971C188A971C088E9
:10637000000AE87105E0308003E0A6F800804FF0E5
:1063800001084046BDE8F0812DE9FC4B0E468046F1
:1063900030780027022891461D466BD1706801783D
:1063A00040780A9CDFF8E0B001EB002080B24FF4A7
:1063B0002851401A06D0401E29D0401E4CD0401E05
:1063C00038D057E0F068FAF7D2FA80B2A04204D38E
:1063D0002919162903DB0D274DE007274BE0F36849
:1063E0002A4649461819FAF7C4FA2C19F068A4B2DB
:1063F000C4F1160200212044FAF7EDFADBF80000A0
:10640000002838D00268100035D0002121E07CBB84
:10641000022DE0D199F8000099F8011000EB01205D
:10642000F1680880DBF8000028B30268100022D071
:1064300001210EE0E4B9062DCDD1F06806224946CF
:10644000FAF797FADBF80000A8B10268100012D042
:106450000321404690470EE054B9012DBBD199F875
:106460000000010013BF0128F1680870802702E0D6
:106470000B2700E001273846BDE8F68B000000003E
:10648000204600204446002050480020A962010018
:106490008963010000000000B1494870704710B5E1
:1064A000AF4C207004F021FB2078BDE8104005219E
:1064B000FAF78CBD7CB5AA4D28780C46210419D575
:1064C000FAF725FB060084F4004411D000F058F8D8
:1064D00058B93078A22806BFA24800786878FF280B
:1064E00003D03146FAF7B5FA02E03046FAF7A2FADD
:1064F000204676BDE10709D5A86820B141680800AB
:106500001CBF0020884784F0010076BDA10709D593
:10651000686820B1416808001CBF0120884784F0EA
:10652000020076BD610727D58F4E31880A001DD045
:10653000481E308080B2E0B9FFF746FD48B18B4974
:1065400001200870686820B1416808001CBF012064
:106550008847FEF717FF694603F0C0F96846FEF763
:10656000BFFF1D20FEF7D3FE308002E0042100F0C3
:106570008BFB84F0040076BD002076BD00F0FCB9F2
:1065800038B502780124912A4FF6FF7102D0A22A71
:1065900076D07BE04278052A49D00E2A04D00F2A13
:1065A00048D03E2A69D071E082886D4941F20905E0
:1065B000531B2DD040F6F9755B1B2FD0DB1E31D05D
:1065C0005B1E08D09B1E022B05D9DB1E012B15D9A3
:1065D000DB1E08D05AE04968002958D009680A0033
:1065E00055D0884750E06249096800294FD04B6870
:1065F00019004CD0014642F20E003CE089680029A7
:1066000045D00B68190042D00146104698473BE040
:106610008068411C0078FEF723FF35E08068FEF7B4
:106620003DFF31E080680078FEF788FF2FE0FFF73C
:1066300059FA2CE0828842F20D05531B13D09B1FA0
:1066400002D09B1F0FD021E04A4B1B888B420AD0FF
:1066500049490968D9B10A68110018D0014642F2C7
:106660001300904710E04249096881B14B68190056
:106670000DD001461046984706E000F00AF803E006
:106680000246408800F04BF8044600E00024204613
:1066900032BD70B505460124A8780128014611D005
:1066A000022806D0032811D0062815D00A2809D0C0
:1066B00032E02B48806880B3416808002DD028461E
:1066C00088472AE02946FFF7A0F926E0A8882A464D
:1066D00000F025F8044620E00E20FAF799F90600AC
:1066E0001BD0A8880122402100F0CDF8D0203070C6
:1066F0003146E87870701120B070A888B080E888C2
:10670000F0802889308168897081A889B081154816
:106710000078FAF79EF900E00024204670BD70B5BD
:106720000C46154600F022F90126042804D112482F
:10673000006858B1026803E00D48006830B1426853
:10674000100003D02946204690470646304670BDCB
:10675000034948607047094908607047000000001D
:10676000F84500207C450020804500207F45002022
:106770005C450020504500200C48002010480020B7
:1067800038B5AE4C00220021204601F0F1FB207804
:106790003025684300F088F96060B8B100210AE054
:1067A00005FB01F202444FF6FF735380491C00239E
:1067B0001371D362C9B222789142F1DB002000212B
:1067C00004EB8002401C0C289160F9DB31BD0021F4
:1067D0009A4A02EB8102936813B9906000207047D7
:1067E000491CC9B20C29F3DB132070472DE9F04195
:1067F00006460C4617469846204600F078F808B141
:10680000112024E04FF6FF7000F071F805001DD054
:1068100085F8058006220699A81DFAF7AAF806222F
:10682000002105F10C00FAF7D6F86C802F712E705C
:106830000020E86200210898A8740998A8820A98A4
:10684000E882204600F0E9F8002000E01520BDE8CD
:10685000F08110B500F04BF8040012D060880121DF
:1068600000F0DBF8E06A08B100F02BF930220021DB
:106870002046FAF7B0F84FF6FF70608000202071D4
:1068800010BD022010BD38B50C46154600F02FF89B
:1068900058B10179002D14BF2143A1430171022198
:1068A000408800F0BAF8002032BD152032BD38B55E
:1068B0000C4600F01CF8050017D02879207006223D
:1068C00068796070A91DA01CFAF753F8062205F13B
:1068D0000C0104F10800FAF74CF8A87CA073A88A10
:1068E0002082E88A6082002032BD012032BD10B5CE
:1068F0000022524B00E0521C1C78D1B2A14209D2B6
:106900005968D2B23024544321444C888442F2D195
:10691000084610BD002010BDF0B5484B5C68002251
:106920004FF6FF7700E0521C19788A420BDA3021CB
:1069300001FB02F561194E88BE42F4D0655D8542C7
:10694000F1D10846F0BD0020F0BD10B50C464FF661
:10695000FE71884206D0FFF7CAFF00281CBF0079ED
:10696000204201D0012010BD002010BD80B5FFF7EE
:10697000BEFF00B1807C02BD10B5002000212F4A6F
:1069800008E05368C9B230244C4323441B7903B157
:10699000401C491C1478CBB2A342F2D3C0B210BD44
:1069A00026480078704710B50C46FFF7A0FF002876
:1069B0001CBFC18AA14202D0C482002010BD0120A8
:1069C00010BD80B5FFF793FF00B1C08A02BD70B55E
:1069D00005460C461646FFF78AFF28B94FF6FE70AB
:1069E000854218D0142070BD0179C06A28B9CA0642
:1069F00009D5C90609D40F2070BD01F01202102A72
:106A0000F7D1002EF5D0052070BD20B1807EA042C8
:106A100001D20C2070BD002070BD70B504460D463B
:106A20000026064800EB86008268100002D0294646
:106A300020469047761C0C2EF3DB70BD5448002096
:106A400002000A4A08BF0FF22100506051707047DF
:106A50007047064A010004BF5178012902D011781D
:106A60005268104770470000704700009C440020A7
:106A700000F10103810704D010F8011B89B18107DF
:106A8000FAD10268B2F10131914311F0803F04BFA5
:106A900050F8042FF6E710F8011B11B110F8011B94
:106AA000FBE7C01A70470000E0B50821ADF8001000
:106AB0000190042100F00FF808B100200EBD0298EB
:106AC0000EBD00B583B00821ADF80010019005217E
:106AD00000F001F807BDADF80210684601490968E9
:106AE00008470000D847002062F30F2262F31F42DC
:106AF000401810F0030308D0C91A1FD3DB0748BFA2
:106B000000F8012D28BF20F8022D130030B41446E0
:106B10001546103928BF20E93C00FAD8490728BF9C
:106B200020E90C0048BF40F8042D890028BF20F858
:106B3000022D48BF00F8012D30BC7047C91818BF9E
:106B400000F8012DCB0728BF00F8012D7047000089
:106B500000B583B00820ADF8000012209C490968F8
:106B6000ADF802006846884701980EBD10B5994CF3
:106B70000020A060FFF7ECFF606010BD70B5044618
:106B80000D46164600F018F808B1466070BD10209A
:106B9000FFF78AFF78B184720581466000210160A9
:106BA000C1608C490A6812B9086070BD0A46116854
:106BB0000029FBD1106070BD864A12682AB1138982
:106BC0008B4204BF937A8342F7D11046704708B1D5
:106BD0000021018170472DE9F041FFF7B9FF7D4E9B
:106BE0007D4977680C68C51BB4F57A7F14D0A4FB87
:106BF00005014FF47A72002303F08EFF4FF47A7888
:106C0000A8FB0023054608FB01331046194622461F
:106C1000002303F081FFC01970602846BDE8F041F1
:106C200003F0F2BFF8B504466A4800680D46164600
:106C300008B9FFF7D0FF69480068804700F01FF8E7
:106C400000F048F80446384688470CB10020F2BDF1
:106C50000820F2BDF8B50446604800680D461646A7
:106C6000804700F00CF804005D4918BFE660096831
:106C7000384688470CB10020F2BD0820F2BD074617
:106C800032462946204679E770B500F026F80646D8
:106C900029462046FFF790FF040018BFFFF797FF33
:106CA00000F018F8304688470CB1002070BD06206F
:106CB00070BDF8B500F011F8074629462046FFF7E9
:106CC0007BFF002600B1466800F004F8384688478C
:106CD0003046F2BD42490968704704463F480068A3
:106CE0000D4600472DE9F147DFF8F080394DD8F81F
:106CF0000000DFF8ECA081B080470246A868019947
:106D00000818A8601046DAF8001088472E68002E90
:106D10004DD00027D8F8000080478146BDF8060016
:106D20000024002804BF9DF80500002807D1307911
:106D30009DF80420904202D3801A307106E07068FA
:106D4000019981423ABF401A70607460B08858B9A6
:106D5000F08858B9F06868B1318908000AD0B07A73
:106D6000F9F74DFFF0687060B08808B9F08808B195
:106D7000308930B93068002F0CBF28603860344645
:106D800000E037463668DAF800104846884764B1B4
:106D9000A088002804BFE088002803D12189A07AB8
:106DA000F9F72DFF2046FFF78CFE002EB2D1BDE88B
:106DB000F3870848016841B10A484A680968824275
:106DC00098BF10460029F8D1704700207047000096
:106DD000D8470020FC470020B4440020DC470020B6
:106DE000E04700208EC2F52800B583B00821ADF839
:106DF00000108DF804001721ADF8021068461D49F7
:106E0000096888479DF805000EBD1B480021818058
:106E10000121017070472DE9F0410D4617490978AD
:106E200001248842064602D2134F387808B901205F
:106E30001DE01348006880478046B88804FA06F6CB
:106E40004DB920EA0601B98060B159B90020FFF7B9
:106E5000CBFF044606E010B90120FFF7C5FFB88854
:106E60003043B88040460749096888472046BDE856
:106E7000F0810000D8470020F447002018FE0000F1
:106E8000DC470020E047002030B585B014460822DA
:106E90000291ADF8002000223A490968ADF80400DB
:106EA000ADF802201D46684688479DF80C102170F9
:106EB0000499296005B030BD1CB51420FFF7F4FD1E
:106EC0003149086014220021F9F785FD002000F007
:106ED0000BFE012003F0D2FD022002F071F9032025
:106EE00003F0C2FE0420FFF7DAFA052004F012F8DE
:106EF0000620FDF719FA0720FAF70CFA0820FCF72C
:106F000028FE0920F9F74CF801AB6A460021102051
:106F1000FFF7BAFF9DF800100920F9F768FD00247B
:106F20009DF800102046F9F76AFD641C092CF7DB78
:106F300013BD10B582B004F061F8144B144A154922
:106F40005020FFF7A1FF60B10520FFF782FD082068
:106F5000ADF800000C200B490968ADF80200684646
:106F600088470D48006880470446FDF783F9F9F724
:106F7000AEFE0A49096820468847F9F7DEFE002080
:106F800016BD0000D8470020F0470020B044002084
:106F9000DB480020F70D0100DC470020E04700201F
:106FA000F8B505460C46AF892FB3AA6816783006A7
:106FB0000FD50D2F1FDB0C3FBFB2D01900903B4601
:106FC0006888012102F02EFE002814BF0220012053
:106FD00000E000202070B00900F00100607006F0B1
:106FE0003F00A070781EA08080B208B1A868401C45
:106FF000A0600020F2BD0120F2BD0A7802704A882C
:1070000042704A88120A8270097985E0022B00D109
:1070100063E00420704700BF0A8802700988090AEB
:10702000417002207047042B00D17DE0042070479E
:107030008A7802708878098801280CBF0420122001
:107040004843401C80B2704770B51E46062E144659
:1070500019DB049D2078617800EB01202880022252
:10706000A078E17800EB01206880211D02202871C2
:10707000681DF9F77EFCB01F288180B200B1A01D09
:10708000E860002070BD042070BD08888004000CFA
:10709000704710B5029C062B104612D102212171B7
:1070A0004278017801EB02212180C278817801EBDE
:1070B00002216180011D2279601DF9F75AFC002030
:1070C00010BD142B08BF1021E9D0042010BD4DE0E5
:1070D000022B00D101E0042070471078517800EBBA
:1070E000012000990880002070470888704710B57B
:1070F000022B0FDB029C207261721078517800EB3A
:1071000001202080981E608080B200B1901C6060D9
:10711000002010BD042010BDC17004207047042B56
:1071200000D101E00420704700981178537801EBFA
:10713000032101809178D27801EB02214180002067
:1071400070470888704703EBD3704008B3EB4000EA
:1071500007D15908022904DB0098818002600020D1
:107160007047042070470888704700BF4A88098824
:107170000270514389B2481C80B2704710B5042B8D
:107180000EDB00F031F8D478917801EB04214180D6
:10719000191F818089B201B1111D8160002010BDCD
:1071A000042010BD00BF0A8802700A88120A4270CB
:1071B0004A8882704A88120AC2708888001D80B28C
:1071C0007047012B04D10099107808700020704797
:1071D0000420704700BF0A8802700A88120A4270B1
:1071E0004888801C80B2704702981178547801EB6F
:1071F0000421018070472DE9F04784B080460C9D42
:107200000C4691469A4655B91720FDF7C5FC012654
:10721000050005D11324204604B0BDE8F087002600
:107220002846012700F8019B14B15146A047471C8E
:107230005FEA09600DD510214046FFF786FBD8B9FB
:10724000BFB2EA193946284602F09FFC044668B9E5
:107250000C370420ADF800000195ADF808706946C0
:107260004046F9F7C8FE00280446D4D0002ED2D0FC
:107270002846FDF7B6FCCEE71924F7E730B502291A
:1072800018BF102985B00446154603D1022B18BF3C
:10729000102B01D0002017E00A469A4203D129465C
:1072A000F9F78BFB10E01029694606D1284600F05B
:1072B0000DF810226946204604E000F007F810227D
:1072C00069462846F9F779FB05B030BD38B50400AA
:1072D0000D4618BF002D0BD010220FF26401284676
:1072E000F9F747FB2078287360786873012032BD76
:1072F000002032BD38B504464FF6FE7084420D467C
:107300000BD0172D09DBF9F7FAFE2946884204D382
:107310002046BDE83440FFF746BB012032BD80B5B2
:107320004FF6FE71884205D0FFF74BFB010005D1F7
:10733000172002BDBDE80140F9F7E1BE02BD000023
:10734000FB349B5F80000080001000000000000004
:1073500038B54FF6FF74A0420DD10020164A1378BD
:1073600098420EDA21F8204001EB80050023401CF2
:10737000AB70C0B2F3E700F00BF810B1048000214D
:10738000817031BD80B500F003F800B1807802BD96
:1073900010B5002200E0521C074C2478D3B2A3425F
:1073A00007D2D2B231F822308342F4D101EB82000D
:1073B00010BD002010BD000054480020DFF800F090
:1073C0001DB50010DFF800F03DAC0010DFF800F054
:1073D00089D10010DFF800F0C9B40010DFF800F028
:1073E00019570010DFF800F061840010DFF800F09A
:1073F0008D670010DFF800F0BD800010DFF800F0AE
:107400002D8A0010DFF800F071940010DFF800F012
:10741000A9AC0010DFF800F0E5730010DFF800F011
:1074200035A30010DFF800F0E1AC0010DFF800F049
:10743000EDAB001080B54FF49E720FF23001DFF813
:10744000E00C01F057FEDFF8080D00210170012269
:10745000DFF8001D0A7302220A70DFF8FC1CC0F876
:107460000D10DFF8081EC0F82D1001BD9904002191
:107470001905002179040021F0B5174C402161184D
:10748000C878022805D009480021016008498847CA
:10749000F0BD256E074E35606007284320662768DB
:1074A00024600E48804727603560F0BD2C110440F1
:1074B000A56500002840044010B5074CA17D0029B7
:1074C00005D10121A175480204493E398847206849
:1074D000002800D0804710BD540200218B390000E5
:1074E00010B50549054A72B6C878012802DC0120AA
:1074F0004870121D62B61047940200216D470000CB
:10750000F8B51A4E0546316B1948CC09E401002D37
:1075100011D01849097802290FD0007B044372B6B4
:107520000120154F4002B847114820380088C10992
:10753000C90704D016E0C07AF0E7407BEEE70F49B8
:107540003463CC61400AC0070CD001208003F16A8B
:10755000002D01D0014300E081430846F162074954
:10756000403948630020B84762B6F8BD8002002168
:107570008800002196020021DF3C000040400440CA
:107580000749002800D00420064A72B60978C907C6
:1075900001D0105800E0802062B640B27047000071
:1075A0006B020021586004402DE9F0410FF24C00BD
:1075B000DFF8581D2722036844688568C668076994
:1075C000D0F814C0D0F818E0D0F81C800B604C60E4
:1075D0008D60CE600F61C1F814C0C1F818E0C1F829
:1075E0001C8020302031521EE5D14268836800683B
:1075F00008604A608B60BDE8F081000054610000C3
:107600007F140200060005000F0008004800520029
:1076100080FF3F00000000000000000000000000AC
:1076200000000000304000400140034007400F4090
:107630004F40CF40CF41CF43CF47CF4FCF3FCF2F4A
:10764000CF1FCF0F000000000000000000000F005F
:10765000080000003F00000040003F000000040060
:1076600068000E00DC00060043001A000500000060
:107670000000020000000000000000000400C00044
:1076800000000400C000000007000000000000002F
:1076900000000000000000000000000050C0009149
:1076A000007070C00091007082312100319110B1E2
:1076B0000070018101B100A18231329110B10191BC
:1076C0001110418141226340F106007051C00191C7
:1076D00030181039833108D01831416F31003191A1
:1076E00010B1831414166F680070251050C00091FB
:1076F000F4C340C12014036F311041045082F022C2
:107700008440512622C082312100319110B1633969
:107710003110410482C082312100319110B16339AE
:107720003110A2C082312100319110B150101531B9
:10773000051405920070536452C031103106613156
:10774000C102566412C13110213971065131E10272
:107750005664007051C0019101CCE2C0566453647C
:1077600011C1C2C0566454B0007154A064B0F0801E
:107770000022B54011C122C1566451C00191E2C03E
:10778000823160820200329110B100C3C868536434
:107790004012B09032B000C3CE6840C2D0688012B0
:1077A000B09032B00070536401C122C1566401C16F
:1077B000C2C0566453829D64C012B09032B0007053
:1077C000536472C281C0566422C111C1566402C0A2
:1077D00011C1566462C031C3566462C311C156649C
:1077E00002C311C15664538253399D64E2C35B6482
:1077F0001122F84042C281C8566452C211C1566477
:1078000072C2E1CE566402C281C8566402C201C887
:107810005664B0C00C690070536442C201C856641B
:1078200052C211C0566472C2E1C0566402C001C1A6
:10783000566462C001C3566422C101C1566462C36A
:1078400001C1566402C301C1566453829D64007035
:1078500002C1623101C0A080001E3241101A3461A1
:107860002010101A136F236E11161216346900704F
:10787000E092D08200223B45C0B2007000000000C0
:1078800000000000000000000000000000000000F8
:1078900000000000000000000000000000000000E8
:1078A00000000000067305720B720E7250B000717A
:1078B000818060B050A09280F0EFF19202933A651F
:1078C000412278458080F1C1100430160111011465
:1078D000016C8B618C618D618E618F6190619161B2
:1078E0009361956197619961706273629180F2C052
:1078F000210421318280422A1214321601112114EE
:10790000016CA661C761AC617362A661C761AC61BD
:1079100073629B619B619B619B619B619B61AC649A
:107920009B61D5649B61E2649B610E659B612A65E6
:107930009B618280E0DFF2923A65B0B0A261B1B0A3
:107940000673057230B05861D0CF3A6584C203C067
:10795000C0C36864907850916078103161781014D9
:1079600000925078403161781000403171781000F9
:107970001092B078609281782192307840314178CD
:107980001000309210C0F0919B6154A0F080502202
:10799000CF45408000226646C76100C8609159818A
:1079A00050B0918041222E46C0CF3A65128282317A
:1079B00082394239281077641282F11212042F1092
:1079C0001F312F1440C120140D6F6D39DE10F4C328
:1079D0004E0482C082312E006D39A2C082312D004A
:1079E0001A828A392082803180390BC00B18AC781A
:1079F00030824039021011C0013010C00118021845
:107A000082312100C126919103B013B063B053B00D
:107A100003823914418001226646B481C491D58124
:107A20009518B51C1C4EC51C544A6591F080102257
:107A30000C422C623D9110B13E9110B165910F92B4
:107A40005981F914AB18BC10F0805022C7411022A4
:107A50002C460C62B0CF3A6563B030820010F2C0A1
:107A60002004021011C0013010C001180218823128
:107A70002100C1269191919113B003B063B053B02E
:107A800064B054B0007141800122664663B064B0B6
:107A9000F0805022C741B181C191D181911861918B
:107AA00031B04462128282318239423928107764BF
:107AB00059810582591420820BC00B18AC7880C004
:107AC000007163B0626A0C62018262818231823D20
:107AD000A0EFF19202933A6503A09B61A2807764C4
:107AE0009B6150B000719B612DE9F04FDFF8D44AE3
:107AF000DFF8D45A207007210020E86183B0DFF856
:107B0000980B01700D21418040F222218180DFF825
:107B10008C0BDFF89C1B29628A7E0270FF2ACB7EC9
:107B2000437008BFFF2B0E7F86704F7FC77091F8A0
:107B30001EC080F804C0C97F417116D1FF2E08BF56
:107B4000FF2F12D1BCF1FF0F08BFFF290DD1DFF8C5
:107B5000641B0A7802704A7842708A788270CA7808
:107B6000C2700A79027149794171DFF84C1B0278C1
:107B7000DFF8488BDFF8487BDFF8483BDFF8486BDD
:107B80000A7042784A7082788A70C278CA70027924
:107B90000A714079DFF8342B4871FF21DFF8AC0B14
:107BA000017041708170C1700171417101202871B3
:107BB000101D017141718171C17101724172002109
:107BC00001708172A0218181032181730721C1731A
:107BD0000021017428214182012101750021817554
:107BE00002F15A0100224A7001220A7042750020F7
:107BF000DFF85C1B0880D8F82C104878A87008784B
:107C00003870801C8A782A708A681279521E1A701D
:107C1000CA786A70CA682A618969DFF8382BA96155
:107C20004FF4967111801821484380B2FEF73CFF53
:107C3000B060002855D03878010055D04FF49071CD
:107C4000484380B2FEF730FFDFF80C9BC9F8040010
:107C500008B9B06843E0387838214843FEF724FF7C
:107C6000686120B900F070F8D9F8040037E038787E
:107C7000DFF8E8AA0001FEF717FFCAF8000028B9EC
:107C800000F062F800F05CF8686928E03878DFF806
:107C9000D0BA0001FEF708FFCBF8000048B900F0A9
:107CA00053F800F04DF86869FEF70BFFDAF80000B2
:107CB00015E0387830214843FEF7F6FEDFF8A01BC8
:107CC000086088B900F040F800F03AF86869FEF7FB
:107CD000F8FEDAF80000FEF7F4FEDBF80000FEF72D
:107CE000F0FE4FF4804126E000F0BBFA0746082082
:107CF000ADF800001E20ADF802004FF40050DFF890
:107D0000641B096801906846884703F0B1F9D8F808
:107D10000C00697800880843DFF84C1B088038465F
:107D2000DFF8481B096888470C21DFF8300DFFF7A2
:107D300045FB4FF400512078F8F761FFBDE8F78F5D
:107D4000D9F80400FEF7BDBEB068FEF7BABE70B544
:107D50000C46E00788B00DD5FFF734FB38B10021A1
:107D60008160DFF80C0B0068010018BF804784F0C9
:107D7000010072E0A00707D500F071F83C2000F088
:107D8000E2FF84F0020068E06007DFF83C5827D586
:107D9000DFF8C409817840684FF490724A43024486
:107DA0006869382359430144901D12F82C3F06930B
:107DB00053891B090593838B0493D288520803923D
:107DC00000220292019201F12C020092012291F80C
:107DD00028300178002000F0B6FF84F004003CE079
:107DE000200607D500F03BF83B2000F0ACFF84F004
:107DF000800032E0A00508D5DFF8A00C016841F052
:107E00000041016084F4007027E0600504D5FCF7B0
:107E100069FA84F4806020E0600405D5812001F0D7
:107E2000CDF884F4804018E0A00415D54FF0FF3061
:107E3000E86103F0C4FC2E69366805F1340305F1EE
:107E4000480205F1240105F16000B047E86000F048
:107E500012F884F4005000E0002008B070BD00204B
:107E600006900590049003900290019000900023EA
:107E7000012200217047F8B5DFF84C47DFF8D858E9
:107E80002369E068DFF83868183300221B684FF078
:107E9000FF319847DFF82408DFF8641BC06A806868
:107EA00040790870002703F0AEFCDFF8580BFFF7AD
:107EB0008DFAFFF78FFAFFF791FADFF8780B0021C0
:107EC0000170017141718171C171017241720022B1
:107ED000DFF8F80700F10E010A70A0224A8007229D
:107EE0004A7103220A7100220A738A7200F8592F1C
:107EF0000122CA720021427081700BE068684FF461
:107F00009071794308444179012908BF03F03AFA96
:107F10007F1CFFB230788742F0DBFFF763FAA0786E
:107F2000DFF8641B087003F063FE03F098F9DFF8D4
:107F30005C1B00200870DFF8581B08700120DFF878
:107F4000541B08700020DFF8501B08700120DFF878
:107F5000501B08700020DFF84C1B0870DFF8481B2E
:107F60000870DFF8481B0880DFF8441B0870F2BD7A
:107F70002DE9F0411446DFF8485708B12A7802701D
:107F8000DFF8D48711B198F801000870002C3ED0BA
:107F9000002600271CE0C9B2DBB2605402F12800C1
:107FA0000179E154591C427900F034F8827900F0EB
:107FB00031F8C27900F02EF8027A00F02BF8427AFC
:107FC00000F028F80078C9B24E1C60547F1CFFB244
:107FD000287887421BDA3846FFF708FA0028F5D1DF
:107FE000D8F804004FF490717943F6B20844DFF8F2
:107FF000C41A4969A7553822006800787A430A44B0
:10800000711C4B1C80280CBF00200120C3E70020FE
:10801000BDE8F081C9B26254491C704738B50C0004
:10802000054601D1122032BDFFF7E0F9010017D15A
:1080300000F0DFFC01680978402901D00C2032BD36
:1080400000214B42625C0344491C102983F8E22062
:10805000F7DB012180F8E410052103F01EFA00206F
:1080600032BD10B50446FFF7C1F9010016D100F08A
:1080700036F801680978402901D00C2010BD00F1C4
:10808000F0010A78012A03D106220A77022102E0D0
:1080900006224A700D2103F000FA002010BD10B531
:1080A0000446FFF7A3F901000CD100F018F890F88E
:1080B000F810022907D1817900F1F902002000F0BF
:1080C0009DFD002010BD01680978802903D1082199
:1080D000FFF790F9F5E74029F3D1112010BDDFF843
:1080E000D80940684FF4907161430844704710B557
:1080F000040001D1122010BDDFF85C06407808B101
:108100000C2010BD03F0ABF8DFF8B00922784178FD
:10811000114041706278817811408170002010BD5B
:108120000404002138B50C00054606D0DFF88C1594
:10813000C96A89680979884201D3122032BD03F0E7
:1081400099FBDFF8BC08057001202070002032BDCB
:10815000A30300216C03002111040021DFF85C253A
:10816000D26A92681279904201D312207047DFF8E8
:10817000541508700020704710B5140019D011B1C3
:10818000012908D015E003F09AFB10F1800F207050
:108190000DD1302010BDDFF82405C06A8068016869
:1081A000007900EB4000084410F8030C2070002018
:1081B00010BD122010BD2DE9F8430C000546904675
:1081C000994605D05FEA090018BFB9F1010F01D047
:1081D000122044E0DFF8F0733878404504D28A205A
:1081E00000F0ECFE30203AE02846FFF7FFF80100EF
:1081F00035D1DFF86405DFF8906840684FF490717E
:1082000069434518307820B90120FFF7F7F80720B7
:1082100025E000F026F83178491E3170DFF84C1661
:1082200009688847B8F11C0FBCBF38781C280ADBE6
:1082300042462146284603F0A4F901000FD120460A
:10824000FCF7CFFC07E0102000904B464246214649
:10825000284603F0EEFB284603F05BFA0020BDE859
:10826000F283DFF85C080068004700005104002139
:1082700030B5DFF83C08017883B009B121203EBD5C
:10828000DFF84018DFF840480B7B496003F0E0035B
:1082900043F085030B7341F60A024B7B0A8003F01F
:1082A000F00343F002034B73002266238B734A8072
:1082B0008023CB7340F6C412DFF810388A600B615C
:1082C0004C615A6001251A7A1D8002F0FE021A7272
:1082D0002525DA7A9D7002F0F002002542F00102B5
:1082E000DD705D72DD60DA7225800D220270B64CA1
:1082F000DFF8DC27E068DFF8DC37CDE90025256909
:10830000083502222D68A84741E0000000C0002186
:1083100030B5282983B003DA050018BF012D01D03C
:1083200012203EBDDFF88847207808B121203EBDED
:10833000480000F6621081B2012003F0E2FBDFF892
:108340009817DFF89037496040F608000880002051
:1083500048808860012D087B00F06000087300F001
:1083600056F80CBF03200A2088730022DFF86C0740
:108370004861002008828861CDE90022C87C00F0B5
:1083800041F8C87402220B2000F048F8A847208169
:1083900000203EBD30B5282883B001DB12203EBD51
:1083A000DFF80C47217809B121203EBD400000F6DE
:1083B000621081B2002003F0A4FBDFF82417DFF87D
:1083C0001437496040F607000880002200204880EA
:1083D0008860CDE90022087B00F06000087302226B
:1083E00000F015F802208873DFF8F006086100201D
:1083F0004861C87B00F006F8C8730C2000F00EF846
:10840000A847C4E700F0F00040F001007047487B47
:1084100000F0F00040F00200487370472070DFF871
:1084200094462569E06808352D68704780B5DFF807
:10843000800600780B281CBF0C280D2801D02120B5
:1084400002BD40F2014003F04CFBFFF714FD002099
:1084500002BD2DE9F04F0D462828B8BF262D83B068
:10846000804616460FDA310018BF012E0DD0022EBD
:1084700018BF032E09D0042E18BF052E05D0062ED6
:1084800018BF072E01D0122099E0DFF8249699F842
:10849000001009B1212092E0DFF82846DFF82C76A1
:1084A000DFF824A641F60A01218040000021618006
:1084B0006460A1606630217B01F06001217340F6A9
:1084C000C41B617B01F0F00141F002016173A073F4
:1084D00029468020E0732761C4F814A0002038806A
:1084E000BD701846012818BF0228FE701BD100225B
:1084F00003F0DDFAB0F5BC7FD8BFC7F804B02EDDBD
:10850000B0F57A7FD8BF41F2883027DDB0F5CB6F68
:10851000D8BF41F64C5021DD40F6490188421EDAB1
:1085200042F210701AE003280CBF082002204143D9
:10853000C9001B2202FB001000F5BC7080B2F930AC
:1085400040F2712190FBF1F140F27122796002FB5F
:10855000110000B1012040180BFB00F07860387A60
:1085600000F0FE003872002100207872F860F87A7E
:10857000FFF748FFF8720020AAF80000DFF8640552
:108580008180C18080F800808021457086700172F2
:108590004C48DFF86C140078DFF818650870092083
:1085A00089F8000003F02FF900F07AF83569F068D7
:1085B000083502222D682146A84730810020BDE8F9
:1085C000FE8F0000844C00202843002030B528286E
:1085D00083B001DB12203EBDDFF8D4140B780BB161
:1085E00021203EBDDFF8DC4441F609032380420030
:1085F00000236380A3606632237BA27303F06003D1
:1086000023738022637BE27303F0F00343F00203E1
:1086100063736460DFF8D024DFF8D03422616361D3
:10862000002515600F25157101255571DFF8AC5433
:108630009560552515735573957300251561D57B88
:1086400005F0F00545F00105D57300221A805A8027
:108650009A8080229A7100229A60DFF85854DFF8DD
:108660008424107000205070FF20907000209080B3
:10867000D080802010720A20087003F0C4F800F047
:108680000FF8022221462C69E86808342468A047C4
:10869000288100203EBD00008C4C00206C4C002046
:1086A000DFF84C04DFF82C340021CDE900017047DD
:1086B000B63F0050E81200507C4C002058FE0000ED
:1086C000BC4C0020854C0020F44E0020EC490020DA
:1086D00070B5DFF8DC432078092818BF0A2801D0DC
:1086E000212070BD00F045F92078DFF8F813092843
:1086F0000CD1DFF8D40300888880C148007803F0EB
:10870000B9F800210020FEF77DFE1BE00A2819D1F0
:10871000DFF8D823538810889688CB801D187519E8
:108720008D809279802A18BF812A0FBF7F22DFF8BF
:10873000C43393F90030D21A0A720121FEF762FEA7
:1087400003F061F80020207070BD0000744C002020
:10875000984C0020964C0020B04C00200C4F00207C
:108760001C4F00202DE9FC4B834617461C46DFF8C2
:1087700044930A9A0B9B00203D0089F804000CD01A
:10878000012F05D0032F18BF022F0AD0042F35D197
:10879000A3B3150018BF012A30D1032F18BF022F31
:1087A00009D143F66175ABF1A000A8423CBFA1F12D
:1087B000A000A84222D23D0018BF042F09D143F6E1
:1087C000E175ABF12000A8423CBFA1F12000A84216
:1087D00014D2594512D3002C18BF012C0ED10D9D77
:1087E000280018BF012D03D0022D18BF032D05D17D
:1087F000DDF83080072118EA010F01D112202DE0A9
:10880000BD4EB07B012808BF0C2027D0012F18BF18
:10881000042F06D1874800F8042B06221946F8F7E2
:10882000A8F808F00700F074B77435751CB93471F6
:108830000622B24904E0012C06D134710622B04967
:1088400006F10800F8F795F8012F08BF4FF0000B6C
:10885000A6F810B0012089F804000020BDE8F68BCE
:10886000104F0020D8470020944C0020E047002003
:10887000C44C0020F8B58E4C2178092918BF0A296C
:1088800052D00B291CBF0C290D294DD089490979DB
:10889000002908BF01286AD00028974D42D001283E
:1088A00065D1A87B01283FD0A87C01001CBF01280E
:1088B00004280ED1FEF7AAFDFD21084234D19148CB
:1088C0000078010053D07C494978814201D10920C8
:1088D000F2BD012003F0A5F9286000260120A8734D
:1088E000FEF798FD1821884871434718387B40F0FF
:1088F00080003873A87C012807D026B903F04DFA10
:1089000000F5C87000E00020B860761C032EE9DB9B
:10891000207828B9A97C7D48405C2070FEF77EFD58
:108920000020F2BDA87B08B92120F2BDFFF799FC19
:108930000646FEF777FD012804D0FEF743FD2968BF
:10894000884203D100F015F8012700E0002700203D
:10895000A8732846FEF76AFD207800281CBF002F68
:10896000FEF75CFD6A49096830468847D8E712205F
:10897000F2BD40F2024003F0B4B8017841F08F013B
:108980000170C17841F02001C170817841F030015F
:1089900081700020704710B147494978017000206C
:1089A000704738B50546424800780C280C4606D179
:1089B0004049C86809694031096888470DE00A28BC
:1089C00002D14A48807908E02846FEF70FFD0100F1
:1089D0000ED100F00EF890F87400C0B2802818BFD5
:1089E00081280FBF7F2043490978401A207000205A
:1089F00032BD314840684FF4907169430844704774
:108A0000B94C00208C4A002070B506460C4615462D
:108A1000FEF7ECFC01000BD1274840684FF4907141
:108A2000714308444FF48E7108440470458000205F
:108A300070BD00009C4C002002000CD01D4A9278B2
:108A4000824208D3002918BF012904D1124A1170AB
:108A50001049FFF78EBB122070470000E84E00203F
:108A60002C4B10B1012803D00CE019800020704776
:108A7000188810701888000A50706E2090701920A5
:108A8000D070F3E7122070478B4C0020864C0020FA
:108A9000BA4C0020874C0020884C0020040009407C
:108AA000BB4C0020894C00208A4C0020BE4C00208A
:108AB000B84C002028430020B04C0020D04E0020AD
:108AC000DC470020284E0020204F0020A84E002028
:108AD000010000803DD90100784D002029417671C8
:108AE000404E0020DC4E0020844E0020C44E00206A
:108AF00002000080C04C0020EC4900206C4C00209B
:108B0000744C0020BC4C0020244C0020C0D9001024
:108B1000E0470020984C0020DFF800F0818C001026
:108B2000DFF8F004902101708821417001218170EB
:108B30000221C170002101718021417100218171E8
:108B40002021C1710021DFF8D0048160C1601F21A4
:108B5000017000214170418041601F20DFF8BC148A
:108B6000087070472DE9F04100F076F81F463ED5B9
:108B7000DFF8A4040078400739D5DFF8A48498F81A
:108B8000000098B10C20F7F743FF80B391210170EA
:108B900084803E214170C5800321817006810021BF
:108BA000C1704781014698F800001FE01520F7F7D3
:108BB0002FFFE0B101210170042200F0BEF80A701D
:108BC0004C713E224A70CD710A228A704E72032285
:108BD000CA70CF7200220A71220A8A712A0A0A72A6
:108BE000320A8A723A0A0A7300F003F8E2E1BDE839
:108BF000F0810146DFF82C0400787047F8B500F0EA
:108C00002BF828D5DFF810040078000723D51720AB
:108C1000F7F7FEFE07001ED001203870082200F092
:108C200085F90C207968887004207968C8707868A4
:108C3000047178684571280A7968887131467868C6
:108C4000C01DF7F796FE3946BDE8F440DFF8D403BF
:108C50000078F7F7FEBEF1BD0446DFF8B803C0792F
:108C600080060D4616467047F8B5DFF8BC63074628
:108C700030780C46154620B3B8000C3080B2F7F7B8
:108C8000C7FE00284CD090210170877013214170DD
:108C900000F10C01416000EB47010C3181600021C3
:108CA0000AE0436834F8112023F81120836835F86E
:108CB000112023F81120491CB942F2DB014630781B
:108CC0002AE0B800461C06F10B00C0B2F7F7A0FE80
:108CD00030B30121017000F030F8042142681170B6
:108CE00013214268517041688E704168CF70002135
:108CF0000EE000F01CF8137100F019F81B0A537114
:108D000000F00FF8937100F00CF81B0AD371491CA6
:108D1000B942EEDBFFF76DFFBDE8F440F7F799BE0F
:108D2000F1BD426835F8113002EB810270474268AC
:108D300034F8113002EB81027047FF21417000F1DD
:108D40000801416070472DE9F54FB248C0798006AF
:108D500081B08846994605D5AF4E31787078C907FD
:108D600002D4810740F1DB80AD4909780F9C109D4A
:108D7000DDF844A0DDF848B0002950D02220F7F7F4
:108D800047FE070058D0912038703E2078709DF83B
:108D9000040038B9F87006220C9907F10800F7F7BB
:108DA000E8FD07E03120F8700622002107F10800F5
:108DB000F7F711FE707880071AD50A20B8700D9861
:108DC00030B10146062207F11500F7F7D2FD01E0A8
:108DD00000F0BEF80E9830B10146062207F11B00E4
:108DE000F7F7C7FD01E000F0ADF887F8079008E05D
:108DF0000120B87000F0ACF800F0A4F809F0010010
:108E0000F871A7F8048039469DF80800B871FC8114
:108E10003D82A7F812A087F814B0814879E0800756
:108E20004CBF1F2013208DF800009DF800000B3070
:108E3000C0B2F7F7EDFD070071D00120387000F0E7
:108E400075F879689DF800008870717878688907EE
:108E50004CBF0A210121C17079689DF80400087196
:108E6000786880F805804FEA1820796888717968F9
:108E70009DF80800C8717178786889074EBF80F83E
:108E8000089009F00101017278680C9921B106225D
:108E90000930F7F76EFD03E006220930F7F79BFD76
:108EA00071780F20890718D578680D9921B10622AD
:108EB0000F30F7F75EFD03E006220F30F7F78BFD6A
:108EC00078680E9921B106221530F7F752FD03E0BC
:108ED00006221530F7F77FFD1B2079680C54401CE3
:108EE0007A68C0B2210A00F01CF80D54401C7A6860
:108EF000C0B2290A00F015F801F800A0401C7A68F9
:108F0000C0B24FEA1A2100F00CF801F800B039465F
:108F10004448007803B0BDE8F04FF7F79ABDBDE8CC
:108F2000F78F1154401C7968C0B27047FF207870E9
:108F300007F1080078600420796808703E2079689D
:108F4000487070470622002107F11B00F7F743BD68
:108F50000622002107F11500F7F73DBD2DE9F0418C
:108F60002F4F044638780D469046C8B12F480078F8
:108F7000B0B905F10C0080B2F7F74AFD060017D032
:108F8000912030702A46FF207070B570B48006F1D1
:108F90000C00B0604146F7F7ECFC3878314609E048
:108FA00043462A462146BDE8F041FF20FFF7B4BD05
:108FB000BDE8F081BDE8F041F7F74BBD38B5044698
:108FC00014484078000623D5154D287870B117480D
:108FD000007858B90320F7F71BFDC8B19121017043
:108FE0008470102141700146287810E00C20F7F7BA
:108FF0000FFD01000CD000F01BF810204A685070E3
:1090000001204A6890704868C470FFF7F3FD1AE0C9
:1090100031BD0000004F0020BC480020084F002058
:10902000E3480020E1480020E4480020284F0020C9
:1090300001200870FF20487001F1080048600420FA
:109040004A6810707047BDE83440F7F702BD000071
:1090500070B514461D4600F01CF806460848006826
:10906000804703E016F8011B04F8011B29464D1E3A
:1090700089B20029F6D1BDE8704002490968084765
:10908000DC470020E04700200B460146184600F070
:1090900010B81D2290FBF2F21D2303FB120001F514
:1090A000E83101EB0030704780B50849096849692B
:1090B00005E080B5054B1B689B69984700E0884731
:1090C000034A0021116002BD00000000A801001049
:1090D0008404604262B38B0708D0521E11F8013B32
:1090E00000F8013B00F024808B07F6D1830740F0A5
:1090F000208000BF103A07D330B4B1E83810103ADE
:10910000A0E83810F9D230BC530724BFB1E80810EA
:10911000A0E8081044BF51F8043B40F8043BD207D4
:1091200024BF31F8022B20F8022B44BF0B780370C8
:109130007047083A07D3B1E80810083A40F8043BF2
:1091400040F804CBF7D25307E4E700000300002007
:1091500013F0030F09D0521E22BF13F8010B11F8B0
:1091600001CBB0EB0C00F3D07047121F22BF53F8B5
:10917000040B51F804CB6045F7D0121D0AD200BA97
:109180009CFA8CFCB0EB0C0038BF6FF0000088BF7D
:1091900001207047521E22BF13F8010B11F801CBBA
:1091A000B0EB0C00F6D0521C08BF10467047000010
:1091B000006801074CBF042000F003007047000066
:1091C0005F4B1988FF2905D1188078220021181DCE
:1091D000F7F701BC70472DE9F04104460D4628041D
:1091E00048BF85F4004030D428002DD05548006891
:1091F000804780462F46002025FA00F1C9071AD57E
:109200004F490A88121BC2EB0212821801EBC201FD
:109210000F1D012101FA00F6396808001CBF7868AB
:109220008847B1B22046FDF744FD08B93860786040
:1092300086EA050702E0401C0F28DDDB4249096889
:1092400040468847B8B200E00020BDE8F08110B584
:1092500082B00024FFE7009400F02AF816BDF8B5AC
:1092600004463848384E006880470F2C05461ADA05
:10927000334800EBC4077968A9B10F2194FBF1F2E0
:10928000C2EB021300880121E31A9940801889B2C9
:10929000C0B2FDF7F9FC00207860B860284631685C
:1092A00088470020F2BD3168284688470220F2BD79
:1092B0002DE9F44F80462348234C006889461E461A
:1092C000804783465FEA080004D1216858468847F2
:1092D000022031E00025DFF868A00AEBC5077868B6
:1092E00018BB9DF82800009A01280CBF174B184B9B
:1092F0000F2095FBF0F0C0EB001E4FF0010CA5EB2A
:109300000E010CFA01F1BAF800C0604489B2C0B293
:10931000984750B9C7F80480C7F8089006B135706F
:10932000216858468847002006E06D1C0F2DD4DBCD
:109330002168584688470820BDE8F28F00000000E9
:10934000C8440020DC470020E0470020556C0100A5
:10935000256C0100DFF800F0C59B0010DFF800F07D
:10936000E19B001080B5DFF85C05007840074CBF3A
:10937000DFF85405002000F04BFE002002BDF0B5E0
:1093800089B004460D461646102200216846F7F7BC
:1093900022FBDFF83875386850B3C188A14204BF9A
:1093A0000178002924D1417806290DD100F1480225
:1093B00000F1280104AB083000F077FBC0B901F0E0
:1093C00023F9024604A924E0806D88B1028A11299C
:1093D00027D1964209D100F033F8012805D101F0D8
:1093E00013F902463868816D13E0322001F0F4F879
:1093F0002046FDF77CFA07001CBFF86A002819D048
:10940000018A8E4216D100F01BF8012812D1F96AA8
:109410008A7E6846F7F7ADFA69462046FFF79AFF5D
:109420000BE09642E4D100F00BF80128E0D1386857
:10943000816DEDE72046FFF791FF012009B0F0BDF7
:1094400000F1120108222846F7F7B7BAF0B5DFF8A5
:109450007C640746306885B01546002488B9012928
:109460000ED1281D00F056FBE9680291297A01917E
:1094700000906B782A7879880020FCF797FC002010
:10948000DBE0C2887B889A4218BF0820F8D10278B6
:10949000012A08BF0720F3D0491E092960D8DFE858
:1094A00001F0055F142CC849617F92B2284600F094
:1094B0006DFF30B9DFF8180400780421F7F79FFB3F
:1094C000BAE0182831D10324B6E0102229463830FA
:1094D000F7F74FFA30684178042908BF03215ED0BE
:1094E00000F1180200F12801083000F091FE00F0B0
:1094F0002CFF00B10824052062E0102229464830E4
:10950000F7F737FA306800F148016A46083000F092
:109510007FFE306800F1380110226846F7F74DFAF7
:10952000012805D100F01DFF002874D1062047E076
:10953000042481E041780C2912D1C06D20B91C208F
:10954000FDF7B2FA3168C8653068C06D40B100F00F
:1095500076F801F059F83168C96D88760D202FE052
:10956000072469E0C36D002BFAD040780D28F7D1AD
:10957000288818820822A91C03F11200F7F7F9F9CC
:109580003068816ED1F89810C1F34022002A1FBFC5
:10959000C26ED268C2F34022002A27D00E2130E0EA
:1095A00041780E29DCD1006E20B91720FDF77CFA36
:1095B000316808663068006E08B100F040F80F208E
:1095C0003168487038E041780F29C9D1006E062211
:1095D000691C1130F7F7CDF931682878096E40F031
:1095E000020008743068816ED1F89810C1F38021B0
:1095F00000291FBFC16EC968C1F38021002916D0A0
:109600001021417018E0406E38B91420FDF74CFA73
:109610003168486608B908240EE03068406E30B101
:1096200000F00DF83168496E4FF0FF3008610020FE
:1096300000E0287800F0D0FF204605B0F0BD1022F1
:109640002946F7F796B910B500F069FE002842D117
:109650009E4C2068816E91F89510C90709D5C16E9E
:10966000097901F00301012903D1C17841F0010119
:10967000C17020680179022904D0032918BF042988
:109680000AD10121C0880022FCF7BDFB00F024F8BC
:1096900004202168487010BD012918BF05291AD17E
:1096A0000221417020680179012905D11022002191
:1096B0000830F7F790F907E0816E1022891C083016
:1096C000F7F757F900F008F810212068BDE81040BE
:1096D000283000F00ABA10BD2068C17841F00401BA
:1096E000C17070472DE9F041784C2068017800295D
:1096F00040F0E5804778D0F86880C66E062F2FD1FD
:10970000D8F89810CA0704D5327BD20748BF07277C
:1097100031D4C1F34002002A1EBFF268C2F34002F6
:10972000002A08D00927FBF72DFE01462068C088D3
:1097300000F013FF10E0C1F3800100291EBFF168A3
:10974000C1F3800100290BD00B27FBF727FF01464F
:109750002068C08800F018FF072F50D1082090E043
:10976000F91F0429F8D8DFE801F0062F05380400B6
:10977000F2E7EAE7D7E7806D20B91C20FDF794F9FE
:10978000216888652068856D002DE5D000F03CFFDC
:10979000A876102200212846F7F71DF9A97E0800B7
:1097A00004D01129BCBF284600F09FF9F7F71DF936
:1097B0002882082105F1120000F097F92068C0887E
:1097C000294600F0B3FEC7E7816DD1B101F1120265
:1097D000098AC08800F0ADFE13E0FBF7F3FE012715
:1097E0000546012D0CBF002700253846FBF7EDFE8E
:1097F00002462068C088294600F0B4FE14E0082F15
:109800000CD1D8F89800C0F3400000281EBFF068C3
:10981000C0F34000002807D0092032E0092F08BF1C
:109820000A202ED00A2F0BD1D8F89800C0F3800060
:1098300000281FBFF068C0F3800000280B2020D153
:10984000D8F89800C0F3002100291FBFF168C1F3C8
:10985000002100290C2014D1C0F3402100291FBF92
:10986000F168C1F3402100290E200AD1C0F3802005
:1098700000281EBFF068C0F38020002814BF10200D
:1098800012202168487020684178072918BF0829EC
:1098900004D009291CBF0A290B2910D1C088FDF763
:1098A00026F800281ABF818A01EB51024FF4FA72A0
:1098B000BDE8F041064800780221FDF7B3B9BDE8E4
:1098C000F08100007D450020D4460020CC480020D7
:1098D000E7480020DFF800F0D557001038B5040045
:1098E0000D4618BF002D01D1022032BD032168466C
:1098F00000F0FBF800F030F82A466946204600F0F8
:1099000050F8040004D103226946E81CF7F731F847
:10991000204632BD30B504000D4618BF002D83B07F
:1099200001D102203EBD0322E91C6846F7F721F869
:1099300000F012F801AA6946204600F032F8010052
:1099400009D10322294601A8F7F737F8012801D1E8
:1099500000203EBD01203EBD9DF8021001F03F01F8
:1099600041F040018DF80210704780B52020FBF7D0
:10997000CEFC38B1024607480078BDE80840012116
:10998000FDF750B901BD034800780121FDF77CB90E
:1099900000000000E7480020102221466846F6F744
:1099A000F2BF70B58CB000F00FF8FFF7F5FF03229F
:1099B00029460DF11D00F6F7E6FF00F00DF804460C
:1099C00003220DF12D0185E004460D461646302296
:1099D00000216846F6F7FFBF6846D0E0F0B595B0C5
:1099E00005460C4616461F463022002108A8F6F709
:1099F000F2FF1022294608A8F6F7C5FF1022002121
:109A00006846F6F7E8FF07223146FFF7C7FF07224F
:109A100039460DF10700F6F7B6FF1C9901B1012197
:109A20008DF80E101A9901B101218DF80F10102236
:109A3000002104A8F6F7CFFF1B99062205A8F6F728
:109A4000A2FF1D9906220DF11A00F6F79CFF1022C5
:109A500021460CA8F6F797FF69460CA800F01AF803
:109A600008A800F08CF80446102210A90CA8F6F7FC
:109A700080FF04A90CA800F00DF808A800F07FF8FA
:109A800005461E98102210A9F6F77DFF45EA04004E
:109A900015B0F0BD10B51022037811F8014B6340EA
:109AA000521E00F8013BF7D110BD70B50C468CB0CA
:109AB000154601461E461022FFF770FF0822214678
:109AC00004A8F6F760FF00F00BF8FFF785FF0446E7
:109AD000102208A93046F6F756FF20460CB070BD9C
:109AE0000822294606A8F6F74EBF70B504460D4673
:109AF00000260BE0F6F779FFF6B2010AA155761CB5
:109B0000F1B2A94202D2F6B2A055761CF0B2A84238
:109B1000F0D370BD00688208920000F0030102F0EB
:109B200004021143C208D20002F0080211430209E4
:109B3000120102F010021143400941EA4010C0B284
:109B400070470268920841EA820222F004038A0800
:109B500002F0010243EA820222F00803CA0802F07E
:109B6000010243EAC20222F0F0030A0902F00102F4
:109B700043EA0212490942EA41110160704700F1CB
:109B8000200200F11001FFF7A5BE2DE9F047070004
:109B9000144614BF002C022088B089463FD009F13A
:109BA0000405A8B2FCF780FF060036D0FBF7F9FCED
:109BB00080464A463946301DF6F7E5FE86F80380B2
:109BC0004FEA1827B7704FEA184986F801904FEA14
:109BD000186A86F800A0FBF7E1FC0146102203A8F2
:109BE000F6F7D1FE0820009001ABAAB2314603A8D7
:109BF00000F085F805000DD184F80080677084F8C6
:109C0000029084F803A0082201A9201DF6F7BBFEEC
:109C1000FBF7CBFC00F070F800E01325284608B0F5
:109C2000BDE8F0872DE9F04F89B015001CBF129FE9
:109C3000002F80460E469A4615D0FCF758FE0400C9
:109C400008BF142055D03878797800EB0120B97816
:109C500000EB0140F97800EB0169A06A484504D3A4
:109C600010F1010F01D0022043E026B120798007D6
:109C700058BF01203DD50822002101A8F6F7ABFE10
:109C80000AF1040B1FFA8BF0FCF70EFF060008BF69
:109C900013202ED052462946301DF6F774FE0422BA
:109CA00039463046F6F76FFE102204F1180105A878
:109CB000F6F769FE0820009001AB1FFA8BF23146DF
:109CC00005A800F01CF8050010D1082201A903A87E
:109CD000F6F759FE0822391D03A8F6F76EFE012893
:109CE00011BF012549464046FBF762FE00F004F82B
:109CF000284609B0BDE8F08F3046FCF7E2BE2DE9FA
:109D0000FA4F834685B0924600F0D6F8814600F0BF
:109D1000D3F8B9F1000F804608BF132400F0C280C9
:109D2000B8F1000F08BF132400F0B98000F0C4F8A8
:109D3000064600F0C1F805460EB9132434E00DB90B
:109D400013242FE010220021F6F745FE3246294663
:109D50005846FFF718FF040024D130780FF294170B
:109D6000000604D44946304600F0B7F808E029461A
:109D7000304600F0B2F84A463946284600F0A3F8CB
:109D800099F80000000604D44146484600F0A5F8C2
:109D900008E02946484600F0A0F8424639462846E1
:109DA00000F091F8FFF7A8FF15B12846FCF789FEEF
:109DB000200074D100F080F8054600F07DF80646DA
:109DC0000DB9132468E00EB9132462E0514601F185
:109DD0000F00C21000EB12700003001403D14FF00B
:109DE000000A00220AE0CA0801EB12721209A1EB74
:109DF0000212521E9241D20FA0F1010A4FEA0A103C
:109E0000059B80B2184422B13246494600F05BF807
:109E100018E0CA0801EB12721209A1EB021100222C
:109E2000C9B28A42B8BF835C02DB0CBF8023002327
:109E30000DF80230521C102AF3DB324641466846C8
:109E400000F041F8102200212846F6F7C4FD002753
:109E50000BE00598390189B201446A46284600F0B2
:109E600032F800F02CF804467F1C3FB2574501DA67
:109E70002000EED020000CD16A463146284600F082
:109E800022F800F01CF80446109A06982946F6F7C6
:109E900070FD2846FCF715FE0EB1FFF72DFF484672
:109EA000FCF70FFEB8F1000F1CBF4046FCF709FE9F
:109EB000204607B0BDE8F08F1020FCF7F5BD2A461C
:109EC000694658465FE630B50023C45CCD5C6C4003
:109ED000D4545B1C102BF8DB30BD10B500220F23CF
:109EE000C45C42EA4402CA54C25CD2095B1EF7D584
:109EF00010BD000000000000000000000000000095
:109F0000000000872DE9F047DFF860670446002570
:109F10003068884692461F46A94608B1112036E0AF
:109F20006FB12120FBF7F3F997F89C10814206D31B
:109F30002220FBF7ECF997F89C10884201D202200E
:109F400025E07020FCF7B0FD306008B913201EE05A
:109F500070220021F6F73FFD31684D7030680470C3
:109F6000306880F802803068A0F806A08766C56671
:109F700005711CB100F0D3F90546A94631680120EE
:109F80004870B9F1000F18BF00F001FB2846BDE88A
:109F9000F08738B5DFF8D4562B68002443B11A791E
:109FA000022A18BF032A05D0042A18BF062A01D0A6
:109FB000122032BDDA888A4201D0022032BD014629
:109FC000102203F10800F6F7D4FC2868102128308D
:109FD000FFF78BFD286800F1180200F12801083016
:109FE00000F016F92868417802781AB103290DD1DA
:109FF000022107E0042902D10221417006E0032971
:10A0000004D10521417000F0A0F90446204632BD7C
:10A01000DFF8581648607047DFF85026126802B91A
:10A02000704780B5D288824208BF012904D100F070
:10A03000AEFABDE801402FE301BD1720CCE20000DD
:10A0400070B586B0044600208DF80000A068057841
:10A05000691E0A293BD8DFE801F006060F13171B1B
:10A060001F23272B2F0001A900F095FB122826D1D2
:10A0700006218DF8001022E001A900F0FFFB1EE090
:10A0800001A900F017FC1AE001A900F02AFC16E073
:10A0900001A900F03EFC12E001A900F057FC0EE01F
:10A0A00001A900F07DFC0AE001A900F084FC06E0B3
:10A0B00001A900F097FC02E001A900F0ACFCD8B9BE
:10A0C0006088FCF714FC052628B9082612E0072052
:10A0D0008DF8000013E0827CDFF89015082A0CBF91
:10A0E0008968496831B10B68190003D001AA294673
:10A0F000984706468DF800609DF8000020B1608802
:10A10000694600F007F803E00B2D18BFFFF72DFCA0
:10A1100006B070BD38B50C46DFF854352246022132
:10A1200000F087FC0546207800F056FA284632BD3C
:10A1300070B5DFF838450646206800280D463FD048
:10A14000C188B1423CD14178062930D1017811B3A0
:10A15000816ED1F89810C26ECB0704D5137BDB0754
:10A1600048BF072113D4C1F34003002B1FBFD3689E
:10A17000C3F34003002B092109D1C1F38001002959
:10A180001EBFD168C1F38001002902D00B214170AC
:10A1900007E0A06800E0606818B14068010018BFDF
:10A1A000804720684078122818D1002005E0112946
:10A1B00006D1280018BF3225284600F00DFA0DE020
:10A1C000280007D13046FCF792FB18B1017941F025
:10A1D0001001017131462846FBF7BFFD012070BD1B
:10A1E00010B5DFF88844206888B1007800280CBFDB
:10A1F0006068A06818B14068010018BF80472068F7
:10A200004078122803D1BDE810400020E4E110BDE1
:10A210002DE9F34FDFF8546430688DB0904608B9EB
:10A22000122041E0C088FCF762FB050008BF142043
:10A230003AD009A800F0F9F93068017879B1D0F87E
:10A240006CA0FBF7BFF9040018BF01240020FBF746
:10A25000BCF96F7909AE814605F1060B0EE0C66EBA
:10A26000FBF7B0F9070018BF01270020FBF7ADF995
:10A270006C790DF1240A834605F1060907A95046B9
:10A2800000F032FA05A9304600F02AFACDF8108025
:10A29000CDF80CB00297CDF8049000940E990D986B
:10A2A00005AB07AAFFF79AFB0FB0BDE8F08F70B5BA
:10A2B000DFF8B8530446686886B000281CBF006801
:10A2C00000280E461CD030788DF8040070788DF888
:10A2D000050002A8B178FFF734FCF0786B688DF8C0
:10A2E0000C0001AA7068049001211B682046984761
:10A2F000010005D08DF8000069466088FFF70AFF6D
:10A3000006B070BD38B5D94CA46834B1A5682C002E
:10A3100003D0049C0094A84732BD022032BD1FB573
:10A3200000F031F870B1684600F07FF92168C88804
:10A330000978002914BFCF4BCF4B6A46072100F0A4
:10A3400078FB00E0012004B010BD1FB500F01BF841
:10A3500000F1180110226846F6F70BFB2068C74B86
:10A360000AE01FB500F00FF800F12801102268463E
:10A37000F6F7FFFA2068C24BC0886A46112100F048
:10A3800058FB04B010BDB94C20687047F8B5B74F02
:10A3900004463868C06E0025002840F0C4801020B4
:10A3A000FCF782FB39680028C86600F0BA808E6E20
:10A3B00010222146F6F7DDFA38680178002940F0CE
:10A3C0008880C16ED6F8982011F80C7F02F0010346
:10A3D00007F00107BB4218BF0023520843EA4202BC
:10A3E000C6F89820C2F340030F68C7F34007BB428A
:10A3F00006BF530803F00103002322F0020242EAE1
:10A400004302C6F89820C2F380030F68C7F38007A1
:10A41000BB4206BF930803F00103002322F00402AD
:10A4200042EA8302C6F89820C2F3C0030F68C7F35C
:10A43000C007BB4206BFD30803F00103002322F08C
:10A44000080242EAC302C6F89820C2F300230F684C
:10A45000C7F30027BB4206BF130A03F00103002322
:10A4600022F4807242EA0322C6F89820C2F3402305
:10A470000F68C7F34027BB4206BF530A03F001032E
:10A48000002322F4007242EA4322C6F89820C2F365
:10A4900080230F68C7F38027BB4206BF930A03F0EF
:10A4A0000103002322F4806242EA8322C6F8982046
:10A4B000C2F3C0230968C1F3C0218B4206BFD10A91
:10A4C00001F00101002122F4006242EAC121C6F834
:10A4D0009810617800291EBF7178002905211CD1D0
:10A4E0006168C1F3800139B996F8951011F0040143
:10A4F00008BF012111D012D00178002919BF31788D
:10A500002278327821780529B8BF052A07DA0FF2B8
:10A51000B41302EB82021A44515C017104E0182565
:10A5200002E0132500E011252846F2BD0A46554BEE
:10A5300015E010B586B00446ADF80010104601468F
:10A5400008220DF10200F6F714FA4F4B6A460B2170
:10A55000204600F06EFA06B010BD0A464B4B1121A2
:10A5600000F067BA1CB58DF800100446104601468D
:10A5700006220DF10100F6F7FCF9454B6A46082169
:10A58000204600F056FA13BD0A46424BE7E710B5E5
:10A59000FFF7F9FEE0B1C06E08B1FCF792FA20684F
:10A5A000806D08B1FCF78DFA2068C06D08B1FCF72A
:10A5B00088FA2068006E08B1FCF783FA2068406EC4
:10A5C00008B1FCF77EFA2068FCF77BFA00202060D7
:10A5D000BDE81040FFF7D7B9244900B5096885B038
:10A5E00081B14A6E03920A6E0292CA6D01928A6D1F
:10A5F0000092CB78CA880978FBF739FC05B05DF882
:10A6000004EBC4E705B000BD184909681020002913
:10A610001CBFCA6E002A07D0896E29B191F89C0030
:10A62000117A814238BF0846704770B504460F481A
:10A63000006800281CBF856E002D0FD02878207080
:10A6400005F1950668786070201D3178FFF779FA7A
:10A65000F0792072D5F89800E06070BD2046BDE822
:10A66000704010220021F6F7B6B90000CC48002057
:10A67000CBA80100E1A60100E9A601006BA801003A
